:020000040800F2
:100000000000011099CD0308D11D030895C5000813
:100010009DCE03089DCE03089DCE0308000000007E
:100020000000000000000000000000001924030888
:100030001524030800000000112403082D93000874
:100040009DCE03089DCE03089DCE03089DCE0308D8
:100050009DCE03089DCE03083D9E00082D9F0008FD
:100060009DCE0308F19E0008B59E000849B800081F
:1000700039B8000829B8000819B8000809B80008FC
:10008000F5B70008E1B700089DCE03089DCE030830
:100090009DCE03089DCE03089DCE0308799E0008DF
:1000A0009DCE0308C1CB00089DCE0308D1CB00082C
:1000B000B1CB0008A1CB00089DCE030825BE0008E7
:1000C0002DBE000819BE000821BE00089DCE030801
:1000D0009DCE0308999400089DCE0308FD93000867
:1000E000019E00089DCE0308892F030861CB0008FC
:1000F00071CB00089DCE030881CB0008CDB7000866
:100100009DCE03089DCE030891CB00089DCE030829
:100110009DCE03089DCE03089DCE03089DCE030807
:10012000B9B70008A5B7000891B700087DB7000867
:1001300069B700089DCE03089DCE03089DCE030835
:100140009DCE03089DCE03089DCE0308D51D030850
:1001500055B7000841B700082DB7000861930008A3
:100160000DBE000815BE00089DCE03089DCE0308F5
:100170009DCE03089DCE03089DCE03089DCE0308A7
:080180009DCE03089DCE03088B
:10018800020203007C1E0020781E002000000000F0
:100198000000000016000800881E0020901E0020A5
:1001A80000000000E80500081D000100CC22002026
:1001B8005C23002000000000F00500082700040070
:1001C800EC2200206023002000000000F205000857
:1001D8000300010020250020282500200000000041
:1001E8000000000001010400902A00202C390020A2
:1001F800000000000000000008020900D8380020B4
:100208003039002000000000D781000806020C00E9
:10021800E13800203C39002000000000238F00084E
:1002280007020200143900204839002000000000AD
:10023800F6050008FF0101002A3900204C3900208A
:1002480000000000F805000802000C00F03800204B
:1002580050390020000000000000000003123200A6
:10026800723B0020403B002000000000000000001E
:1002780025005A008C3A0020E63A002000000000D1
:1002880000000000F60108005C390020843A0020D4
:1002980000000000000000000E00DE00083C002006
:1002A800384A002000000000C5E9020813000400D5
:1002B800583D0020184B002000000000FC050008F5
:1002C80002010300F73B00201C4B00200000000047
:1002D80091E001081E000400EC4C0020D44E0020E0
:1002E800000000000006000822000C00584C002006
:1002F800D84E002000000000040600081F000E0071
:10030800545000207450002000000000100600081F
:100318000502010040500020845000200000000029
:100328001E06000803010600CE4F0020885000205A
:1003380000000000200600082C00100034540020A3
:100348002454002000000000999302082B00240088
:1003580068540020445400200000000069930208FB
:100368001B00F40040580020345900200000000011
:10037800995E02080B100C00AC560020285A002089
:10038800000000002606000801000A00AC640020F6
:10039800B864002000000000320600081A000800B7
:1003A80094640020C4640020000000003C0600089B
:1003B8002A0060002C650020CC64002000000000AA
:1003C80059E9020815007000585D00208C6500206E
:1003D800000000000000000029005000C86800204C
:1003E8001C6900200000000000000000140002004A
:1003F800C46800206C690020000000004406000862
:1004080010000300B8680020706900200000000098
:100418004606000828000C00AC680020746900201B
:10042800000000004A06000826000800A468002012
:1004380080690020000000005606000823000E0016
:10044800946800208869002000000000DD87020809
:10045800190005008C680020986900200000000041
:100468005E060008F801010088680020A0690020E5
:1004780000000000640600080001040084680020F1
:10048800A4690020000000006606000818002C007F
:100498000C7500203875002000000000599C0208E7
:1004A80006001A003070002064750020000000006B
:1004B800E5E90208340010005C6F00208075002018
:1004C8000000000081E90208FB010100386E0020ED
:1004D80090750020000000002DBF0008FC010900F5
:1004E800006D00209475002000000000F9BE00088F
:1004F800F7010600F86C0020A0750020000000003D
:100508006A060008050005004D760020A876002040
:1005180000000000700600080400C00024A40020A9
:1005280018A600200000000000000000F9010400E7
:10053800D8860020D8A6002000000000C981000845
:100548000A001200F8B9002040C200200000000094
:10055800760600080D003400C4B9002054C20020FB
:100568000000000029C5010811000C0058AE002049
:1005780088C2002000000000DDC40108FD0124003D
:100588004CA7002094C200200000000059810008F8
:10059800FE01080038A70020B8C2002000000000B3
:1005A80035BF000812001600E8C2002054C300201E
:1005B80000000000880600080C002400FEC200208D
:1005C8006CC300200000000069E00108000205007B
:1005D800C0C2002090C300200000000000000000FE
:1005E800C409000019012828000020030000013C6C
:1005F800010000000801000000000100C800141EEE
:10060800010064002C012800000000000000010027
:1006180000000005000000000401010000002B217B
:10062800231E0002000001000A010A0AE803000074
:10063800640001007E05EA05B405320003000001EC
:100648000500000000010000000000000000011586
:100658005802D903C50300002801000004009001D6
:100668000000240100000000010102000100003028
:100678000100005A0000000090012C01C80064002D
:100688000000000100000000000000000000000061
:060698000000000000005C
:10069E000000803F0000803F0000803F50010000BE
:1006AE000700000002000000000000000000000033
:1006BE000102030406070809FF0100000000803F45
:1006CE000000803F81AC020839AC020889AB0208F9
:1006DE0000000000F5A80208DDAA02085DAB0208C2
:1006EE0045AA02080000000000000000E9A8020868
:1006FE00C51B0308C11B0308BD1B0308B11B030860
:10070E00AD1B0308B91B0308B51B0308D51B030853
:10071E00C91B0308591C03086D1C0308451C03085C
:10072E00311C03081D1C0308800004080508040082
:10073E00000000002C090408C40804086C0004081A
:10074E0000000000AC00040805080A0000000000CC
:10075E002C090408C4080408F81D04080000000051
:10076E00006002401060024000000000000B00001C
:10077E0000002000000000000000000000600240A9
:10078E002860024000000000060C0000000020005F
:10079E0000000000000000000060024040600240C7
:1007AE0000000000100D00000000200000000000FE
:1007BE00000000000060024058600240000000008F
:1007CE00160E0000000020000000000000000000D7
:1007DE00006002407060024000000000200F000028
:1007EE000000200000000000000000000060024039
:1007FE00886002400000000026100000000020006B
:10080E00000000000000000000600240A0600240F6
:10081E000000000030110000000020000000000069
:10082E000000000000600240B860024000000000BE
:10083E00362F000000002000000000000000000025
:10084E000064024010640240000000000038000006
:10085E0000004000000000000000000000640240A4
:10086E00286402400000000006390000000040002D
:10087E0000000000000000000064024040640240DE
:10088E0000000000103A00000000400000000000D0
:10089E0000000000006402405864024000000000A6
:1008AE00163B0000000040000000000000000000A9
:1008BE00006402407064024000000000203C000012
:1008CE000000400000000000000000000064024034
:1008DE008864024000000000264400000000400032
:1008EE00000000000000000000640240A06402400E
:1008FE000000000030450000000040000000000035
:10090E000000000000640240B864024000000000D5
:10091E00364600000000400000000000000000000D
:10092E00FFFFFFFF00000101FFFF00000000803FFE
:10093E00703C04080E00000019710208000000004F
:10094E000000000020040020343C040800000000D9
:10095E00000000000000000000000000905E04088F
:10096E000000000000000000AB04002004000000A6
:10097E00C03B04080C000000E1790208E8080020E2
:10098E0000000000E43A04080C000000B9790208E7
:10099E00DC08002000000000543C040808000000A1
:1009AE0000000000D008002004000000443C0408B1
:1009BE000C00000039850208C40800200000000069
:1009CE00D03A040803000000A9650308AC08002013
:1009DE00000000004C3C040803000000A965030859
:1009EE009408002000000000D43A04080100000022
:1009FE0000000000000000000000000000000000E9
:100A0E000D000000000000000000000000000000CB
:100A1E00343C04080000000000000000000000004C
:100A2E0000000000905E04080000000000000000BE
:100A3E00AB04002004000000643B04080300000027
:100A4E00FD7602087C08002008000000443C0408E3
:100A5E000C00000039850208C408002000000000C8
:100A6E00D03A040803000000A9650308AC08002072
:100A7E00000000004C3C040803000000A9650308B8
:100A8E009408002000000000D43A04080100000081
:100A9E000000000000000000000000000000000048
:100AAE000D0000000000000000000000000000002B
:100ABE005C3C040800000000000000000000000084
:100ACE0000000000905E040800000000000000001E
:100ADE00AB040020040000006C3B0408030000007F
:100AEE00A9650308F408002000000000D43A0408A9
:100AFE0001000000000000000000000000000000E7
:100B0E00000000000D0000000000000000000000CA
:100B1E000000000000FFFF0000000000AA550300C7
:100B2E009FAA5505010000AA550B010000AA550702
:100B3E00010000AA550902000000012D202D2D20D4
:100B4E002D2D2D2D202D2D2D00000000000000003C
:100B5E00000000000000000000002D202D2D202D93
:100B6E002D2D2D202D2D2D2D00000000000000001C
:100B7E000000000000000000000000000100000066
:100B8E00C0120000EE4E002088130C17010000006A
:100B9E00F04E002088130C1700000000A83A04083D
:100BAE000000000000000000000000000000000037
:100BBE00B83A0408080000000000000000050020FC
:100BCE0004000000C43A0408080000000000000001
:100BDE00F404002000000000D03A040804000000D5
:100BEE005D7402080000000000000000D43A040802
:100BFE0001000000000000000000000000000000E6
:100C0E00000000000D0000000000000000000000C9
:100C1E0000000000EC4E002088130C1701000000AD
:100C2E00EA4E002088130C1700000000143B040845
:100C3E000E000000697102080000000000000000B4
:100C4E000C050020184F002001000000EC080408DD
:100C5E00E94E002001000000F8080408F24E0020C2
:100C6E000200000000090408DEA5002000000000BC
:100C7E0000000000DCA500200000000000000000C5
:100C8E00DAA500200000000000000000D8A500201A
:100C9E000000000000000000D6A5002000000000AB
:100CAE0000000000D4A5002000000000000000009D
:100CBE00F00400200000000000000000E84E0020BC
:100CCE00020000000C0904081C3B04080000000090
:100CDE00000000000000000000000000B83A040808
:100CEE000800000000000000900500200400000035
:100CFE00C43A04080800000000000000840500202B
:100D0E0000000000D03A04080400000049710208F7
:100D1E000000000000000000D43A040801000000AA
:100D2E0000000000000000000000000000000000B5
:100D3E000D00000000000000000000000000000098
:100D4E002C3B040800000000000000000000000022
:100D5E00000000003C3B04080C00000089730208F0
:100D6E00CC05002004000000483B04080C000000E5
:100D7E008D710208C005002004000000543B0408D9
:100D8E000C0000004D730208B405002000000000A6
:100D9E00603B0408030000001D7702089C0500203C
:100DAE00080000006C3B040803000000A96503085E
:100DBE00F408002000000000D43A040801000000EE
:100DCE000000000000000000000000000000000015
:100DDE000D000000000000000000000000000000F8
:100DEE00743B04080000000000000000000000003A
:100DFE00000000007C3B040804000000C9840208C7
:100E0E000000000000000000D43A040801000000B9
:100E1E0000000000000000000000000000000000C4
:100E2E000D000000000000000000000000000000A7
:100E3E00C83B040800000000000000000000000095
:100E4E0000000000143604080C0000000000000032
:100E5E002C06002004000000D83B04080800000007
:100E6E00000000002006002004000000E43B0408FF
:100E7E00080000000000000014060020040000001E
:100E8E00EC3B0408080000000000000008060020EB
:100E9E0004000000F43B04080800000000000000FD
:100EAE00FC05002004000000FC3B040808000000C4
:100EBE0000000000F005002004000000043C0408BF
:100ECE000800000000000000E405002004000000FF
:100EDE000C3C04080800000000000000D8050020AB
:100EEE0004000000D43A04080100000000000000D5
:100EFE000000000000000000000000000D000000D7
:100F0E00000000000000000000000000143C040877
:100F1E000E000000597102080000000000000000E1
:100F2E00380600201C3C04080E00000000000000E3
:100F3E000000000000000000B0060020243C040861
:100F4E000E00000000000000000000000000000085
:100F5E00500700203C50002004000000180904082F
:100F6E00E44E0020E0150C1700000000E74E0020B4
:100F7E0008000000C4080408E64E0020050000002A
:100F8E002C0904082C3C04080E0000000000000090
:100F9E000000000000000000A0070020010100007A
:100FAE00518E020800000000000000000100000049
:100FBE0009024300020100C03209040000010202CE
:100FCE000100052400100105240100010424020281
:100FDE000524060001070582030800FF090401002D
:100FEE00020A000000070501024000000705810209
:100FFE0040000000FF00000001000000C83304089C
:10100E000000000000000000A5E00108A08601001D
:10101E0004000000000000000000000000000000BE
:10102E0000000000000000000000000000000000B2
:10103E00545604082C330408000000002D770108D4
:10104E007D0000000600000000000000000000000F
:10105E000000000000000000000000000000000082
:10106E0000000000943C0408000000000000000096
:10107E00B10C0108E80300000300000000000000AE
:10108E000000000000000000000000000000000052
:10109E0000000000000000009C3C0408000000005E
:1010AE0000000000EDEA0208102700000300000017
:1010BE000000000000000000000000000000000022
:1010CE00000000000000000000000000A83C040822
:1010DE000000000041920208EDE60008204E0000DC
:1010EE0005000000000000000000000000000000ED
:1010FE0000000000000000000000000000000000E2
:10110E0020350408000000000000000065070108FB
:10111E001027000001000000000000000000000089
:10112E0000000000000000000000000000000000B1
:10113E0000000000AC3C04080000000000000000AD
:10114E00C5BE0008E8030000050000000000000016
:10115E000000000000000000000000000000000081
:10116E000000000000000000B83C04080000000071
:10117E00000000005DE30108204E000003000000A7
:10118E000000000000000000000000000000000051
:10119E00000000000000000000000000C83C040831
:1011AE00000000000000000065E10108204E000074
:1011BE00030000000000000000000000000000001E
:1011CE000000000000000000000000000000000011
:1011DE00D83C04080000000000000000BD05010816
:1011EE00400D03000300000000000000000000009E
:1011FE0000000000000000000000000000000000E1
:10120E0000000000E82804080000000000000000B4
:10121E004DDC010810270000010000000000000056
:10122E0000000000000000000000000000000000B0
:10123E000000000000000000383304080000000029
:10124E0000000000D59A03081027000003000000DC
:10125E000000000000000000000000000000000080
:10126E00000000000000000000000000E83C040840
:10127E000000000000000000DDBF0308A086010092
:10128E00010000000000000000000000000000004F
:10129E000000000000000000000000000000000040
:1012AE0088280408000000000000000005BF0308A5
:1012BE0050C300000100000000000000000000000C
:1012CE000000000000000000000000000000000010
:1012DE0000000000F03C04080000000000000000C8
:1012EE0075BA0308A86100000100000000000000AC
:1012FE0000000000000000000000000000000000E0
:10130E000000000000000000FC3C0408000000008B
:10131E0000000000E1A50308A08601000100000006
:10132E0000000000000000000000000000000000AF
:10133E000000000000000000000000002C2904083E
:10134E000000000000000000E1290108A00F0000CD
:10135E00010000000000000000000000000000007E
:10136E00000000000000000000000000000000006F
:10137E00083D04080000000000000000B1580208FB
:10138E001027000001000000000000000000000017
:10139E00000000000000000000000000000000003F
:1013AE0000000000A434040800000000000000004B
:1013BE000DC40108A00F0000010000000000000095
:1013CE00000000000000000000000000000000000F
:1013DE00000000000000000080350408000000003E
:1013EE00000000000975020810270000010000002F
:1013FE0000000000000000000000000000000000DF
:10140E00000000000000000000000000203304086F
:10141E000000000000000000916903081A4100005E
:10142E0001000000000000000000000000000000AD
:10143E00000000000000000000000000000000009E
:10144E00143D0408000000000000000051C1030814
:10145E00400D03000000000000000000000000002E
:10146E00000000000000000000000000000000006E
:10147E00000000001C3D04080000000000000000F9
:10148E0051E50108A08601000300000000000000E5
:10149E00000000000000000000000000000000003E
:1014AE000000000000000000303D0408905E0408BB
:1014BE000000000000000000403D0408483D040804
:1014CE0000000000012000004C3D0408543D0408BB
:1014DE000000000001400000583D04084050040880
:1014EE000000000001200000643D0408703D040867
:1014FE000000000004000000743D0408803D040854
:10150E000000000004000000843D0408B4460408F6
:10151E000000000001000000010200000000803FFA
:10152E000101010000000000010203040102030496
:10153E000607080904030904120100020202004012
:10154E0083044057000201020301000049AE020865
:10155E0069AD0208C110030839A9020815AD0208C9
:10156E0049A9020865A9020829A9020819A90208B1
:10157E000000000000000000000101010100000059
:10158E0020700020702D7200105C04080E00000008
:10159E00000000000000000000000000DC1B002026
:1015AE00FFFFFFFFFA000000010000000100000035
:1015BE00743B040800000000000000000000000062
:1015CE0000000000EB57040804000000EB0D0308B8
:1015DE000000000000000000D43A040801000000E2
:1015EE0000000000000000000000000000000000ED
:1015FE000D000000000000000000000000000000D0
:10160E0096A500200100C4090000000094A500204A
:10161E000100C4090000000092A500200100C409C9
:10162E000000000090A500200100C4090000000089
:10163E008CA500200100C409000000008EA500202A
:10164E000100C409000000008AA500200100C409A1
:10165E000000000088A500200100C4090000000061
:10166E000C5804080E0000000000000000000000EE
:10167E0000000000200F0020105000209CFF2C01C5
:10168E0000000000900E00200A000000F81D040863
:10169E00D84F0020E0150C1700000000910E00201E
:1016AE0008000000C4080408920E00200500000087
:1016BE002C0904080B66002002000000101E04080E
:1016CE005376002001200100527600200200000017
:1016DE001C1E0408EE3C00200000F4010100000076
:1016EE00EC3C00200000F40101000000EA3C002068
:1016FE000000F40101000000E83C00200000F401AD
:10170E0001000000E63C002000FF0100BA75002039
:10171E00E803D0070A000000B8750020006401003D
:10172E000A000000B9750020006401000A000000E4
:10173E00B2750020006401000A000000B775002099
:10174E00006401000A000000B6750020006401006C
:10175E000A000000B5750020006401000A000000B8
:10176E00B175002000FF01000A000000B0750020D6
:10177E0000FF01000A000000043C00200000F401FC
:10178E0001000000023C00200000F40101000000F6
:10179E00003C00200000F40101000000FE3B002090
:1017AE000000F40101000000AD75002000C801002A
:1017BE00AC75002000C80100AB75002000C8010008
:1017CE00AA750020006401000A000000A97500201F
:1017DE0000FF01000A000000C575002000C80100CE
:1017EE00C475002000C80100C375002000C80100A8
:1017FE00C275002000C80100C175002000C801009C
:10180E00C075002000C80100BF75002000C801008F
:10181E00BE75002000C80100BD75002000C8010083
:10182E001458040800000000000000000000000032
:10183E000000000024580408090000000000000009
:10184E00C40F0020040000002C58040809000000FA
:10185E0000000000B80F002004000000C85A040861
:10186E000900000000000000AC0F00200400000082
:10187E00345804080900000000000000A00F0020EA
:10188E0004000000385804080900000000000000A1
:10189E00940F0020040000004058040809000000C6
:1018AE0000000000880F00200400000048580408C3
:1018BE0009000000000000007C0F00200400000062
:1018CE00505804080900000000000000700F0020AE
:1018DE0004000000D43A04080100000000000000DB
:1018EE000000000000000000000000000D000000DD
:1018FE00000000000000000000000000585804081E
:10190E0000000000000000000000000000000000C9
:10191E00685804080500000000000000FD3B002090
:10192E0000000000D43A040801000000000000008E
:10193E000000000000000000000000000D0000008C
:10194E0000000000000000000000000070580408B5
:10195E000000000000000000000000000000000079
:10196E00905E04080000000000000000CA04002081
:10197E00040000007C5804080C000000A50D0308AC
:10198E002410002000000000C03B04080C000000E2
:10199E00990E03081810002000000000E43A040815
:1019AE000C0000007D0E03080C100020000000004B
:1019BE00543C040808000000000000000010002045
:1019CE0004000000443C04080C000000610D0308F4
:1019DE00F40F0020000000008058040809000000E9
:1019EE0000000000E80F002004000000D03A0408B8
:1019FE0003000000A9650308D00F002000000000BE
:101A0E00D43A0408010000000000000000000000AD
:101A1E0000000000000000000D00000000000000AB
:101A2E0000000000000000008858040800000000BC
:101A3E00000000000000000000000000985804089C
:101A4E000C00000000000000381000200000000014
:101A5E00A05804080A000000000000005476002080
:101A6E0000000000AC5804080A000000000000004E
:101A7E005C76002000000000B45804080A00000044
:101A8E00000000006476002000000000BC5804082E
:101A9E0007000000000000003010002000000000D1
:101AAE00D43A04080100000000000000000000000D
:101ABE0000000000000000000D000000000000000B
:101ACE000000000000000000C858040800000000DC
:101ADE00000000000000000000000000DC580408B8
:101AEE00070000000000000074100020000000003D
:101AFE00E8580408080000000000000068100020EC
:101B0E0000000000F4580408080000000000000067
:101B1E005C100020000000000059040808000000BE
:101B2E000000000050100020000000000C590408B6
:101B3E00080000000000000044100020000000001B
:101B4E00D43A04080100000000000000000000006C
:101B5E0000000000000000000D000000000000006A
:101B6E0000000000000000001859040800000000EA
:101B7E0000000000F30E00200000000024590408AD
:101B8E000B00000000000000DC1000200000000030
:101B9E002C5904080B00000000000000D01000209B
:101BAE0000000000385904080B000000000000007F
:101BBE00C410002000000000445904080B0000006F
:101BCE0000000000B810002000000000505904086A
:101BDE000B00000000000000AC1000200000000010
:101BEE005C5904080B00000000000000A01000204B
:101BFE0000000000645904080B0000000000000003
:101C0E009410002000000000705904080B00000022
:101C1E000000000088100020000000007C5904081D
:101C2E0008000000000000007C10002000000000F2
:101C3E00D43A04080100000000000000000000007B
:101C4E0000000000000000000D0000000000000079
:101C5E000000000000000000885904080000000089
:101C6E000000000000000000000000009C59040865
:101C7E0008000000000000000C1100200000000011
:101C8E00A859040808000000000000000011002000
:101C9E0000000000B4590408080000000000000015
:101CAE00F410002000000000C059040808000000D5
:101CBE0000000000E810002000000000D43A0408E4
:101CCE000100000000000000000000000000000005
:101CDE00000000000D0000000000000000000000E9
:101CEE0000000000C85904080000000000000000B9
:101CFE00F00E002000000000D85904080B00000070
:101D0E00000000003C11002000000000E45904080F
:101D1E000B00000000000000301100200000000049
:101D2E00F0590408070000000000000028110020F0
:101D3E0000000000FC59040807000000000000002D
:101D4E002011002000000000085A040807000000BF
:101D5E00000000001811002000000000D43A040812
:101D6E000100000000000000000000000000000064
:101D7E00000000000D000000000000000000000048
:101D8E0000000000145A04080000000000000000CB
:101D9E00F00E002000000000205A0408070000008A
:101DAE00000000008811002000000000285A0408DE
:101DBE00070000000000000080110020000000005D
:101DCE00305A0408070000000000000078110020BF
:101DDE0000000000385A0408070000000000000050
:101DEE007011002000000000405A04080700000097
:101DFE00000000006811002000000000485A04088E
:101E0E00070000000000000060110020000000002C
:101E1E00505A04080700000000000000581100206E
:101E2E0000000000585A04080700000000000000DF
:101E3E005011002000000000605A04080700000046
:101E4E00000000004811002000000000D43A0408F1
:101E5E000100000000000000000000000000000073
:101E6E00000000000D000000000000000000000057
:101E7E0000000000685A04080E0000000000000078
:101E8E00A93E02080000000090110020FB3B00203C
:101E9E000A320100FA3B002001FA0100F63B002055
:101EAE0000C80100F43B0020E803D0070100000049
:101EBE00414952424F54463453440000705A04086C
:101ECE000E000000BF3E0208000000007944020828
:101EDE006C120020785A04080E000000250E03082C
:101EEE000000000000000000BC120020805A040810
:101EFE000E0000004D67030825670308756403088C
:101F0E0098130020885A04080E000000F962030896
:101F1E00293F02080000000038140020905A0408DF
:101F2E000E00000079630308B1630308000000008F
:101F3E00D8140020AE750020010301009C5A04083D
:101F4E000E000000053F0208E13E020800000000FE
:101F5E00C8150020A45A04080E00000035630308BB
:101F6E00596603080000000054160020B05A0408F9
:101F7E000E000000D96303089D66030800000000F0
:101F8E00F4160020A875002001030100B85A0408B9
:101F9E000000000000000000000000000000000033
:101FAE00C45A0408080000000000000014180020A5
:101FBE0000000000CC5A04080700000000000000DA
:101FCE000C18002000000000DC5A04080700000076
:101FDE00000000000418002000000000E85A040869
:101FEE000700000000000000FC17002000000000A9
:101FFE00F45A040803000000A9650308E417002042
:10200E0000000000D43A04080100000000000000A7
:10201E000000000000000000000000000D000000A5
:10202E00000000000000000000000000FC5A040840
:10203E000000000000000000000000000000000092
:10204E000C5B04080A000000000000004028040891
:10205E0000000000145B04080A00000000000000ED
:10206E0040550408000000001C5B04080A00000034
:10207E0000000000C675002000000000245B04086C
:10208E000A000000000000002018002000000000E0
:10209E00D43A040801000000000000000000000017
:1020AE0000000000000000000D0000000000000015
:1020BE0000000000000000002C5B0408000000007F
:1020CE00000000000000000000000000602904086D
:1020DE0003000000A96503085C1800200000000042
:1020EE00405B040803000000A9650308A00200205D
:1020FE0000000000485B040803000000A965030807
:10210E004418002000000000505B0408030000008B
:10211E00A96503082C18002000000000D43A04081A
:10212E0001000000000000000000000000000000A0
:10213E00000000000D000000000000000000000084
:10214E00000000005C5B04080000000000000000BE
:10215E000000000000000000685B0408070000009B
:10216E00E5660308F4180020000000005456040829
:10217E0003000000A9650308DC1800200000000021
:10218E00745B040803000000A9650308C41800204E
:10219E00000000007C5B040803000000A965030832
:1021AE00AC18002000000000845B0408070000004B
:1021BE00CD660308A418002000000000DC3B0408D4
:1021CE0003000000A96503088C1800200000000021
:1021DE00905B040803000000A96503087418002032
:1021EE0000000000D43A04080100000000000000C6
:1021FE000000000000000000000000000D000000C4
:10220E000000000000000000000000009C5B0408BD
:10221E000E0000007D3E02084F3E02080000000046
:10222E00FC180020A45B04080E000000496403089B
:10223E0000000000000000009C190020B05B0408A4
:10224E000E00000000000000000000000000000072
:10225E00281A0020C05B04080E0000002164030849
:10226E000567030800000000B41A0020C85B0408CC
:10227E000000000000000000000000000000000050
:10228E00D45B040803000000A9650308C41B0020EA
:10229E0000000000B45B040803000000A9650308F9
:1022AE00AC1B002000000000DC5B040803000000F3
:1022BE00A9650308941B002000000000E85B0408D9
:1022CE0003000000A96503087C1B0020000000002D
:1022DE00F05B0408020000004168030800000000E3
:1022EE0000000000F85B04080200000041680308CB
:1022FE000100000000000000045C04080200000061
:10230E004168030802000000000000000000000009
:10231E000D000000000000000000000000000000A2
:10232E0001000000685E0C00430000000000000089
:10233E00000000000000000000000000000000008F
:10234E00000000000000000043000000000000003C
:10235E00000000000000000000000000000000006F
:10236E00000000000000000043000000000000001C
:10237E00000000000000000000000000000000004F
:10238E0000000000000000004300000000000000FC
:10239E00000000000000000000000000000000002F
:1023AE0000000000000000004300000000000000DC
:1023BE00000000000000000000000000000000000F
:1023CE0000000000000000004300000000000000BC
:1023DE0000000000000000000000000000000000EF
:1023EE00000000000000000043000000000000009C
:1023FE0000000000000000000000000000000000CF
:10240E00000000000000000079D30308B9D10308D2
:10241E00000000009C5E0408E6570408EA39040830
:10242E00EA390408EA390408EA390408EA390408E2
:10243E00EA390408EA390408EA390408EA390408D2
:10244E00FFFFFFFFFFFFFFFFFFFFFFFFFFFF00008C
:10245E000100415343494900000000000000000004
:10246E00000000000000000000000000000000005E
:10247E0000004153434949000000000000000000E5
:10248E00000000000000000000000000000000003E
:10249E0000000000081E00200000000000000000E8
:1024AE00000000000000000000000000000000001E
:1024BE00000000000000000000000000000000000E
:1024CE0000000000000000000000000000000000FE
:1024DE0000000000000000000000000000000000EE
:1024EE0000000000000000000000000000000000DE
:0C24FE00000000000000000001000000D1
:10800000436B826A816930B41C68456A24F00104BC
:108010001144AA421C60D9600DD3016900248A1A58
:108020005A6084621A68002142F0010280F84C1004
:1080300030BC1A607047AA1A5A608562F2E700BF26
:10804000436A8269F0B4D154436A0469426B0133D4
:10805000A34228BF00234362FAB1116811F0010165
:1080600001D0F0BC7047856A1768866927F0010760
:108070002E449D421760D6600BD3641B546081620E
:108080001368002143F0010380F84C10F0BC13602A
:1080900070475D1B55608362F2E7826DD36843F0E1
:1080A0008003D360DDE700BF026B10B462B1836C64
:1080B000C2684469D11A013B615C5DF8044B08BF9A
:1080C00013468364C8B27047016A4369C4685B5C45
:1080D0000131A14228BF114601625DF8044BD8B2BC
:1080E000704700BF436B13B190F84C007047836A30
:1080F000406A181AB0FA80F040097047416A836AF2
:1081000099420AD3CB1A416B026961B14968501E8A
:108110000B4483420AD2C01A704702691144CB1A39
:10812000416B0029F2D1501EC01A704700207047E1
:10813000036B43B1826C5B6893422FBF981AC0688F
:108140009B1AC0187047C269036A9A422FBFD01A9F
:10815000C0688018C01A70470A4B30B503F1140488
:1081600093F900205D78072AC8BF143A81180433B8
:108170000D7313F8025C855413F8012C0A76A342A0
:10818000EED130BD44F8030803682DE9F041DF6902
:108190001FB13B46BDE8F0411847002A164611DDE5
:1081A00004460D460E4400E023689B68204698472D
:1081B0000028F9D0236815F8011B1B682046984752
:1081C000AE42F1D1BDE8F081002325220270437058
:1081D0008370C3707047152303701623C370172371
:1081E00083713A2383703B2343713C2303727047AE
:1081F000F0B5446814B12568A4886C8341F080010F
:10820000046840F2E93501E0002D54D02689013D93
:1082100016F0020FADB2F7D089B2A18140F2E93178
:1082200001E0002958D02589013915F0010F89B2E4
:10823000F7D0A189A1894FF0000C4FF47A714FF665
:10824000FF764FF0FF0E624502D12DE0B1421BD008
:108250002589013915F0020589B2F7D0A4F80CE0A0
:108260004FF47A7102E0B9B2B1420DD0258915F010
:10827000010501F1FF37F6D0A589ADB20BB11D7034
:1082800001330CF1010CDEE71B4B9C4204D0A3F53B
:1082900074439C4208D10225184B03EB05156B89EA
:1082A00001339BB26B816B89436813B11A689B8859
:1082B00013830120F0BD10498C4204D0A1F5744114
:1082C0008C42B7D102250D4901EB051569890131B1
:1082D00089B269816989ADE7074DAC4203D008498D
:1082E0008C42A7D10221054D05EB01114D890135C5
:1082F000ADB24D8149899DE70030014008C400209E
:10830000003C004030B4446814B12368A5885D8304
:10831000036840F2E93001E0002832D01D890138BD
:1083200015F0020F80B2F7D089B2998140F2E9319D
:1083300001E0002947D01889013910F0010F89B2F6
:10834000F7D0998940F2E93100E059B31889013931
:1083500010F0020F89B2F8D092B29A8140F2E9325D
:1083600001E0002A3FD01989013A11F0010F92B2C1
:10837000F7D09B8914B12368A2881A83012030BCEE
:10838000704721498B4204D0A1F574418B42D9D169
:1083900002201E4901EB00104189013189B241815F
:1083A0004189CFE7184A934204D0A2F57442934220
:1083B000E0D10221154B03EB01114B8901339BB234
:1083C0004B814B89D6E71048834203D010498B423A
:1083D000B8D102210D4800EB01114889013080B26B
:1083E00048814989AEE708498B4203D0084A934245
:1083F000C0D10222054B03EB0212538901339BB219
:1084000053815389B6E700BF0030014008C4002003
:10841000003C0040002870B51EDB0928044620DD22
:10842000012303EB83035B00B0FBF3F2092AF8D8C6
:108430007BB10E4EB4FBF3F00928CCBF572230229B
:10844000A6FB03E5024403FB1044EB0801F8012BF3
:10845000F0D100230B7070BD2D230B704042013111
:10846000DBE7303001F8010BF3E700BFCDCCCCCC1B
:10847000884230B44FF001042ED301FB04F4B0FB6A
:10848000F4F58D42F9D284B1AAB901E0B0FBF4F55C
:10849000092DCCBF572230222A4404FB150003F8D3
:1084A000012BB4FBF1F4002CF0D100221A7030BC87
:1084B0007047B0FBF4F5092DCCBF372230222A4497
:1084C00004FB150003F8012BB4FBF1F4002CF0D1F0
:1084D00000221A7030BC70470546002AEBD1D7E75E
:1084E00003685A1C02601970704700BF2DE9F047FD
:1084F000089C2578002B804689460CBF4FF0200A47
:108500004FF0300A661C35B3002A29DD334601E0FE
:10851000024698B113F8011B501E0029F8D1971E8E
:1085200060B13D46013D51464046C8476B1C002B9B
:10853000F8DC257827EAE770013055B1041B29469D
:108540004046C847301916F8015B002DF7D1BDE849
:10855000F087BDE8F087002A04DC2846BDE8F087F4
:108560000020EBE7571EDCE70A44914251D030B4BB
:1085700041F2210411F8013B80EA0320430010F48A
:10858000004F84EA03059BB2ADB208BF1D466B00E5
:1085900015F4004F84EA03009BB280B208BF18466E
:1085A000430010F4004F84EA03059BB2ADB208BF4C
:1085B0001D466B0015F4004F84EA03009BB280B2A5
:1085C00008BF1846430010F4004F84EA03059BB22D
:1085D000ADB208BF1D466B0015F4004F84EA0300DE
:1085E0009BB280B208BF1846430010F4004F84EAE3
:1085F00003059BB2ADB208BF1D466B0084EA0300C1
:1086000015F4004F85B298B218BF28468A42B1D1FE
:1086100030BC704783684268D0ED037A00EB830179
:108620000133934281ED040A836004BF0023836019
:1086300000EB830393ED047A036870EE277A9A4285
:10864000C0ED037A77EEC77AC0ED037A0CDA013316
:1086500007EE103AF8EEC76AB7EE007A87EEA60A80
:10866000036030EE070A704707EE102AB8EEC77AAB
:1086700087EE870A704700BF90ED097A90ED004AB7
:10868000D0ED0A6AD0ED014AD0ED047A90ED035A9C
:10869000D0ED025AA4EE007AB0EE406AB0EE470A7E
:1086A000B0EE667AA6EE247A67EEC07AA0EE457A3E
:1086B000E6EE257A80ED097AC0ED0A7A704700BFB0
:1086C000D0ED057A90ED013AD0ED003AD0ED064AB2
:1086D00090ED024A90ED077A90ED035A90ED086A0A
:1086E000D0ED045AC0ED067AF0EE406A27EE830A18
:1086F000C0ED056AA3EEA60A80ED087AA4EE240A6E
:10870000A5EE470AA5EEC60A80ED070A704700BF2E
:10871000D0ED007A90ED017A30EE670AE7EE007A4C
:10872000B0EE670AC0ED007A704700BF704700BF27
:108730002DE9F04FDFF8F8C1DFF8F8E1BCF80A7076
:10874000DEF80060BCF80C30BCF808A03C028BB02E
:10875000361B4FF00004CDE90034009CBCF8063015
:108760004FEA17654FF0000767EB0507B946B046BB
:10877000A4FB06670024CDE90634009C002304FB1B
:1087800009770024CDE90034AAFB0823CDE90223B0
:10879000039AF30D00930AFB09230393009B43EA1A
:1087A00047230093029B4FEAD31AFB150193039BC7
:1087B0004AEA436ADDE9002344464D46CDE90845CF
:1087C000069C12F5FA62A4FB086743F1000304FB60
:1087D0000977CDE90623BCF80440039BBCF80220CE
:1087E0004FEAE31B230C059323040493340A44EA61
:1087F00007643D12DDE904674FEAC23816EB0A064A
:1088000047EB0B0718EB0408DDE906344FEA524941
:1088100049EB0509B3F5FA6F74F10004B246BB46A3
:108820003CDADDE90067BC00B20044EA9673B41894
:1088300047EB030522463C462B4602FB04F406FBAD
:108840000344A2FB06232344940844EA83749D1046
:108850005B104FEA3202B8EB040869EB0509BAEB8A
:10886000020A6BEB030BDDE90623304C4FF0FF35BA
:10887000A242AB412CDBDDE90856A5FB052305FB35
:1088800006F403EB4403D40F44EA4304DD17DDE9A7
:108890000623121B63EB0503CDE90623DEF8044033
:1088A000A4FB082304FB0933540D44EAC3245D15DB
:1088B000B4EB0A0A65EB0B0B4FEADA3343EA4B439E
:1088C00000B1036009B1069B0B600BB0BDE8F08FEF
:1088D00040F6AC52B4184FF0000347EB03052246B4
:1088E000A2FB022304FB05F403EB4403941843EBBF
:1088F0000305A4185D414FEA850CA6004CEA947C60
:10890000B41A6CEB0305DF00D6006D104FEA340497
:1089100047EA5277921B63EB0703B8EB040869EB55
:1089200005091AEB020A4BEB030BA4E724FAFFFF3D
:10893000945300206C1E00204FF4006303827047A4
:108940004FF40063038270474FF4805303827047F3
:10895000BFF34F8F0549064BCA6802F4E062134328
:10896000CB60BFF34F8F00BFFDE700BF00ED00E01D
:108970000400FA05F8B5027B466903681F2A2DD961
:10898000A2F120055F682024AC402742114617D091
:108990001022AA40DC60DA605A68EA40D40749D461
:1089A000716B756A0A68B46A22F00102A5420A6016
:1089B00037D1012286F84C20027B11461F2A20D98C
:1089C0002039082258688A40024200D0DA60042226
:1089D000586802FA01F1014221D1F8BD20241D6836
:1089E0009440254211460CD0102191409C60996022
:1089F0001968D140C907D3D5012101FA02F29A6062
:108A0000CEE7082218688A40024200D09A60042209
:108A1000186802FA01F101420BD09960F8BDD960E3
:108A2000F8BD04463046FFF7EBFA227B2368114677
:108A3000C4E7F8BD012202FA05F5DD60B0E700BF2A
:108A400070B4037B04681F2B08D9203B2021626887
:108A500001FA03F31A421CD170BC7047202122682E
:108A600001FA03F31A42F7D042691449582000FB77
:108A7000021251685689CD680868296821F0010101
:108A80002960828992B222EA06028281A36070BCC8
:108A9000704742690949582000FB02125168568903
:108AA000CD680868296821F001012960828992B2A5
:108AB00022EA06028281E36070BC70475C7000208D
:108AC00030B4094B1C786CB1084A002502EBC40491
:108AD000116893884D628889083203439BB2A24291
:108AE0008B81F5D130BC70477C74002080740020ED
:108AF00010B4037B01681F2B09D9203B20224C684E
:108B000002FA03F31C4214D15DF8044B7047202293
:108B10000C6802FA03F31C42F6D00C4A40680024A9
:108B2000147002685DF8044B22F0010202608B6051
:108B30007047064A40680024147002685DF8044BD0
:108B400022F001020260CB60704700BF664B00203C
:108B5000F0B5C40022189200AE498B585B689D8A1C
:108B6000ADB2EEB2F7070A445CD4B70732D5BFF313
:108B70005F8F167EF6B2012E00F0C780A64D1A8BCD
:108B8000BFF35F8F221801EB8202167E022E00F0E7
:108B9000D580221801EB8202167E032E00F0888019
:108BA0009A8895F9086092B242F480629A802218FD
:108BB00001EB8202127E013296425BD1AA7A002634
:108BC0006E72002A40F09580204401EB8000002363
:108BD0004375F0BD77074ED416F0400600F0C9800B
:108BE0008D4D1E8A95F908E0176AF6B207F80E60F7
:108BF0005FFA8EFE0EF1010C4FFA8CFC177E85F8A1
:108C000008C00CF103029742664600F01C8122184E
:108C100001EB8202127E9445C9D10EF1020676B2B2
:108C20002E72C4E71E887C4D26F400663604360C8E
:108C30001E801E88B6B246F480661E80967E00278F
:108C40002F72002E48D06E7A002E42D0221801EBEF
:108C500082020126127E6E72022A00F0B98022186A
:108C600001EB8202927D42F001021A82204401EB64
:108C70008000037EF0BD684D967E0127AF72002E06
:108C800073D06E7A002E7BD1221801EB8202527EC5
:108C9000002A00F0A3801A882E7A92B2013642F49C
:108CA000007276B21A802E721A88D205FCD47EE742
:108CB000927E002A3FF474AF6A7A002A3FF470AFC4
:108CC0009A8895F9086022F480621204120C9A8046
:108CD0006DE7D27DFF2AB9D0221801EB8202967D82
:108CE00006F0FE061E82D37DFF2BBFD0FF232B7222
:108CF000BCE79A8822F4407212042044120C01EB63
:108D000080009A8000234375F0BD927E424D002A78
:108D10003FF435AF6A7A002A3FF431AF1A8822F463
:108D200080621204120C1A80BFF35F8F1A8B1A88AC
:108D3000AE7292B242F400721A8031E7927E002A3B
:108D40003FF427AF6A7A002A3FF423AF1A8895F9D7
:108D5000086022F480621204120C1A809A8822F4AD
:108D600080621204120C9A8021E76A7A002A8BD062
:108D700091E715F0800F284D3AD195F9086016E774
:108D8000167ED2F820E01F88022E95F9086045D99A
:108D900027F480673F043F0C1F801F8AFFB20EF844
:108DA00006701F88D2F820E0BFB247F400771F801A
:108DB000F2B21F8A561C76B2FFB20EF806709F8878
:108DC000961CBAB276B242F480622E729A806BE739
:108DD0001A8892B242F400621A8040E71A8895F924
:108DE000086092B242F4807201271A806F725BE7CA
:108DF00095F90870B7F1FF3F2CD0D669F65D1E8259
:108E000092F818E001377AB2964516462A727FF436
:108E1000CEAEA3E798C300206C1E0020BFB247F47B
:108E200000771F801F8AFFB20EF80670F6B21F8A05
:108E3000D2F820E0721C52B20336FFB276B20EF8BE
:108E400002702E7230E79A8822F480621204120CAB
:108E50009A80DCE6D77D1F822E72957E1DB9127E28
:108E6000002A7FF403AF9A8822F480621204120C65
:108E70009A80FBE690F8493013B1002280F849202F
:108E80001846704770B5044682B01830256D94F8C6
:108E90005C106B460622A847A8B19DF804009DF817
:108EA00000609DF801109DF802509DF803209DF888
:108EB000053041EA062143EA002342EA0522A18463
:108EC000E2842385012002B070BD00BF70B5044666
:108ED00082B00830256A6B4606223B21A847A8B11C
:108EE0009DF804009DF800609DF801109DF8025067
:108EF0009DF803209DF8053041EA062143EA00234E
:108F000042EA05226182A282E382012002B070BDA2
:108F100050F8043C012280F83520143803B118477A
:108F20007047002301224360836003600371437034
:108F3000C2718372837043710272C3727047F8B555
:108F40000468C4F30D0405460E4604B32F6828F0E8
:108F50001FFC092840F08880454C236923F44073A6
:108F60002361236943F400732361236943F0010300
:108F700023613E6028F00CFC2369092823F00103DB
:108F8000236171D12B6804332B600020F8BD394B6D
:108F9000394A93422BD902F58042934226D902F5F1
:108FA000804293422AD902F58042934228D902F5A1
:108FB0008032934226D902F50032934224D902F539
:108FC0000032934222D902F50032934220D902F5B1
:108FD000003293421ED902F5802293421CD9B3F18C
:108FE000016F1BD3052004F013F8FBE7082428F0D9
:108FF000CFFB092814D04FF0FF30F8BD1024F6E75E
:109000001824F4E72024F2E72824F0E73024EEE7E0
:109010003824ECE74024EAE74824E8E75824E6E768
:10902000134F3B6923F440733B613B6943F4007386
:109030003B613B6923F0F8033B613B6943F002036A
:109040001C433C613B6943F480333B6128F0A0FB47
:109050003B6923F002033B613B69092823F0F803D5
:109060003B613FF473AFC6E76FF00100F8BD00BF8E
:10907000003C024000400008FF3F0008F8B50446ED
:109080000D468E180027B54201D12069F8BDE3686E
:10909000591CE160234415F8012B1A720429F2D1FE
:1090A000206918B9A1682046FFF749FF2061E760F1
:1090B000E9E700BFF0B583B004466B460622032102
:1090C0001E2031F029FC00283CD09DF800509DF86E
:1090D00001109DF802709DF803209DF804609DF832
:1090E000053041EA052142EA072243EA062309B294
:1090F00012B21BB2144D06EE901A07EE102A07EEBC
:10910000903AF8EEE66A95ED005AD5ED025A95EDE3
:10911000016AB8EEC77AF8EEE77A66EE856A27EE5E
:10912000257A67EE867AFDEEE66ABDEEC77AFDEE39
:10913000E77A16EE901A17EE102A17EE903A218071
:10914000A280638003B0F0BD0000002000B583B0B2
:1091500001AB03220021772031F0DEFB9DF80530C2
:109160009DF804209DF806001B0243EA02431843C1
:1091700003B05DF804FB00BF08B5FFF7E7FF014B44
:10918000586008BD6C1E002008B5FFF7DFFF014BDB
:10919000186008BD6C1E0020682031F0BDBB00BF08
:1091A00070B582B00446694618302FF06DFAA8B148
:1091B0009DF805009DF801609DF802109DF8035090
:1091C0009DF804209DF8063041EA062143EA002379
:1091D00042EA0522A184E2842385012002B070BD09
:1091E000204B5B68C3F3080330B4BBB9EFF31183C2
:1091F000A3B91D4B1D4C1868A16800BF1A689042A6
:10920000F9D11B4B1C684FF47A7202FB04F3591A14
:10921000B1FBF4F130BC02FB00107047EFF3118298
:10922000102383F3128811498C680B6813F4803F74
:10923000104B02D0012018608C680B49D2B20D6827
:10924000186882F311880A4B19684FF47A7228441F
:1092500002FB01F31B1B30BCB3FBF1F302FB00303C
:10926000704700BF00ED00E0F8C5002010E000E00E
:10927000FCC50020F4C500202DE9F84F8046FFF71B
:10928000AFFF254E2549DFF8A0E0254A254D84464D
:1092900010274FF47A740120DEF80430C3F308037A
:1092A000D3B9EFF31183BBB90B68D2F808A000BFA4
:1092B000D1F800904B45F7D1D6F800B004FB0BF97C
:1092C000A9EB0A09B9FBFBF904FB0393A3EB0C031D
:1092D0004345E1D3BDE8F88FEFF3118A87F3128895
:1092E000D2F808B01368DB0344BF2860D2F808B096
:1092F0000B68D5F800905FFA8AFA8AF31188D6F8DD
:1093000000A0994404FB0AF3A3EB0B03B3FBFAF3AD
:1093100004FB0933DAE700BFFCC50020F8C50020D4
:1093200010E000E0F4C5002000ED00E030B4EFF301
:109330001183102282F312880649074C0A680748F5
:10934000013200250A602560DBB2026883F31188D0
:1093500030BC7047F8C50020F4C5002010E000E0E4
:1093600038B5254B5C69236B73B1A36D626BCAB1D1
:10937000998A1A88C90592B201D5D20700D438BD9E
:109380004FF6F7721A8038BDA36D99891A8889063D
:1093900092B2EBD59206E9D5E26ACAB1988880B25A
:1093A0009047E2E799891A880D0692B2E0D5100637
:1093B000DED5A26A616A8A4219D0A1692569885CF2
:1093C00098800132B2FBF5F105FB1122A262CFE7D2
:1093D0009B88E2696169DBB28B54E269E068A36D46
:1093E0000132B2FBF0F100FB1122E261BEE7DA6864
:1093F00022F08002DA60BBE7C038002038B5254B88
:109400009C68236B73B1A36D626BCAB1998A1A8889
:10941000C90592B201D5D20700D438BD4FF6F77214
:109420001A8038BDA36D99891A88890692B2EBD546
:109430009206E9D5E26ACAB1988880B29047E2E71D
:1094400099891A880D0692B2E0D51006DED5A26A77
:10945000616A8A4219D0A1692569885C98800132C5
:10946000B2FBF5F105FB1122A262CFE79B88E2690E
:109470006169DBB28B54E269E068A36D0132B2FB33
:10948000F0F100FB1122E261BEE7DA6822F080020F
:10949000DA60BBE7C038002038B5254B1C68236B69
:1094A00073B1A36D626BCAB1998A1A88C90592B269
:1094B00001D5D20700D438BD4FF6F7721A8038BDF7
:1094C000A36D99891A88890692B2EBD59206E9D5DF
:1094D000E26ACAB1988880B29047E2E799891A880F
:1094E0000D0692B2E0D51006DED5A26A616A8A4204
:1094F00019D0A1692569885C98800132B2FBF5F129
:1095000005FB1122A262CFE79B88E2696169DBB2A9
:109510008B54E269E068A36D0132B2FBF0F100FB0D
:109520001122E261BEE7DA6822F08002DA60BBE76E
:10953000C038002003685B6A03B11847704700BF5A
:1095400003681B6A03B11847704700BF03682DE921
:10955000F041DF691FB13B46BDE8F0411847002AE2
:10956000164611DD04460D460E4400E023689B6854
:10957000204698470028F9D0236815F8011B1B687E
:1095800020469847AE42F1D1BDE8F08103689B695F
:10959000184700BF03685B69184700BF03681B6971
:1095A000184700BF0368DB68184700BF03689B6863
:1095B000184700BF03685B68184700BF03681B6853
:1095C000184700BF014B1868F8E700BF8C1F002048
:1095D00038B50C46097849B1054601342B68284650
:1095E0001B68984714F8011B0029F7D138BD00BF4C
:1095F000064B53F820302BB11A689B8851690B42F7
:1096000001D1138370475383704700BFC4C5002046
:1096100010B50409013C032C17D80D4B33F8142066
:1096200000F00F0042FA00F313F001030DD0012304
:1096300003FA00F00138104033F09AFB054A064B5C
:10964000125D104403EBC00010BD002010BD00BF30
:10965000942704089027040838C400202DE9F04F0F
:109660004A484B494B4B4C4C4FF0010A4FF0020912
:109670004FF004084FF0080C4FF0100E2027402642
:10968000802530F8022B12F0010F03D01960A3F8E7
:1096900004A0083312F0020F03D01960A3F804905D
:1096A000083312F0040F03D01960A3F804800833C4
:1096B00012F0080F03D01960A3F804C0083312F0A9
:1096C000100F03D01960A3F804E0083312F0200F44
:1096D00002D019609F80083312F0400F02D0196049
:1096E0009E80083312F0800F02D019609D800833ED
:1096F00012F4807F05D04FF4807B1960A3F804B08A
:10970000083312F4007F05D04FF4007B1960A3F8F2
:1097100004B0083312F4806F05D04FF4806B1960E9
:10972000A3F804B0083312F4006F05D04FF4006BB7
:109730001960A3F804B0083312F4805F05D04FF429
:10974000805B1960A3F804B0083312F4005F05D001
:109750004FF4005B1960A3F804B0083312F4804F93
:1097600005D04FF4804B1960A3F804B00833D20B36
:1097700004D04FF4004219609A80083301F58061EB
:10978000A1427FF47EAFBDE8F08F00BF94270408AC
:109790000000024038C400200010024000286AD0B7
:1097A00003682DE9F04F03F13F4404F57E045F4E5A
:1097B000A40A0125345D04F01F066409032C05FA90
:1097C00006F559D0042C00F0AC80022C59D08588C5
:1097D000B5FA85F0C0F11F0080B2C40803EB840421
:1097E00000F00700266A80000F27874026EA070658
:1097F0002662276A01F003068240701E3A43012860
:10980000C1F3810CC1F300182262C1F341113DD9AB
:109810000024224601274FF0030E03E0102A04F132
:10982000020426D007FA02F0A84302F10102F5D1A2
:10983000D3F800C00EFA04F0C04300EA0C0CC3F8E1
:1098400000C0D3F8008006FA04FC4CEA080CC3F808
:1098500000C0D3F80CC000EA0C00D860D3F80CC0EC
:1098600001FA04F040EA0C00102AD86004F1020466
:10987000D8D1BDE8F08F70472D4C266C3543256458
:10988000A5E72B4C666C35436564A0E700200246D3
:109890004FF0010E4FF0030904E00132102A00F1ED
:1098A00002003CD00EFA02F737EA0504F5D1D3F8EE
:1098B00000A009FA00F4E4430AEA040AC3F800A08D
:1098C000D3F800B006FA00FA4AEA0B0AC3F800A07F
:1098D000D3F808A004EA0A0AC3F808A0D3F808B02D
:1098E0000CFA00FA4AEA0B0AC3F808A0D3F804A05D
:1098F0002AEA07075F60D3F804A008FA02F747EAEC
:109900000A075F60DF683C40DC60DF6801FA00F452
:1099100001323C43102ADC6000F10200C2D1BDE8F4
:10992000F08F034C266B3543256350E7BC1D0408BC
:1099300000380240002855D0026802F13F4303F589
:109940007E032DE9F04F9B0A544DEB5C03F01F059D
:109950005B090124032B04FA05F444D0042B00F026
:109960009780022B44D001F00306731E012BC1F334
:10997000810CC1F300188588C1F341113DD9002441
:10998000234601274FF0030E03E0102B04F10204DD
:1099900026D007FA03F0A84303F10103F5D1D2F86A
:1099A00000C00EFA04F0C04300EA0C0CC2F800C07C
:1099B000D2F8008006FA04FC4CEA080CC2F800C099
:1099C000D2F80CC000EA0C00D060D2F80CC001FA4A
:1099D00004F040EA0C00102BD06004F10204D8D14E
:1099E000BDE8F08F70472E4B1D6C2C431C64BAE70A
:1099F0002B4B5D6C2C435C64B5E7002003464FF0B5
:109A0000010E4FF0030904E00133102B00F10200B6
:109A10003CD00EFA03F737EA0504F5D1D2F800A0DE
:109A200009FA00F4E4430AEA040AC2F800A0D2F8F2
:109A300000B006FA00FA4AEA0B0AC2F800A0D2F80F
:109A400008A004EA0A0AC2F808A0D2F808B00CFA82
:109A500000FA4AEA0B0AC2F808A0D2F804A02AEADF
:109A600007075760D2F804A008FA03F747EA0A0785
:109A70005760D7683C40D460D76801FA00F40133DE
:109A80003C43102BD46000F10200C2D1BDE8F08F3E
:109A9000034B1D6B2C431C6365E700BFBC1D040812
:109AA0000038024038B590F84D3003B938BD04464F
:109AB0001846FFF7ADFD0546D0B120230021837184
:109AC000C171FFF737FF21460F4B41F8143F28467D
:109AD0002EF070FDAB88B3FA83F3C3F11F030122AC
:109AE00012FA03F3E2D009490A6813430B6038BD48
:109AF0000146FFF71FFF2146034B41F8143F28465C
:109B0000BDE838402EF056BD118F0008003C0140E2
:109B100038B5044600F11805FFF7C4FF636D8022D5
:109B20006B2128469847642004F042FD636D0722AC
:109B3000682128469847642004F03AFD636D0022AE
:109B40006B2128469847642004F032FD636D0122A2
:109B50006B21284698470F2004F02AFD94F84720EF
:109B6000636D022A8CBF1A2218221B2128469847AF
:109B70000F2004F01DFD636D18221C212846984714
:109B80000F2004F015FD636D94F846201A21284635
:109B900098470F2004F00CFD636D94F848201921BC
:109BA00028469847642004F003FD636D1022372196
:109BB000284698470F2004F0FBFC2846636D0122DD
:109BC000382198470F20BDE8384004F0F1BC00BFB1
:109BD00010B504460120A269138823F040031B043A
:109BE0001B0C138013889BB223F0380343F030031F
:109BF000138013889BB243F040031380FFF73CFBB4
:109C00002046FFF785FF10226A2104F11800FEF7B5
:109C100079FB642004F0CCFCA06930F0B7FF012090
:109C2000BDE81040FFF728BBF8B5434E0446FFF7E8
:109C300039FFF77AC7B104F11805A06930F0BAFF0F
:109C400094F846201A212846FEF75CFB0120FFF716
:109C500013FBA06930F09AFF2046FFF713F994F93F
:109C6000263001335FD0F8BD254655F8180F30F087
:109C7000A1FF80226B212846FEF744FB962004F0CA
:109C800097FC032268212846FEF73CFB962004F04F
:109C90008FFC03226B212846FEF734FB0F20FFF7D1
:109CA000EBFA10226A212846FEF72CFB0F20FFF763
:109CB000E3FA3A466C212846FEF724FB0F20FFF713
:109CC000DBFA94F8482019212846FEF71BFB0F20E9
:109CD000FFF7D2FA18221B212846FEF713FB0F20AC
:109CE000FFF7CAFA10221C212846FEF70BFB0F20B3
:109CF000FFF7C2FA102237212846FEF703FB0F2098
:109D0000FFF7BAFA012238212846FEF7FBFA0F20A6
:109D1000FFF7B2FAA06930F039FF0120FFF7ACFA83
:109D20000123F37289E794F9243001339BD1062093
:109D3000BDE8F84003F06CB96C1E002010B1036858
:109D400082885A83704700BF10B1036882881A83E3
:109D5000704700BF18B10368828809B95A837047F9
:109D60001A8370470E4B1B8801463BB90D4B0E4AB8
:109D70001B7810680BB981F00101EBE70B4B5A69B6
:109D80001AB118B91A68106058747047084A1868F0
:109D90001188084A92FBF1F2012102605974704760
:109DA000D0C50020D2C50020D4C50020D8C50020D1
:109DB000F0C5002020A1070010B40A4B0A4A1C7805
:109DC00001238340234052F8200029B9B3FA83F1DC
:109DD00049095DF8044BBDE7191C18BF01215DF866
:109DE000044BB7E7C0C50020C4C5002030B10368EC
:109DF00082881B691A4214BF01200020704700BFEF
:109E00002DE9F0410B4E346873691C400FD0DFF828
:109E100028800127B4FA84F3C3F11F0307FA03F57E
:109E200058F8230003689847AC437561F2D1BDE848
:109E3000F08100BF003C0140DCA600202DE9F0418C
:109E40000B4E346873691C400FD0DFF8288001275F
:109E5000B4FA84F3C3F11F0307FA03F558F823009B
:109E600003689847AC437561F2D1BDE8F08100BF4B
:109E7000003C0140DCA600202DE9F0410B4E346887
:109E800073691C400FD0DFF828800127B4FA84F3EF
:109E9000C3F11F0307FA03F558F823000368984736
:109EA000AC437561F2D1BDE8F08100BF003C0140D8
:109EB000DCA600202DE9F0410B4E346873691C408C
:109EC0000FD0DFF828800127B4FA84F3C3F11F0311
:109ED00007FA03F558F8230003689847AC43756107
:109EE000F2D1BDE8F08100BF003C0140DCA60020BB
:109EF0002DE9F0410B4E346873691C400FD0DFF838
:109F000028800127B4FA84F3C3F11F0307FA03F58D
:109F100058F8230003689847AC437561F2D1BDE857
:109F2000F08100BF003C0140DCA600202DE9F0419B
:109F30000B4E346873691C400FD0DFF8288001276E
:109F4000B4FA84F3C3F11F0307FA03F558F82300AA
:109F500003689847AC437561F2D1BDE8F08100BF5A
:109F6000003C0140DCA60020084A094808B5536CB3
:109F700043F4804353640021402235F0AEFB054B8F
:109F80004FF0FF321A60C3F8032008BD00380240CA
:109F9000DCA600201CA700202DE9F041044618464D
:109FA0000D461646984632F039FA2768E67228447C
:109FB000A07229467D69434632462046AC46BDE83C
:109FC000F0416047036810B504461B689847236852
:109FD00020469B689847A37B0133A37310BD08B547
:109FE000FFF716FB38B12C2282710022C2712021AA
:109FF000BDE808409EE408BD10B5044682B0406844
:10A00000FFF79CFE206841F0800140F2E93300E058
:10A01000EBB10289013B12F0020F9BB2F8D089B27A
:10A02000818140F2E93300E08BB10289013B12F0FB
:10A03000010F9BB2F8D083890DF1070130F0BAFC13
:10A040006068FFF781FE9DF8070002B010BD084A66
:10A05000904203D0074B9842EED10223064A02EB0E
:10A0600003135A89013292B25A815B89E4E700BF37
:10A0700000300140003C004008C40020F8B5050154
:10A08000684C694B625961199A4204EB050704BF99
:10A0900001230B730646387A30F020FC3B7A03F03C
:10A0A0001F015B090122032B02FA01F26DD0042B80
:10A0B00066D0022B5CD0631901361879FFF7A8FA35
:10A0C000F6B2074610B11223C6718371631958792D
:10A0D000FFF79EFA10B11323C67183716319987943
:10A0E000FFF796FA10B11423C671837166190A211D
:10A0F000F2793846FFF752FB7079FFF789FAF27967
:10A100000A21FFF74BFBB079FFF782FAF2790A21B7
:10A11000FFF744FB6359454A934247D0444A934270
:10A1200050D0414A934259D0424A934262D0424A67
:10A1300093426BD0414A93422CD02C44227BE2B90B
:10A1400001200222198801F4415141F445710A436A
:10A1500002431A809A8B22F400621204120C072127
:10A160009A8319821A8892B242F040021A80F8BD8E
:10A17000334B596A0A435A629DE700200246E1E7E1
:10A180002F4B19690A431A6195E72D4B196A0A4347
:10A190001A6290E702F564424FF40010536A43F4E8
:10A1A0000013536227F054FB6359C6E702F584326B
:10A1B0004FF48050536A43F48053536227F048FBB6
:10A1C0006359BAE702F500324FF48040136A43F452
:10A1D0008043136227F044FB6359AEE702F5FE3279
:10A1E0004FF40040136A43F40043136227F038FB36
:10A1F0006359A2E702F582324FF40050536A43F4E8
:10A200000053536227F024FB635996E702F5684236
:10A210004FF48010536A43F48013536227F018FB05
:10A2200063598AE708C40020003C00400030014028
:10A23000003800400034014000500140005401400B
:10A2400000380240427A02B9704710B504460368EC
:10A25000406804F10A0198470023637210BD00BFF3
:10A26000437A5A1C0344D2B242729972037A9342DF
:10A2700000D802B9704710B504460368406804F17D
:10A280000A0198470023637210BD00BF302827D011
:10A29000312827D0322827D0332827D0342827D078
:10A2A000352827D0202827D0212827D0102827D0AC
:10A2B000112827D0122827D0132827D0142827D0D8
:10A2C000152827D0162805D0172808BF0F2202D03E
:10A2D000002070470E22104B03EB4203587D70475D
:10A2E0000022F8E70122F6E70222F4E70322F2E770
:10A2F0000422F0E70522EEE70622ECE70722EAE770
:10A300000822E8E70922E6E70A22E4E70B22E2E76F
:10A310000C22E0E70D22DEE744F8030870B544881C
:10A3200006460D46C4F30B0422460021284635F0AC
:10A33000D4F93369094A934209D3094A934206D2B0
:10A34000224628461946BDE8704032F047BF23B187
:10A3500021462846BDE87040184770BDE805000852
:10A360009E060008064B07498B4202D3002318467D
:10A3700070471A88C2F30B029042F8D01433F3E707
:10A3800088010008E8050008024A136823EA000073
:10A3900010607047583D0020F8B51A4D2B789F2B60
:10A3A0002ED16B78BE2B2BD105221749A81C35F076
:10A3B000DFF928BB072229464FF6FF70FEF7D4F8D5
:10A3C000124FEC1D22884AB1A618BE4218D2052AA7
:10A3D00016D92146FEF7C8F83446F3E72146022293
:10A3E000FEF7C2F80222A118FEF7BEF80634084BA9
:10A3F000641B1C8041F60F53C31A58425841F8BDE4
:10A400000020F8BD004000089C27040800800008D8
:10A41000783900202DE9F04FDFF85891504F8DB07A
:10A420000326A7EB090718220DEB0200002135F0E7
:10A4300054F94C4BCDF8189007971A69002A04DAA2
:10A44000494A5A6002F188325A6001228DF82C2064
:10A45000F322DA60454B464C18689A8804909B7941
:10A46000ADF8142004A9072206A88DF81630FEF7CF
:10A4700005FE072204A94FF6FF70FEF775F8DFF816
:10A48000F8B080464FF0000A5C4539D30CAC00258B
:10A4900024F82C5D0222214606A8FEF7EFFD0222D9
:10A4A00021464046FEF760F840BAC043ADF80800C8
:10A4B000022202A906A8FEF7E1FD099878B108ABCF
:10A4C000C0F104022946184435F007F90A9818B972
:10A4D000089906A8FEF733FD00230A9009939DF81A
:10A4E0002C300A9A23B11F490B6943F000430B61DA
:10A4F000013E2DD0002A96D1FFF74EFF50B32CE03D
:10A5000065888DF80DA0C5F30B05AA1DADF80820D0
:10A510002288C2F30B01120BADF80A108DF80C2043
:10A5200002A9062206A8FEF7A9FD062202A94046B6
:10A53000FEF71AF8616880462A4606A8FEF79EFDD7
:10A54000616840462A46FEF70FF8143480469BE7C0
:10A55000002AD1D0052002F05BFD0DB0BDE8F08FE0
:10A5600000800008003C02402301674578F803089A
:10A570008801000800400008E80500080378202B47
:10A58000024600F10100F9D0092BF7D02D2B2CD079
:10A590002B2B03BF5378B7EE000A0246B7EE000A32
:10A5A000A3F13001C8B209289FED467A10D8F2EE27
:10A5B000046A07EE901AF8EEE77A12F8013FE7EE28
:10A5C000267AA3F13001C8B20928B0EE677AF0D933
:10A5D0002E2B4CD003F0DF03452B0BD0F7EE007A87
:10A5E00067EE276A20EE260A70475378BFEE000A0E
:10A5F0000246D5E710B451782D2959D02B290ABF2E
:10A600009178501C901C0024A1F13003092B53D8E1
:10A61000002303EB830301EB430310F8011FA1F1B7
:10A620003002092AA3F13003F3D9B3F59A7F28BF8A
:10A630004FF49A73072B42D9DFED236A1A46F7EEDF
:10A64000007A083A072A67EEA67AFAD803F00703D9
:10A650002BB1F2EE046A013B67EEA67AFBD124B37C
:10A66000C7EE276A5DF8044B20EE260A7047537840
:10A67000A3F13001C8B2092802F10102AAD8F2EE12
:10A68000046AF0EE665A07EE901AF8EEE77A12F8CE
:10A69000013F87EEA66AA3F13001C8B2092866EE31
:10A6A000A56A37EE067AEED994E767EE276AD9E70E
:10A6B000901C91780124A7E7F7EE007ACFE7F7EE38
:10A6C000007AC5E70000000020BCBE4CB5EEC00A11
:10A6D000DFED317AF1EE10FACCBF30EE270A30EE22
:10A6E000670ADFED2E7A20EE270A30B5FDEEC07A3C
:10A6F00087B017EE904A054684EAE470002303A968
:10A70000A0EBE4700193009302932DF0D3F9002C99
:10A71000ACBF20232D2303A88DF8003031F07EFE3E
:10A72000012803A924D002282DD0032805BF3023F7
:10A73000684668468DF8013034F0F5FF684631F020
:10A740006DFE0338C4B222466946284635F049F802
:10A7500000232B55284631F061FE2E22431C2A543B
:10A760000DEB0401E81834F0FBFF284607B030BDBC
:10A77000302368468DF801308DF802308DF80330B3
:10A7800034F0D1FFDAE7302368468DF801308DF8D8
:10A79000023034F0C8FFD1E76F12033A00007A4468
:10A7A0002DE9F041064615460846B6FBF2F43CB9E1
:10A7B00005FB1464124B1B5D00F8013BBDE8F08102
:10A7C000B4FBF2F767B90E4B05FB174705FB1464A2
:10A7D000DA5D00F8012B1B5D00F8013BBDE8F0815C
:10A7E000B7FBF2F8B8F1000F02D04046FFF7D8FFF0
:10A7F00005FB1878024B13F8082000F8012BE3E75B
:10A80000A427040830B402681146531C036011F8F1
:10A81000024B0160D31C517803609378151D0560CD
:10A820001B0443EA0123D078234343EA006030BC91
:10A83000704700BF0368591C1A46016012F8021BDA
:10A840000260587841EA0020704700BF38B50446DE
:10A850000068154632F0C2FC22682A44226038BDE6
:10A86000036810B40A0E5C1C04601A7003680A0CBA
:10A870005C1C04601A7003680A0A5C1C04601A708D
:10A8800003685A1C026019705DF8044B704700BFE2
:10A89000036810B40A0A5C1C04601A7003685A1C2E
:10A8A000026019705DF8044B704700BF03685A1CC2
:10A8B000026010B4197003680A0A5C1C04601A7004
:10A8C00003680A0C5C1C04601A700368090E5A1CA9
:10A8D000026019705DF8044B704700BF03685A1C92
:10A8E000026019700368090A5A1C026019707047E7
:10A8F0002DE9F047002488B080460F461E46A14649
:10A9000005AD531C0393117839B3252933D1931C1A
:10A91000CDF810900393507830284ED04FF0000AB5
:10A92000A0F13003DBB2092B42D96C2819D064287E
:10A9300000F0938024D825281CD063D9582876D0DD
:10A9400063281BD131784046B847039A531C0393C0
:10A950001178043601340029D7D1204608B0BDE86B
:10A96000F087039B5A1C03921B78642B7CD02AD857
:10A97000252B54D1252140460134B847039AC0E71E
:10A98000732833D044D975284FD106F1040E3068AE
:10A990002B4600220A217646FDF76AFD049A0095AF
:10A9A000534639464046FDF7A1FD039A0444A8E703
:10A9B00004AA03A92DF05AF8B7E7D31C03939078A3
:10A9C0004FF0010AACE7732B10D05BD9752B3AD04E
:10A9D000782B96D1A3F15802B2FA82F2306852096C
:10A9E0002B4610210436FDF743FDD7E73368049A60
:10A9F0000093394600234046FDF778FD04360444B1
:10AA0000039A7EE70028B9D1204608B0BDE8F08758
:10AA10006E28B3D1039A336804361C6071E72AD9D3
:10AA2000582BD7D0632B8DD06BE77828A6D1A0F117
:10AA30005802B2FA82F2306852092B461021FDF713
:10AA400017FD0436AAE706F1040E30682B460022F3
:10AA50000A217646FDF70CFDA0E7331D3068294634
:10AA60001E46FDF7D7FC99E7331D306829461E4680
:10AA7000FDF7D0FC92E7002B7FF443AF204608B0EF
:10AA8000BDE8F0876E2BC6D03BE700BF0EB400B523
:10AA900084B005AB019053F8042B0649039301A839
:10AAA000FFF726FF019B00221A7004B05DF804EB4B
:10AAB00003B07047E18400080FB430B583B006AB33
:10AAC0000A490B4853F8042B096800680193FFF703
:10AAD0000FFF084C05462068FEF75CFD0028FAD001
:10AAE000284603B0BDE8304004B07047B4380020B9
:10AAF000B83800208C1F0020DFED2B7AB4EEE70A77
:10AB0000F1EE10FA4ADDDFED296A9FED297A01E0C6
:10AB1000B0EE670AB4EEC70AF1EE10FA70EE667A8C
:10AB2000F6DC9FED247AF4EEC77AF1EE10FA38D510
:10AB3000DFED1E6A9FED207A01E0F0EE407AF4EE40
:10AB4000C77AF1EE10FA37EEA60AF6D4DFED1B7ADB
:10AB5000B4EEE70AF1EE10FA14DDDFED137A37EE0A
:10AB6000C00A60EE006A9FED166A9FED167ADFED6F
:10AB7000167AA6EE867A20EE266AE6EE877AA6EEAA
:10AB8000270A7047DFED117AB4EEE70AF1EE10FA0A
:10AB900044BFDFED087A37EEC00AE2E7F0EE407A14
:10ABA000BFE7B0EE670AD1E7DB0F4940DB0FC940D2
:10ABB000E4CB1641DB0F49C0E4CB16C1DB0FC93F24
:10ABC00092E741B99730083C15A82ABEDB0FC9BFF0
:10ABD00041404A0011F0800F82F0D503D2B2DBB2BF
:10ABE00008BF1346590013F0800F81F0D502C9B297
:10ABF000D2B208BF0A46510012F0800F81F0D5038F
:10AC0000C9B2DBB208BF0B46590013F0800F81F0C8
:10AC1000D502C9B2D2B208BF0A46510012F0800F65
:10AC200081F0D503C9B2DBB208BF0B46590013F05F
:10AC3000800F81F0D502C9B2D2B208BF0A465100D6
:10AC400012F0800F81F0D503C9B2DBB208BF0B460A
:10AC50005A0082F0D50013F0800FD2B2C0B208BF04
:10AC60001046704780EAE073A3EBE0738B4205DB8C
:10AC7000002801DD401A704702D17047002070475C
:10AC80000844704709B909E0194690FBF1F301FB4C
:10AC900013030846002BF7D1084670470146FBE72F
:10ACA000F0EEC07AB0EEE07AB4EEE77AF1EE10FAA8
:10ACB000B4BFB0EE676AB0EE476AB5EE406AF1EE37
:10ACC00010FA46D0B4EEE77AF1EE10FA8CBFF0EE4F
:10ACD000675AF0EE475AC5EE866A9FED1F3A9FED20
:10ACE0001F6A9FED1F4A9FED1F5ADFED1F3ADFEDF0
:10ACF0001F4ADFED1F5AA6EEC36AE6EEA34AA6EE90
:10AD0000864AB7EE006AA6EE845AA6EEA46AE6EE7C
:10AD1000855AC5EE866AB4EEE77AF1EE10FA48BFBE
:10AD2000DFED147AF5EEC00A48BF77EEE66AF1EE81
:10AD300010FA48BFDFED107AB5EEC00A48BF77EED3
:10AD4000E66AF1EE10FA48BFF1EE666AB0EE660A06
:10AD50007047DFED076ADEE739094E3DE3B59E3EF9
:10AD600088FA163E45FE7F3F99FB243F69A2163EB6
:10AD7000A7DFA834DB0FC93FDB0F4940DFED317A95
:10AD800030EE277AFDEEC76A16EE903A2033402B5C
:10AD900002D99FED2D0A7047B4EEE70AF1EE10FAE2
:10ADA0004DDD9FED2A6ADFED2A6A01E0B0EE677A99
:10ADB000B4EEE67AF1EE10FA77EE467AF6DC9FED25
:10ADC000257AF4EEC77AF1EE10FA35D5DFED1F6A79
:10ADD0009FED217A01E0F0EE407AF4EEC77AF1EED1
:10ADE00010FA37EEA60AF6D4DFED167AB4EEE70ACB
:10ADF000F1EE10FA1BDCDFED197AB4EEE70AF1EEA2
:10AE000010FA44BFDFED137A37EEC00A60EE006A35
:10AE10009FED136A9FED137ADFED137AA6EE867A23
:10AE200020EE266AE6EE877AA6EE270A7047DFED67
:10AE30000F7A37EEC00AE9E7B0EE670AD4E7F0EE22
:10AE4000477ABCE7DB0FC93F00000000DB0FC940B9
:10AE5000E4CB1641DB0F49C0E4CB16C1DB0FC9BF01
:10AE600092E741B99730083C15A82ABEDB0F49404C
:10AE7000FDEEC07A17EE903A2033402B51D8DFED2B
:10AE80002D7AB4EEE70AF1EE10FA50DDDFED2A6A12
:10AE90009FED2A7A01E0B0EE670AB4EEC70AF1EE40
:10AEA00010FA70EE667AF6DC9FED257AF4EEC77A3A
:10AEB000F1EE10FA38D5DFED206A9FED227A01E03D
:10AEC000F0EE407AF4EEC77AF1EE10FA37EEA60A09
:10AED000F6D4DFED1D7AB4EEE70AF1EE10FA1BDCD2
:10AEE000DFED1A7AB4EEE70AF1EE10FA44BFDFEDB7
:10AEF000147A37EEC00A60EE006A9FED156A9FED86
:10AF0000157ADFED157AA6EE867A20EE266AE6EE51
:10AF1000877AA6EE270A7047DFED067A37EEC00A79
:10AF2000E9E79FED0E0A7047B0EE670AD1E7F0EE51
:10AF3000407AB9E7DB0F4940DB0FC940E4CB16414B
:10AF4000DB0F49C0E4CB16C1DB0FC93FDB0FC9BF24
:10AF500092E741B99730083C15A82ABE00000000CE
:10AF600010B507EE901A2DED028BB8EE678ADFED73
:10AF7000227A28EE008A044628EE278AB0EE480A94
:10AF800032F0ECFAF0EE408AB0EE480A32F048FABD
:10AF9000F7EE007A9FED197AF0EE675AE8EE875ADD
:10AFA0000023A361B0EE676AC7EEA56A63612362FE
:10AFB000E361A3626362A8EEC76ABDEC028B77EE21
:10AFC000C07AB6EE007AF8EE005A27EE877A20EEC5
:10AFD000250A27EE267A26EE266A67EEA67A20EE66
:10AFE000260A84ED046AC4ED017A84ED007A84EDCA
:10AFF000027A84ED030A10BD27D4D236F304353F1C
:10B0000010B44C09012250F8243001F01F0102FA5B
:10B0100001F10B4340F824305DF8044B704700BF4A
:10B020004B0901F01F0150F82320012303FA01F11D
:10B03000114214BF18460020704700BF0C4B9842C5
:10B0400013D0A3F5806398420FD003F58043984254
:10B050000BD003F58063984207D003F580639842D4
:10B0600003D0044B186840087047024B18687047BB
:10B07000000401402C700020F0B5774B774A87B070
:10B080001968914200AF00F0DB800023744A3B60F6
:10B090007B60136843F48033136003E03B68B3F5CF
:10B0A000A04F09D0136803F400337B603B68013381
:10B0B0003B607B68002BF1D0694B1B6813F40033B5
:10B0C00018BF01237B607B68012B7BD0654D644BEF
:10B0D000654AEA606549586F654A0860AA605E6B18
:10B0E000644C654A654826F080065E635E6F46F0F4
:10B0F00080765E67196B0C431C63596B5963996BBF
:10B100009963196C41F05B5141F47B1141F41F616B
:10B1100041F00F011964596C07F118040A4348F211
:10B12000FF715A6444F8101D002621460123FB7369
:10B130003E737E73BE7326F03FFB21464FF6FF73CE
:10B140004F48BB6026F038FB4FF6FF7321464D4851
:10B15000BB6026F031FB21464B4826F02DFB2146F3
:10B160004A4826F029FB2146494826F025FB21467E
:10B17000484826F021FB2146474826F01DFB214682
:10B18000464826F019FB204626F020FC444B454C4F
:10B190001B68BA6844484549A4FB03439B09A0FBCC
:10B1A0000202013B920CB3F1807F0A6007D2404A51
:10B1B000F0200721536085F82300966011601C374A
:10B1C000BD46F0BD264B3B4C1A6C3B4942F08052C9
:10B1D0001A6420680A69CD68496940F440402060DB
:10B1E000986898609868120640F40040986042EAB7
:10B1F0008512986842F48002490842F00802013939
:10B2000042EA014240F4A05098605A601A6842F045
:10B2100080721A601A689201FCD52849104A40F2DF
:10B2200005700860996821F003019960996841F000
:10B2300002019960936803F00C03082BFAD145E7EB
:10B2400000221A6062B61E4B1B6883F308881D4BF0
:10B250001B689847FEE700BFFCFF0120EFBEADDE94
:10B260000038024000ED00E00005FA05D08600201D
:10B2700000000008FF916700335F070000000240F4
:10B280000004024000080240000C0240001002408E
:10B290000014024000180240001C0240002002403E
:10B2A0002C700020D34D621083DE1B43FCC50020B0
:10B2B00010E000E00070004000000020003C024070
:10B2C0000000FF1F0400FF1F08B5054B1B6803B1FA
:10B2D0009847044B044A1A6072B6FDF739FB00BF69
:10B2E000AC690020FCFF0120EFBEADDE08B5034BCA
:10B2F0001B6803B1984772B6FDF72AFBAC690020C2
:10B30000084B10B507281B68C8BF143818440C46F2
:10B31000007EFEF77DF920B12146BDE81040FEF722
:10B3200019BD10BD48A7002030B50446806D61717D
:10B330008389A26823F400531B041B0C838185B00E
:10B34000A379009213F0040230D04FF4805213F02E
:10B350000203ADF8042056D1ADF806304FF48063F7
:10B360000022ADF8083011F00103ADF80C2028D10F
:10B37000ADF80A3008238D07694648BFADF80A309A
:10B3800026F06EFBA279A36DD10724D412F0080F2A
:10B390009A8A1BD122F008021204120C9A829A890E
:10B3A00092B242F400529A8105B030BD13F002030C
:10B3B000ADF8042024D04FF400551346ADF80650E4
:10B3C000CEE70423ADF80A300C23D4E792B242F062
:10B3D00008029A82E3E70D498B420FD0A1F548415C
:10B3E0008B4209D00A498B42D0D105200121FFF7B9
:10B3F00087FFA279A36DC9E70220F7E70020F5E7F0
:10B40000ADF80630ACE74FF40053A5E7001001405B
:10B410000014014010B50446806DA160838923F4B7
:10B4200000531B041B0C8381A37984B013F0040226
:10B43000009135D04FF4805213F00203ADF8042090
:10B4400056D1ADF806304FF480636279ADF808301C
:10B45000D1074FF00003ADF80A30ADF80C3045BF0E
:10B460000423ADF80A3008230C236946920748BF2D
:10B47000ADF80A3026F0F4FAA279A36DD1071FD4F3
:10B4800012F0080F9A8A16D122F008021204120C48
:10B490009A829A8992B242F400529A8104B010BD05
:10B4A00013F00203ADF804201FD04FF400511346EF
:10B4B000ADF80610C9E792B242F008029A82E8E7B6
:10B4C0000D498B420FD0A1F548418B4209D00B4961
:10B4D0008B42D5D105200121FFF712FFA279A36D80
:10B4E000CEE70220F7E70020F5E7ADF80630ACE73D
:10B4F0004FF40053A5E700BF0010014000140140C5
:10B5000038B50D4B07281B68CCBFA0F114040446C6
:10B5100023440546187EFEF77BF858B101342722F4
:10B52000C47182710121FEF705FA28460021BDE8A9
:10B530003840E5E638BD00BF48A70020064A002392
:10B540005168814202F11C0204D00133102BF7D163
:10B5500000207047D8B27047D000002070B50F4C63
:10B560000F4DC0EBC00004EB8004286B266930430C
:10B57000286382B09209667BA1600025012101A8A1
:10B5800063618DF804608DF805208DF806508DF804
:10B5900007102FF081F902B070BD00BFD00000206D
:10B5A00000380240074BC0EBC00030B403EB800012
:10B5B000054C0569236B2B4323630176427630BC2F
:10B5C000704700BFD0000020003802402DE9F04F46
:10B5D000534C54F8204083B0002C00F09C80E56D63
:10B5E000002D00F09A8017464E4A9846064604F110
:10B5F00062032869226004F262226361A2614FF44F
:10B6000000736A68A160E3602361A265A24668B125
:10B61000FFF794FF721CD2B20C21FFF7C3FFA36D9A
:10B62000A9682A6922630433A1636365E868A0B14D
:10B63000FFF784FF721C8146D2B20B21FFF7B2FFE5
:10B640002346EA7F38494846FFF788FFA36DA9687B
:10B65000EA6862630433E163236594F86100FDF7EF
:10B66000D7FF814694F86000FDF7D2FF8346287F1C
:10B6700000284DD118F0080F36D1BA070DD5B9F111
:10B68000000F0AD00B22731C89F8062089F80730B6
:10B6900048466A7F2221FEF781F8FB0715D4A36B89
:10B6A0007BB995F82020A97F8DF8063001A8930971
:10B6B00001228DF805308DF804108DF807202FF049
:10B6C000EBF8504603B0BDE8F08FBBF1000FE6D0B9
:10B6D00001360C238BF807608BF8063058466A7FDA
:10B6E0002221FEF75BF8DAE70136F6B2B9F1000F76
:10B6F00004D00B2389F8076089F8063018F0100F82
:10B70000484614BF022112216A7FFEF747F8C6E7B8
:10B710002FF0E4F8AEE7A246D3E7AA46D1E700BF90
:10B72000C038002080F80308758900080348D0F865
:10B73000AC3113B100F5D27018477047D00000202B
:10B740000348D0F8903113B100F5C4701847704722
:10B75000D00000200348D0F8743113B100F5B67062
:10B7600018477047D00000200348D0F8583113B173
:10B7700000F5A87018477047D00000200348D0F8A3
:10B780003C3113B100F59A7018477047D000002083
:10B790000348D0F8203113B100F58C70184770477A
:10B7A000D00000200348D0F804310BB1FC3018471A
:10B7B000704700BFD00000200348D0F8E8300BB13C
:10B7C000E0301847704700BFD00000200348D0F891
:10B7D000CC300BB1C4301847704700BFD0000020F8
:10B7E0000348D0F8B0300BB1A8301847704700BFFD
:10B7F000D00000200348D0F894300BB18C301847AB
:10B80000704700BFD00000200248836F0BB170303A
:10B8100018477047D00000200248C36D0BB1543068
:10B8200018477047D00000200248036C0BB1383035
:10B8300018477047D00000200248436A0BB11C3003
:10B8400018477047D00000200248836803B11847AA
:10B85000704700BFD0000020431C00F019812DE983
:10B86000F04F4FEAC00B0BEB00039B00DFF8908218
:10B8700058F803A087B008EB0304BAF1000F00F0FA
:10B880000481143308EB03010022DAF8047048F84D
:10B8900003204A608A60CA60A568D4F80C90431CF3
:10B8A000DBB215B11522EB71AA71B9F1000F04D00A
:10B8B000162289F8073089F8062001909AF80E00C0
:10B8C0002FF00CF8BB8823F440731B041B0CBB80C7
:10B8D0002846FEF739FA4846FEF736FA112128467F
:10B8E000FEF728F811214846FEF724F808266424BC
:10B8F00004E00A203CB1FDF7BFFC013C2846FEF7FE
:10B9000075FA0028F5D02846FEF718FA0A20FDF748
:10B91000B3FC2846FEF718FA0A20FDF7ADFC013EFD
:10B92000ECD14846FEF70AFA0A20FDF7A5FC2846A6
:10B93000FEF704FA0A20FDF79FFC2846FEF704FAFA
:10B940000A20FDF799FC4846FEF7FEF9019B0BEB38
:10B95000030408EB84042846637C002B0CBF1221EF
:10B9600032210422FDF71AFF637C002B0CBF122149
:10B97000322148460422FDF711FF584B9F4200F048
:10B980009880574B9F4200F09E80564B9F4200F09C
:10B990008680BB880199544A544C23F440731B049D
:10B9A0001B0CBB803B888B4408EB8B089BB243F09D
:10B9B000010398F810103B80BD8802A8002918BF29
:10B9C000144626F003F8049A4948B2FBF4F325F034
:10B9D0003F05A0FB02122D04900C2D0C0543BD80E9
:10B9E000444C39884FF4967202FB00F284FB02400B
:10B9F0009BB2D217002BC2EBA01221F0010108BFAD
:10BA000001230904013243F40043090C92B2398046
:10BA10003A84BB833B889BB243F001033B803B8865
:10BA200023F4816323F002031B041B0C4FF48042B8
:10BA300043F480633B803A813B8823F080031B04FE
:10BA40001B0C3B809AF810308DF80830002402A8B7
:10BA500001258DF809408DF80A408DF80B502EF025
:10BA60001BFF9DF80B209AF80F308DF808308DF8E9
:10BA700009408DF80A4062B95A09203203F01F03C9
:10BA80001D4905FA03F341F8223007B0BDE8F08FF5
:10BA9000704702A82EF000FF07B0BDE8F08F174AEC
:10BAA000136A43F4000313624FF4000025F0D8FE3C
:10BAB0006FE7124A136A43F4001313624FF4001045
:10BAC00025F0CEFE65E70D4A136A43F48003136246
:10BAD0004FF4800025F0C4FE5BE700BF0054004037
:10BAE00000580040005C0040009F2400804F12007E
:10BAF00083DE1B43D34D621000E100E000380240BA
:10BB000098C30020F0B5C60033189B00254DEA58B5
:10BB10005468A28A83B092B20192019A2B4412F423
:10BB2000706F1CBF01221A75019B13F4E06F07466A
:10BB30000CD1A38A3E4423F4706305EB86051B04F5
:10BB40001B0C0022A3826A7503B0F0BD238BA3886F
:10BB500023F480631B041B0CA380019B9B05E8D48A
:10BB600023889805E5D42388D9050ED52388DA05DE
:10BB7000FCD423889BB243F40073238023889B0565
:10BB8000FCD43846FFF768FED3E723889BB243F422
:10BB900000732380A38823F440731B041B0CA38031
:10BBA000C7E700BF98C30020F0B583B0441C8DF8F0
:10BBB000073001D0032802DD002003B0F0BDC7002C
:10BBC000244E3B1806EB83035D68002DF4D049003A
:10BBD000C9B2997501240021DA755C7699761C76D4
:10BBE0005C751975A9880DF107028905DA611A6279
:10BBF00014D42B88DA050CD44FF4805401E0013CB6
:10BC00001ED02B889B05FAD42B889BB243F48073FB
:10BC10002B80AB889BB243F44073AB80074406EBA8
:10BC200087024FF4805401E0013C09D0537D002B82
:10BC3000FAD106EB87073C7D84F0010003B0F0BD2C
:10BC4000054A138801339BB21380FFF705FE204697
:10BC5000B3E700BF98C3002004C400202DE9F043DF
:10BC6000322083B002F0A4FC112300221E21012007
:10BC7000FFF79AFF0122104660231E21FFF794FF71
:10BC8000642002F095FC6846FDF714FA0024DFF802
:10BC90005481254626460A270123184602221E21E2
:10BCA000FFF782FF322002F083FC6846FDF702FABC
:10BCB000BDF900E0BDF90210BDF904208E457346C0
:10BCC000A8BF0B469342A8BF134643454FF001005F
:10BCD00076440D44144479DBFDF78AFC013FDBD147
:10BCE0004FF00109122300221E210120FFF75CFF03
:10BCF000DFF8F0800A270123184602221E21FFF7F1
:10BD000053FF322002F054FC6846FDF7D3F9BDF929
:10BD100000E0BDF90210BDF904208E457346A8BFAE
:10BD20000B469342A8BF134643454FF00100A6EBD4
:10BD30000E06A5EB0105A4EB02044ADBFDF758FC57
:10BD4000013FD8D107EE906AF8EEE76A07EE905A05
:10BD5000B8EEE77A07EE904ADFED1F5A9FED1F5AC3
:10BD60001F4EF8EEE77A85EEA66A702300221E21A8
:10BD70000120C5EE876A85EE277AB0EEC66AF0EE3E
:10BD8000E66AF0EEC77A86ED006AC6ED016AC6ED96
:10BD9000027AFFF709FF0122104620231E21FFF738
:10BDA00003FF002302221E210120FFF7FDFE642075
:10BDB00002F0FEFBB9F1000F04D14FF07E53336067
:10BDC0007360B360012003B0BDE8F0834FF0000959
:10BDD00088E74FF00009B5E700406F4601C05E46B6
:10BDE0000000002001F0FFFF0123184648227721C0
:10BDF000DAE600BF0123184658227721D4E600BFB7
:10BE0000134601200A466821CEE600BF0220FCF757
:10BE10009FBE00BF022075E60120FCF799BE00BF5F
:10BE200001206FE60020FCF793BE00BF002069E60A
:10BE30001549164B1648CA6810B44C691549B2FB2F
:10BE4000F4F203FB02F30360D1F88820124B134C89
:10BE500042F47002C1F888201A68002042F0010202
:10BE60001A6098601A6822F0847222F480321A6094
:10BE70005C601A684FF0006422F480221A60D86077
:10BE80008C605DF8044B70470000002040420F00BA
:10BE90002C70002000ED00E000380240103000243B
:10BEA000044B4FF4F07002210A22D86059611A61E4
:10BEB000FFF7BEBF0000002003680A7A591C01602A
:10BEC0001A70704738B50B4C23688BB15A68821AC8
:10BED000002A054604DA0CE05A68AA1A002A07DB91
:10BEE0009A68226018461A6890472368002BF3D19D
:10BEF00038BD38BD3C5300200B4B002210B40272F9
:10BF000003F59074032102E0072A09DC9979890777
:10BF100002D51979815401329C4203F11803F3D1FF
:10BF20005DF8044B704700BF8C2404082E23037077
:10BF3000704700BF012310B4312132241022447015
:10BF40004171C2700370037183705DF8044B7047D8
:10BF50002DE9F0410B78047BDB43DEB200F11002E7
:10BF600000F1380342F8044F9342FBD1DFF89CC044
:10BF700000F16001002243F8042F8B42FBD14FF007
:10BF8000140E0521002546FA01F303F00103002BEE
:10BF90001D4414BF4FF019084FF00A0811F0010FAB
:10BFA000EDB214BF2746002700220EEB02039BB21E
:10BFB00000EB8303013242455F61F6D1013A92B250
:10BFC000013201390EEB02034A1C9BB201D09E469E
:10BFD000D9E715F0010F14BF19250A2500215A18B9
:10BFE00092B200EB82020131A9425461F7D10B44B5
:10BFF0009BB21A1D00EB8202013300219BB25160FB
:10C00000ACF800300361BDE8F08100BF801E002065
:10C01000254B5B880B332DE9F04F8A4601F1060B67
:10C020001FFA83F94FF00108002100271AF801EBED
:10C030003E464C460122A4F10B039BB207E00133BC
:10C040009BB2B0F80CC0C5F814C09C420AD000EBFB
:10C050008305002AF3D100EB830501339BB29C4298
:10C060006A61F4D1231D00EB83030136092FF6B278
:10C0700059600CD0092E14D008FA07F313EA0E0FFA
:10C0800014BF012200220C34A4B20137D3E709F116
:10C090007809DA451FFA89F9C7D1034B5980BDE801
:10C0A000F08F0022EFE700BF801E00202DE9F0474F
:10C0B000DFF85C80B8F8043004338A461FFA83FC4A
:10C0C00001F109094FF0010E1AF8017B64460026C0
:10C0D000231F0EFA06F29BB23A40BAB1818900EBF7
:10C0E000830501339BB29C426961F6D10136043469
:10C0F000082EA4B2ECD10CF1200CCA451FFA8CFC1E
:10C10000E2D10023A8F80430BDE8F0871146E6E745
:10C11000801E002010B4037B01681F2B09D9203B2F
:10C1200020224C6802FA03F31C4214D15DF8044B40
:10C13000704720220C6802FA03F31C42F6D00C4A26
:10C1400040680024147002685DF8044B22F001027C
:10C1500002608B607047064A4068002414700268D1
:10C160005DF8044B22F001020260CB60704700BF13
:10C1700054AE002070B54E680546304630F04EF99A
:10C18000314604460246286831F028F82A68131917
:10C1900001333B212B60115570BD00BF08B523F062
:10C1A0002BFEFFF7A3F800BF024A034B1278197861
:10C1B00018F02EBB0C2000200D20002038B5384B85
:10C1C0005A899989914224BF00225A81198ADA89B1
:10C1D000914224BF0022DA81DA788AB1072A0FD08F
:10C1E000304C3148A27801210025062A017099704F
:10C1F000DD714CD92379DFED2D6A002B36D138BDA6
:10C20000DA799B78284807EE103A002A44D0DFED0F
:10C21000276A0178234CB8EEC77A07EE901AA27805
:10C22000F8EEE77A27EE267A062A67EE877A2BD889
:10C230001F4B03EB8203D3ED006AF4EEE76AF1EEE5
:10C2400010FA10DDC6EE877AFDEEE77A17EE903A27
:10C25000102BA8BF1023012BB8BF0123DBB28B42E8
:10C2600028BF0B4603702379002BC8D0013A032A5C
:10C27000C5D8B7EE000A80EE260A31F023F92388EC
:10C28000984238BF208038BDDFED086AD5E7DFED82
:10C29000097AB0EE677ACBE7DFED076AB9E700BF4E
:10C2A000F8B9002030700020886800206F12033831
:10C2B000A8F803086F12833A6F120339038A2DE935
:10C2C000F0478589ADB21D4029D00F4606464FF094
:10C2D00000484FF00009B5FA85F328FA03F2D2437B
:10C2E00091B21B3B15403182042B16D8DFE803F0D6
:10C2F0003129211903007B6A002B32D003F1FF3A68
:10C300001FFA8AFAC7F824903C6A34B123682046A1
:10C31000514698476468002CF8D1002DDBD1BDE868
:10C32000F0873868716B036889B29847002DD2D1C5
:10C33000F5E77868B16B036889B29847002DCAD1D8
:10C34000EDE7B868F16B036889B29847002DC2D158
:10C35000E5E7F868316C036889B29847002DBAD1D7
:10C36000DDE7F36A1FFA83FACEE700BFF0B54B4B67
:10C370004B491A68096883B00123570200935CBFD8
:10C3800003F180530093D6005CBF43F01003009389
:10C390008C0744BF43F0C6030093480744BF43F0F3
:10C3A000080300930F0748BF43F020033D4948BFEF
:10C3B0000093160648BF43F44063097848BF0093D2
:10C3C000D40548BF43F0006301F0EF0048BF00937D
:10C3D00008286D4655D00E2953D0D0033248009B13
:10C3E00000784CBF43F4204343F40053D7044CBFC0
:10C3F00043F0C84343F0884300280CBF07200F20B8
:10C40000960648BF43F48073540748BF43F4003393
:10C4100043F400245205009402D5244A1279A2BBA9
:10C42000182936D001900027012639462846FCB24B
:10C43000FEF7F6FD60B11E4B002203F5D87103E054
:10C440008B420FD013F80C2CA24203F10C03F7D14E
:10C450000137242FE9D195E80300164B83E8030048
:10C4600003B0F0BD7A0904F01F0455F8223006FA33
:10C4700004F4013723EA0404242F45F82240D4D1E0
:10C48000E9E743F480530093A7E743F4C013009314
:10C49000C6E7009B43F060730093C3E7D486002097
:10C4A000B0690020C468002058700020545000205B
:10C4B000F4F90308042000202DE9F84F4E014FF055
:10C4C000000B174D8146904606F120075C46594601
:10C4D00028465FFA8BFAFEF7A3FDC0B1A64215D835
:10C4E000A74213D900200F4A014604E00131242954
:10C4F00014D012F80C0C504502F10C02F6D10A4B84
:10C5000001EB410103EB81014846C04701340BF1C7
:10C51000010BBBF1240FDAD1BDE8F88F0021F3E75E
:10C5200004200020F4F90308E8F9030800210A4A6E
:10C530000B4604E00133242B0BD012F80C1C88426C
:10C5400002F10C02F6D1054803EB430300EB830034
:10C5500070470020704700BFFCF90308E8F90308A2
:10C5600000210A4A0B4604E00133242B0BD012F8B9
:10C570000C1C884202F10C02F6D1054803EB430380
:10C5800000EB830070470020704700BFF4F90308F8
:10C59000E8F903081C4C08B501210220FDF70CFC4A
:10C5A000237803F00502052A29D003F00903092B9B
:10C5B00008D000210120FDF7FFFB00210846FDF710
:10C5C000FBFBFEE7114A124B11681A680B68114C0D
:10C5D00023F001030B601388206823F001031B0480
:10C5E0001B0C138018B1292200238271C371092208
:10C5F0004A21FDF7D3F82068FDF7A0FBD9E723F027
:10C60000ABFC2378D1E700BFBC38002034250020E4
:10C61000382500203C250020022828BF022010B425
:10C62000084C094B207000EBC00200EB8202074966
:10C630005DF8044B013003EB4203C0B20B6011F014
:10C64000CFBB00BFE8C20020083C002014570020E8
:10C6500008B51DF0BDFDFDF7DDFEBDE808401DF08D
:10C660009FBD00BF38B50D4C0D4DAC4206D2616880
:10C6700020461434FDF752FEAC42F8D3094B0A4C65
:10C680000A4818600025257023F038FA084B094A3B
:10C6900065701A60BDE8384019F048BC8801000890
:10C6A000E805000814570020E8C20020083C0020DC
:10C6B00018570020FEC2002008B5FFF7D3FF1DF079
:10C6C00087FDFDF7A7FEBDE808401DF069BD00BF6E
:10C6D000F0B50C2934D8DFE801F0893333335E3309
:10C6E0003333343333330700048C9689B2F802E0D5
:10C6F0001788734D24F480542404240C0484038C80
:10C700008488818B23F4005321F4E6411B0409043F
:10C710001B0C46EA0E06090C43EA063341EA0721E0
:10C72000A8429BB2A4B289B200F09E8005F5806554
:10C73000A84200F099809268848081830264038417
:10C74000F0BD048C9589B2F802C0B2F800E05C4FED
:10C7500024F480742404240C0484038C8688818B44
:10C7600023F400731B0421F073011B0C45EA0C0435
:10C77000090443EA0423090CB8429BB2B6B241EA69
:10C780000E015CD04F4CA04259D0926886808183C4
:10C79000C2630384F0BD048C9589B2F802C0B2F87C
:10C7A00000E0474E24F010042404240C0484038C7D
:10C7B0008788018B23F0200321F4E6411B04090440
:10C7C0001B0C45EA0C04090C43EA041341EA0E2150
:10C7D000B0429BB2BFB289B25DD03A4CA0425AD0AF
:10C7E00092688780018382630384F0BD048C9789FB
:10C7F000B2F802E01688324D24F001042404240C1F
:10C800000484038C8488018B23F002031B0421F031
:10C8100073011B0C47EA0E0709043B43090CA842AD
:10C820009BB2A4B241EA060125D005F58065A84275
:10C8300021D092688480018342630384F0BDD5894E
:10C84000148A578A23F4006343EA05254FF6FF3321
:10C850002B40958826F440563C4343EA052346EA9C
:10C8600004169BB2B6B290E7158A24F4804444EAD9
:10C870008514A4B25FE7D689158A578A23F0080386
:10C88000334324F4407496883D4323F004032C433F
:10C890003343A4B2CDE7D489158A568A23F08003A6
:10C8A00043EA04134FF6BF741C40938827F4406793
:10C8B000354344EA031347EA85079BB2BFB28FE7CB
:10C8C00000000140000401402DE9F84FF022002152
:10C8D0009348944CDFF87492934D944E944FDFF844
:10C8E000708232F0FAFE93489349DFF868E2DFF88D
:10C8F00068C200221359834200F0F980B3F1804FDF
:10C9000000F0F780AB4200F0F680B34200F0F58013
:10C91000BB4200F0F480734500F0F380634500F003
:10C92000F280434500F0F180DFF830A2534500F07B
:10C93000EE800AF5806A534500F0EB800AF5806AC4
:10C94000534500F0E880AAF5983A534500F0E58099
:10C950000AF5806A534500F09C800AF5806A5345C9
:10C9600008BF0D2300F096801832B2F59C7FC1D12C
:10C97000DFF8B081714E08F59C774FF0030A4FF055
:10C98000020998F804301C09013C032C03F00F0342
:10C9900078D86B4A32F8140040FA03F2D20771D506
:10C9A000012505FA03F3013B184030F0E1F9654B2E
:10C9B0001B5D184416EBC00264D056F83030624C50
:10C9C00098F8081003F13F4000F57E00800A205CD3
:10C9D00000F01F044009032805FA04F500F08180E7
:10C9E000042878D0022804D15348406C05435248AB
:10C9F0004564B2F804E0BEFA8EF2C2F11F0292B2B0
:10CA0000D00803EB800002F00702046A92000F25B1
:10CA1000954024EA05040462046A01FA02F2224302
:10CA2000002502624FF0010C2A4603E0102A05F1AE
:10CA3000020527D00CFA02F030EA0E0102F10102E1
:10CA4000F4D11C680AFA05F1C9430C401C60D3F804
:10CA500000B009FA05F444EA0B041C609C680C4021
:10CA60009C609C689C605C6824EA00005860586880
:10CA70005860D8680140D960D968D960102A05F19A
:10CA80000205D7D108F1180847457FF47AAFBDE811
:10CA9000F88F0C2309EBC3034FF0010A93F8203001
:10CAA00003F01F0B5B09032B0AFA0BFA09D0042BC6
:10CAB0000CD0022B7FF458AF4B6C4AEA03034B6453
:10CAC00052E70B6C4AEA03030B644DE70B6B4AEA2F
:10CAD00003030B6348E71848006B054316480563DA
:10CAE00087E71548006C05431348056481E7002378
:10CAF000D0E70123CEE70223CCE70323CAE70423D0
:10CB0000C8E70523C6E70623C4E70723C2E70823CF
:10CB1000C0E70923BEE70A23BCE70B23BAE700BF3F
:10CB200070A700208C240408000400400008004086
:10CB3000000C0040000001400038024038C40020D2
:10CB40009427040890270408BC1D0408A8F80308CB
:10CB5000000401400010004000140040004001406B
:10CB600001490248FFF7AABB38A80020001800407E
:10CB700001490248FFF7A2BB10A8002000040140B1
:10CB800001490248FFF79ABB10A8002000040140A9
:10CB900001490248FFF792BBE8A70020000C0040C3
:10CBA00001490248FFF78ABBC0A7002000040040EB
:10CBB00002494FF08040FFF781BB00BF98A70020DB
:10CBC00001490248FFF77ABB70A70020000001402E
:10CBD00001490248FFF772BB70A700200000014026
:10CBE000F0B504684B4DA30AAB4276D009D94A4D43
:10CBF000AB425CD00135AB4273D03B3DAB425AD027
:10CC0000F0BDB3F5801F64D0023DAB4257D14FF069
:10CC1000700E02264779B0004FEA970C002964D0C5
:10CC200063460227A5899F4083190CEB43032F43DA
:10CC300003F1040C394DBFB245F8231045F82C2000
:10CC4000A781EFF31181502282F31288821905EB3C
:10CC5000C2021369002B33D013620433821905EB2F
:10CC6000C202576917B11F6053690433821905EB7B
:10CC7000C202976917B11F6093690433821905EBEB
:10CC8000C202D76917B11F60D36904330027CAB243
:10CC90001F6082F31188304405EBC000036A93B92A
:10CCA000A38923F001031B041B0CA381F0BD4FF0EB
:10CCB000200E0026AEE74FF0E80E0526AAE7F0BDED
:10CCC00005EB0E03CAE7A3899BB243F00103A381DE
:10CCD000F0BD4FF0480E01269CE74FF0980E03265A
:10CCE00098E74FF0C00E042694E70223BF0803FA2A
:10CCF00007F7A389094D9BB223EA070387190CEBB9
:10CD0000470CA3810CF1040345F82C1045F82320AF
:10CD100097E700BF030010004000100070A700203C
:10CD200010B5036883480139834282B089B200F0AC
:10CD3000CB80A0F58060834200F0C68000F5804083
:10CD4000834200F0B88000F58060834200F0B38039
:10CD500000F58060834200F0AE80774C188824682C
:10CD60006408B4FBF2F4013CA4B282B2B3F1804F88
:10CD70000AD07248834207D000F58060834203D016
:10CD800000F58060834202D122F0700292B26C48BA
:10CD9000834200F0A28000F58060834200F0A7800B
:10CDA00022F4407200F56C4092B283421A80D9623C
:10CDB0001C854FD05F4A93424CD001229A821A8838
:10CDC00092B242F001021A80B3F1804F00F09980D4
:10CDD0005A4A934200F0978002F58062934200F035
:10CDE000948002F58062934200F0918002F58062A7
:10CDF000934200F08E8002F58062934200F08B80B7
:10CE000002F57042934200F0888002F5705293421E
:10CE100000F0858002F58062934200F0828002F586
:10CE2000806293427FD0A2F5983293427DD002F582
:10CE3000806293427BD002F58062934208BF0D224C
:10CE400015D002A84FF0012340F8043D2DF024FD39
:10CE500002B010BD0122002119869A821A88394831
:10CE600092B242F0010283421A80ADD10A46364B9B
:10CE700003EBC20301A893F821408DF8044001237D
:10CE800000228DF805308DF807308DF806202DF042
:10CE900003FD1B2C08D02E2CDAD12C4B019301A8BA
:10CEA0002DF0FAFC02B010BD294B019301A82DF022
:10CEB000F3FC02B010BD204C18882468B4FBF2F4D7
:10CEC000013CA4B282B251E71B4C18882468B4FB21
:10CED000F2F4013CA4B282B256E701201A80D96272
:10CEE0001C8598821A8892B202431A8070E701204A
:10CEF0001A80D9621C8598821A8892B202431A80DD
:10CF000062E70122B3E70222B1E70322AFE704227E
:10CF1000ADE70522ABE70622A9E70722A7E708222B
:10CF2000A5E70922A3E70A22A1E70B229FE70C222B
:10CF30009DE700BF000401402C7000200004004069
:10CF40000010004000000140A8F803082C01000177
:10CF5000190100012C4B98423DD0B0F1804F3CD0DC
:10CF6000A3F57C4398423AD003F58063984238D0C9
:10CF700003F58063984236D003F58063984234D03D
:10CF800003F58063984232D003F57043984230D065
:10CF900003F5705398422ED003F5806398422CD04D
:10CFA00003F5806398422AD0A3F59833984228D09D
:10CFB00003F58063984207D003F58063984208BF69
:10CFC0000D2202D0002070470C22104B03EBC2034D
:10CFD00093F8200070470022F7E70122F5E70222CC
:10CFE000F3E70322F1E70422EFE70522EDE706224B
:10CFF000EBE70722E9E70822E7E70922E5E70A224B
:10D00000E3E70B22E1E700BF00000140A8F80308B6
:10D010002DE98048013085B0C3B203938A4D8B4F10
:10D020008B4C8C4E0A230293DFF82C922DF078FF64
:10D030004FF4FA7A4FF0100C4FF47A70D9F80430AC
:10D04000C3F30803002B40F0C180EFF31183002BE2
:10D0500040F0BC802968A26800BF2B689942F9D1D2
:10D06000D7F800E000FB0EF39B1AB3FBFEF300FBC6
:10D0700001314FF0010E0191D9F80430C3F30803D8
:10D08000002B40F08780EFF31183002B40F082806B
:10D090002B68A16800BF2A689342F9D1D7F800B085
:10D0A00000FB0BF2521AB2FBFBF200FB0323019AC6
:10D0B0009B1AB3F57A7FDFD3BAF1010ABED1039B85
:10D0C000002B40F0BD804FF47A7ADFF88C91504607
:10D0D0004FF0100CD9F80430C3F30803002B40F0D4
:10D0E0009280EFF31183002B40F08D802968A268B5
:10D0F00000BF2B689942F9D1D7F800E000FB0EF38E
:10D100009B1AB3FBFEF300FB01314FF0010E0191BE
:10D11000D9F80430C3F3080303BBEFF31183EBB971
:10D120002B68A16800BF2A689342F9D1D7F800B0F4
:10D1300000FB0BF2521AB2FBFBF200FB0323019A35
:10D140009B1AB3F57A7FE3D3BAF1010AC2D1029BED
:10D15000013B02937FF468AFFEF7C8F8EFF3118844
:10D160008CF31288A1682368DB0344BFC6F800E093
:10D17000A1682B6832685FFA88F888F31188D7F8BD
:10D1800000801A4400FB08F35B1AB3FBF8F300FBC2
:10D190000233D4E7EFF311888CF31288A168236877
:10D1A000DB0344BFC6F800E0A1682B6832685FFA71
:10D1B00088F888F31188D7F800801A4400FB08F338
:10D1C0005B1AB3FBF8F300FB023370E7EFF3118255
:10D1D0008CF31288D4F808E02368D90303D501231F
:10D1E0003360D4F808E02B683168D2B282F311883A
:10D1F0003A68194400FB02F3A3EB0E03B3FBF2F30E
:10D2000000FB013135E7EFF311828CF31288D4F87B
:10D2100008E02368D90303D501233360D4F808E07C
:10D220002B683168D2B282F311883A68194400FB46
:10D2300002F3A3EB0E03B3FBF2F300FB013164E74F
:10D2400018462DF0CFFC3EE7F8C50020FCC50020B5
:10D2500010E000E0F4C5002000ED00E02DE9F0470B
:10D26000AD4FAE4E1CF0B4FFBE421ED2DFF8388385
:10D27000DFF838934446258862197DB14A450DD2BE
:10D28000052D0BD933886188C3F30B03994200F055
:10D29000D880144625886219002DEFD17168304678
:10D2A0001436FDF73BF8BE42E4D39D4B5A78022A70
:10D2B00040F2EC8000225A701A789A489A4901602C
:10D2C000022A00F2DD8002EBC201984B02EB8102E0
:10D2D00003EB4202964C1046226022F00FFC954A66
:10D2E0001378A3F1170102290FD9934911F83300DC
:10D2F000002840F00381D8000144497829B18F49C2
:10D3000011F833300BB9182313708D4B9A78042A17
:10D3100000F0EB8032B91A88B2F5F07F84BF4FF489
:10D32000F0721A80874D884A2B681A40002A00F054
:10D33000EE80DE0700F1B580580400F1B9801907CE
:10D3400000F1BD809A0100F1C1809B0400F1C6800C
:10D3500023689A8CD98C914224BF00229A84FEF7CC
:10D360002DFF28F043FD10B978480FF0DDF82EF0BE
:10D3700017F900213022764832F0AFF9754B256855
:10D3800003F1500102E0043399427DD01A78002A5B
:10D39000F9D19C78D8788442F5D26F496F4B0A70E6
:10D3A00028461D6017F07CF96D4B6E4A1E786E4959
:10D3B0006E486F4B1160C825642212FB06526D4CFB
:10D3C000006B31F8041C5A60002221809A60DA60F8
:10D3D0001A615A619A61DA6183F8202083F821206A
:10D3E00008B11CF031FE644B9FED645A1B88644AFF
:10D3F0009FED646A557B644C64496548086006EE9D
:10D40000903AF8EEE66A1389C5EE265A07EE103A0E
:10D410005389127BC4ED005A07EE903AB8EEC77AF2
:10D420005C4BF8EEE77A1D725A7227EE067A67EEC9
:10D43000867ABDE8F04783ED017AC3ED007A1CF0EF
:10D44000AFBE63799B077FF424AF716894F804A0A2
:10D450003046FCF763FF3388BAEB133F0BD1738878
:10D460007068AA1FC3F30B039A4204F10601A8BF18
:10D470001A462FF0B3FE1436BE42FFF4FBAE14E79B
:10D4800000221A70294A25E7012286E72649254805
:10D4900002EB420201EB82011A780160022AEFD806
:10D4A00011E73D48FCF770FF2B6858047FF547AF44
:10D4B0003A48FCF769FF2B6819077FF543AF3848F6
:10D4C000FCF762FF2B689A017FF53FAF46F2090037
:10D4D000FCF75AFF2B689B047FF53AAF3148FCF705
:10D4E00053FF4020FCF750FF32E71A8BB2F57A7FEA
:10D4F000BFF418AF4FF47A721A8313E7D8000D18EF
:10D500006D68002D7FF4F8AE17251570F4E643F032
:10D5100008032B600DE700BFE8050008880100083C
:10D52000E8C2002018570020FEC20020083C00205E
:10D5300014570020C46800202C1E0408A40C040802
:10D5400030700020583D002009600002C4B900205E
:10D55000481F0020C8680020901C00207C1F00206D
:10D56000AC640020DC1F002098680020C856002012
:10D57000404B00209C520020EC220020C0C9FB48F8
:10D58000801E002017B7D138F0220020E05B002079
:10D590003661023DBC5B00200860000209200002E9
:10D5A00001600002094000020740000800800008F6
:10D5B0002DE9F0430B684A680B388BB00C46D51A3E
:10D5C000EF2800F27881DFE810F07C017601760127
:10D5D0007601760176017601760176017601760193
:10D5E0007601760176017601760176017601760183
:10D5F00076017601760176017601EA0176018A02EA
:10D6000076017B02760176017601740276012602AC
:10D610007601D2017601C1017601BA017601940149
:10D620007601520176017601760176014D0176018F
:10D6300032057601760126057601760176017601BE
:10D64000760176017601760176017601080576018C
:10D65000E204760176013E057601760176017601D7
:10D66000760176017601F000760154057601B20468
:10D670007601DC057601D00476017601760176012B
:10D6800076017601760176017601760176017601E2
:10D6900076017601760176017601760176017601D2
:10D6A00076017601760176017601760176017601C2
:10D6B00076017601760176017601760176017601B2
:10D6C00076017601760176017601760176017601A2
:10D6D0007601760176017601760176017601760192
:10D6E0007601760176017601760176017601760182
:10D6F0007601760176017601760176017601760172
:10D700007601760176017601760176017601760161
:10D710007601760176017601760176017601760151
:10D720007601760176017601760176017601760141
:10D730007601760176017601760176017601760131
:10D7400076017601AF058B04720476013504FF0380
:10D75000F3037601E803BA03A803A1037703760174
:10D76000640376017601550340033803260316034C
:10D770000703F302E902760176017601760176016C
:10D7800076017601760176017601760176017601E1
:10D790007601DE0276017601B3027601760176012A
:10D7A00076017601760176011B020846FDF742F804
:10D7B000054617F021F8FF2854D0B5F57A7F80F0A0
:10D7C00033850AAF002307F8243DEE0839460DF1F2
:10D7D00003008DF80330013616F0EEFF9DF803309C
:10D7E000F6B205F00705B34205F1010503D19DF836
:10D7F0000430AB4203D02946304616F0E9FF94E8E6
:10D800000C009B1A012B2DDD531C0AA8236000235A
:10D81000157800F8253D16F0C3FF9DF80330AB42A4
:10D820000AD0B44B1B683BB19A79AA4204D31B6857
:10D830001B690BB12846984723685A1C226038465A
:10D8400000221C788DF8042016F09EFF9DF804300D
:10D85000A34207D0A74B1B6823B11B685B690BB1C0
:10D8600020469847012318460BB0BDE8F083A24933
:10D87000A1FB05216A1A01EB52018908C1EBC10223
:10D88000B5EB020817D1C9B24E1EF6B20029E9D095
:10D89000DFF8689201365A1C226093F90010974B0A
:10D8A000002593F902208A4203F1080300F09784CF
:10D8B0000135062DF5D14FF0FF3318460BB0BDE80A
:10D8C000F0838F49102D4FF0000328BF10250B6007
:10D8D0004B608B60CB600B74002DC3D023685A194A
:10D8E0000133236013F8010C01F8010B9A42F7D1C0
:10D8F000B8E75A1C0A601A780E2ADCD8991C2160F5
:10D9000058780328D7D87F4D02EB42025200A9185D
:10D91000DE1C487126609878A8541A1D2260DA78B7
:10D920004A705A1D22601A798A709A1D22605A79AB
:10D93000CA70DA1D22609B790B71012393E75A1C90
:10D940000A60714A1B78537501238CE75A1C0A60E0
:10D950001E781F2EAFD8052DADD10846FCF752FF1B
:10D960006A4B43F8260018F0E1FA01237BE7674D84
:10D9700005F140062046FCF75DFF2368A5F880000E
:10D98000591C1A46216012F8021B85F88210226089
:10D990005B7885F883300435AE42EBD162E75A1CE0
:10D9A0000A601E78132E86D89A1C0A6000205D78C3
:10D9B0005749024605E00132242A3FF47CAF11F8B2
:10D9C0000C0C854201F10C01F5D15248524902EB91
:10D9D000420210F8222001F82620D81C206001EB1A
:10D9E000860299785170191D2160D8789070581D61
:10D9F00020604A491B790868D3702DF05FFD31E73C
:10DA0000474B1B78DB073FF556AFFEF721FEFFF7CC
:10DA100025FC012327E75A1C0A603B4E1B78337212
:10DA20000846FCF707FFB0832046FCF703FF30836E
:10DA30002046FCF7FFFE236870835A1C22601B7887
:10DA4000F374082D7FF60EAF2046FCF7F3FEF0844A
:10DA50002046FCF7EFFE0C2D30857FF603AF2368E0
:10DA60001A46591C216012F8021BB17722605B78BC
:10DA700086F820302046FCF7DDFE102DB0847FF6BE
:10DA8000F1AE23685A1C22601B78F3722046FCF723
:10DA9000B9FE2368F0605A1C22601A783274162D81
:10DAA0007FF6E0AE9A1C22605B7886F82130012375
:10DAB000D9E65A1C0A601B4A1B7813700123D2E670
:10DAC0000846FCF7B7FE184D28602046FCF7B2FE6A
:10DAD00068602046FCF7AEFE0123A860C3E6134D44
:10DAE00000232B600846FCF78DFE2B681843286046
:10DAF0000123B8E65C3D002025499224C4B90020EA
:10DB0000EDC200208C3A00200C7500204058002007
:10DB1000FCF90308E8F90308C8680020145700203E
:10DB200020660020C4680020F0380020583D002006
:10DB30005A1C0A601A780F2A3FF6BDAE991C216064
:10DB4000C2EBC202A64958788854D81C20600A4407
:10DB500099785170191D2160D9789170591D2160F3
:10DB60001979D170991D216059791171D91D2160E0
:10DB70009979517103F108012160DB79937121F0EA
:10DB80004FFC01236FE60846FCF754FE954DA88133
:10DB90002046FCF74FFE0123688164E60846FCF747
:10DBA00049FE914B00EB80004000188001235AE6AB
:10DBB00019465A1C22608D4A11F8020B1070216020
:10DBC00059785170D91C216099789170191D216084
:10DBD000DB78D370012346E60846FCF72BFE844D24
:10DBE000A8822046FCF726FEE8822046FCF722FEAB
:10DBF0000123288337E61A46591C216012F8020BCC
:10DC00002260DA1C597822609A781FF029FB0028DC
:10DC10007FF428AE4FE61A46591C2160754912F868
:10DC2000020B087022606F495A788A70DA1C2260F1
:10DC30006D4A9B789370012315E66F4B6F49186806
:10DC40004A222FF0CBFA01230DE619465A1C226016
:10DC50006B4A11F8020B1070216059785170D91C71
:10DC600021609B7893702046FCF7E4FD654A012310
:10DC7000D080F8E50846FCF7DDFD624D288020469F
:10DC8000FCF7D8FD68802046FCF7D4FD0123A8806E
:10DC9000E9E55D4F3B78002B3FF4E4AD5B4E00259A
:10DCA0002046FCF7C7FD22F071F83B78A6EC010A8C
:10DCB0000135AB42F4DCD5E50F2D7FF4FCAD5A1CE9
:10DCC0000A601D78072D3FF6F6AD0846504F05EB6C
:10DCD0004505FCF7AFFDAD007E19B0802046FCF78E
:10DCE000A9FDF0802046FCF7A5FD236830811A4687
:10DCF000591C216012F8021BB17222605B78F3722A
:10DD00002046FCF77FFD01237851ACE50846FCF77F
:10DD100091FD404A01231080A5E55A1C0A6018783D
:10DD2000050600F1E4823C4B1B78DC073FF59AAD19
:10DD3000032828BF0020FEF76FFC012393E55A1C3F
:10DD40000A6008461D78FCF75DFD80462046FCF71A
:10DD500059FD07462046FCF755FD06462046FCF7D0
:10DD600069FD2046FCF766FD236801332360002D22
:10DD700000F0A982102D7FF475AD284BC3F8008008
:10DD80005F600EB1264B1E602649274B0222081FFA
:10DD90001A7016F023FC012365E51F4B1B78D8078A
:10DDA0003FF560ADFEF788FCFFF758FA01235AE50E
:10DDB000194B1B78DA073FF555AD1C4A137843F031
:10DDC0000403137001234EE5134B1B78D9073FF56D
:10DDD00049AD174B4FF4C8721A80012343E500BFC9
:10DDE000585D002094680020AC680020EC4C0020B6
:10DDF00030700020F8B9002014570020E80904080A
:10DE00008C680020946400201A4F00209C6300203E
:10DE10002C650020D44C002020660020801F0020AC
:10DE2000E0220020841F0020BE4B002091560020DD
:10DE30001AC60020092D7FF63EADA94F1A46591C7F
:10DE40003E68216012F8021B317022605A78B2706D
:10DE5000DA1C22609A78642A03F10401A8BF6422C4
:10DE600072712160DA78642A03F10501A8BF642287
:10DE7000B27121601A79F2719A1D22605A79642A6E
:10DE800028BF6422D91D327221609A79F27003F1A1
:10DE900008022260DB7933712046FCF7CBFC0A2DA7
:10DEA000708140F02E822DF07BFB0123DBE48D4A54
:10DEB0001068DA1C01462133951E256012F8035CB8
:10DEC0000D70551E256012F8025C4D70226012F82C
:10DED000015C8D7003329A4201F10301ECD179E1CA
:10DEE0005A1C0A601A788049002A00F099810A7841
:10DEF00042F00202981C0A707C4D20605B782B7007
:10DF00002046FCF77FFC68602046FCF77BFCA8609D
:10DF10002046FCF78FFCA8812046FCF78BFC744A56
:10DF20006882137843F00203137001239BE45A1CA8
:10DF30000A606C4FDFF8E4811B783E6888F8053092
:10DF40000846FCF777FC308420463E68FCF772FCFC
:10DF5000052D708400F29581FEF730F92BF0CAFA96
:10DF6000386821F005FC01237DE41A46591C216024
:10DF7000604912F8020BC87022605F495A780A7033
:10DF8000DA1C22605D4A9B78D37001236BE45A1C33
:10DF90000A601E78112E3FF68EAC9A1C0A60584D0E
:10DFA0005B7805F816300846FCF744FC40F6CA03D7
:10DFB0009842A8BF184640F2EE239842B8BF1846D0
:10DFC000504BA0F2EE2083FB002305EB4605C01763
:10DFD000C0EBE3036B70012345E41A46591C216032
:10DFE000494D12F8021B297022605B786B70204645
:10DFF000FCF720FC236868805A1C22601B782B7178
:10E000002046FCF717FC2368E8805A1C22601B7826
:10E010002B72012327E43D4A03F1080001332360FA
:10E0200013F8011C02F8011F9842F7D11AE4591C99
:10E030001A462160364912F8020B887022605B781C
:10E040004B7001230FE4334A1278012A3FF60AACE1
:10E0500019465A1C2260304A11F8020B9070216058
:10E0600059781170D91C21609B7853700123FFF7F8
:10E07000FABB1A46591C2160284E12F8021BB170D7
:10E08000226027495A780A70DA1C2260254D9A7856
:10E090002A711A1D2260DB78092BA8BF09232046AC
:10E0A000AB70FCF7C7FB236862682880D11A01298E
:10E0B00005DD2046FCF7BEFB626823686882934258
:10E0C00040F0D780FEF77AF8236862689A423FF4FE
:10E0D000C9AB5A1C22601B78EB700123FFF7C3BB4E
:10E0E0001857002014570020915600209456002005
:10E0F000BC4B002094680020A4680020AC6800207D
:10E10000685400201F85EB51AC6400200B75002083
:10E11000B86800204C7600204D760020F8B9002029
:10E120008868002030700020C5F34705122D3FF6A7
:10E13000C2ABBDB10AAB0DF1020703EB45083E4689
:10E14000A8F126082046FCF775FB26F8020FB0451B
:10E15000F8D1734B37F8022F23F8022FBE42F9D1C2
:10E16000112D09D86F4A6B00023B13440021223263
:10E1700023F8021F9342FBD16B4A01231370FFF770
:10E1800072BB0846FCF756FB2046FCF753FB2046C3
:10E19000FCF750FB2368654F9A1C3E6822605A7852
:10E1A00086F82F20DA1C22609A7886F83A201A1D09
:10E1B0002260DA7886F83B20073323602046FCF79C
:10E1C00039FBF08720463E68FCF734FB112DB08701
:10E1D00041D8386821F0B8F90123FFF744BB09EBB7
:10E1E000C5072046B970FCF725FB216829F83500E2
:10E1F0000B464A1C226013F8022BFA7023604B78FE
:10E200003B71CB1C23608B78BB710B1D236008F125
:10E210000108CA787A7146457FF43DABFFF722BB0F
:10E220000A7802F0FD0265E601AF384616F0A0FA62
:10E23000BDF80430AB423FF4E2AA3D4B1B68002B13
:10E240003FF4DDAA1B689B69002B3FF4D8AA28463F
:10E250009847FFF7D4BA23683868591C1A462160DA
:10E2600012F8021B80F8311022605B7880F832309F
:10E27000B0E75A1C22601B78003318BF0123F371EA
:10E2800020E72046FCF7D6FAA8F80A002046FCF75B
:10E29000D1FAA8F80C0020463E68FCF7CBFAB0840F
:10E2A00020463E68FCF7C6FA0D2DF0847FF654AE8A
:10E2B0002046FCF7BFFAA8F80E002046FCF7BAFA91
:10E2C000A8F8100048E61B4B1020C3F800805F60E0
:10E2D0000FF09EFD184A137843F001031370002ECF
:10E2E0003FF4C0AA154A01231660FFF7BCBA00F03C
:10E2F0007F00032828BF002010F02CFB0123FFF72C
:10E30000B2BA23683A68591C2160197851720B2DF2
:10E310003FF4C9AD991C21605B785370C3E500BF21
:10E320003A5A00203C5A0020385A00201457002046
:10E330005C3D0020004C002091560020E02200208F
:10E3400008B51BF045FFFCF765F81BF029FFFEF749
:10E3500085FF0120BDE808400FF042BD2DE9F04FD8
:10E36000013085B0C3B203930B4602918B4C8C4EA7
:10E37000002B00F099808B4D8B4FDFF830922CF002
:10E38000CFFD4FF4FA7A4FF0100C4FF47A70D9F8B1
:10E390000430C3F30803002B40F0DE80EFF3118359
:10E3A000002B40F0D9802968A26800BF2B689942F1
:10E3B000F9D1D7F800E000FB0EF39B1AB3FBFEF394
:10E3C00000FB01314FF0010E0191D9F80430C3F385
:10E3D0000803002B40F08780EFF31183002B40F0FF
:10E3E00082802B68A16800BF2A689342F9D1D7F8D0
:10E3F00000B000FB0BF2521AB2FBFBF200FB03234E
:10E40000019A9B1AB3F57A7FDFD3BAF1010ABED124
:10E41000039B002B40F0BD804FF47A7ADFF88C919B
:10E4200050464FF0100CD9F80430C3F30803002B0A
:10E4300075D1EFF31183002B71D12968A26800BF59
:10E440002B689942F9D1D7F800E000FB0EF39B1A34
:10E45000B3FBFEF300FB01314FF0010E0191D9F83F
:10E460000430C3F3080313BBEFF31183FBB92B682C
:10E47000A16800BF2A689342F9D1D7F800B000FB29
:10E480000BF2521AB2FBFBF200FB0323019A9B1A18
:10E49000B3F57A7FE3D3BAF1010AC4D1029B013B01
:10E4A0000293002B7FF467AF05B0BDE8F08FEFF368
:10E4B00011888CF31288A1682368DB0344BFC6F877
:10E4C00000E0A1682B6832685FFA88F888F3118849
:10E4D000D7F800801A4400FB08F35B1AB3FBF8F38B
:10E4E00000FB0233D2E7EFF311888CF31288A168A6
:10E4F0002368DB0344BFC6F800E0A1682B683268DC
:10E500005FFA88F888F31188D7F800801A4400FB76
:10E5100008F35B1AB3FBF8F300FB023370E7EFF389
:10E5200011828CF31288D4F808E02368D90303D54C
:10E5300001233360D4F808E02B683168D2B282F34B
:10E5400011883A68194400FB02F3A3EB0E03B3FBF6
:10E55000F2F300FB01317FE7EFF311828CF31288B5
:10E56000D4F808E02368D90303D501233360D4F835
:10E5700008E02B683168D2B282F311883A681944F6
:10E5800000FB02F3A3EB0E03B3FBF2F300FB01313C
:10E5900018E718462CF026FB3EE700BF10E000E02D
:10E5A000F4C50020F8C50020FCC5002000ED00E007
:10E5B0002DE9F04FDFF830C1474A4849484E494DF0
:10E5C0008046102718F1FF38C0F08480DCF8043052
:10E5D000C3F30803002B5CD1EFF31183002B58D158
:10E5E0000B68946800BF08688342F9D1D6F80090A0
:10E5F0004FF47A7000FB09FEAEEB040EBEFBF9FE91
:10E6000000FB03EEDCF80430C3F308034FF47A7424
:10E610000120FBB9EFF31183E3B90B68D2F808A02E
:10E6200000BFD1F800904B45F7D1D6F800B004FBFD
:10E630000BF9A9EB0A09B9FBFBF904FB0393A3EB64
:10E640000E03B3F57A7FBDD2DCF80430C3F30803C0
:10E65000002BDFD0EFF3118A87F31288D2F808B0CD
:10E660001368DB0344BF2860D2F808B00B68D5F804
:10E6700000905FFA8AFA8AF31188D6F800A09944CC
:10E6800004FB0AF3A3EB0B03B3FBFAF304FB09331C
:10E69000D5E7EFF3118487F31288D2F80890136856
:10E6A000D80303D501232B60D2F808900B682868A3
:10E6B000E4B284F31188D6F800A04FF47A7400EB2A
:10E6C000030E04FB0AF3A3EB0903B3FBFAF304FB09
:10E6D0000E3E97E7BDE8F08F10E000E0F8C500209F
:10E6E000FCC50020F4C5002000ED00E02DE9F04F4E
:10E6F0009A4A9B49137895B00446099000F59C40CE
:10E7000020300C900860002B00F032849549096895
:10E710008C4240F296809449059109689348944D43
:10E72000DFF888B20391013B137001F4805302902B
:10E730000893002B40F09480029B5B7D002B40F0FF
:10E740006083039B180400F16386039BD9050BD5F6
:10E75000099A884BDFF858A29A429AF8022001F2EF
:10E760001D80002A41F01E80834B0493834C039B41
:10E7700013F4805740F0A483029BBBF906605B8BC7
:10E780009E42B4BF002601267D4B1B6813F08053C8
:10E7900073D0049A127812F0010275D00298794968
:10E7A000808C91ED037A07EE900AF8EEE77AB4EEEA
:10E7B000E77AF1EE10FA80F20487002E69D195F81D
:10E7C000A410002965D170487049006890F83000A5
:10E7D0004FF0000EC1F800E0C1F804E0C1F808E015
:10E7E0006B49002856D10870002A57D0039AD006EA
:10E7F00054D5684A1278D10650D4002F4ED1002B40
:10E800004CD1039B5A0249D494F800C0BCF1000FCC
:10E8100001F05286604B9B78002E41F076863BB12A
:10E820005E4A5F4B12681B689B1A002BC1F29B86E5
:10E8300010200FF0C1F9012385F8A53094F800C02D
:10E840002EE0494B05931B680393484A484D0292BA
:10E8500003F48053DFF854B10893002B3FF46CAFFE
:10E8600000214748FCF7DCFB00287FF465AF14F07B
:10E870001DFE059B1B6803935EE7039A520288D432
:10E88000049A127802F00102002185F8A410002EEB
:10E8900099D03F4901200870002AA7D194F800C000
:10E8A000029ABBF900E0508B918BBBF902208645A0
:10E8B000CCBF8027002747F040038E45A8BF3B46CA
:10E8C0009B0843F080078242C8BF3B4643F04007A5
:10E8D0008A42B4BF3A461A469208BBF904E0BBF933
:10E8E000067042F080038645C8BF1A4642F04003D6
:10E8F0008E45A8BF13469B0843F080028742D4BFD1
:10E900001846104640F0400295F8A6308F42ACBF42
:10E91000014611468B4200F08F84002385F8A61033
:10E9200085F8A730BCF1000F00F0F885059B1D4A63
:10E930001B68039203F00403002B40F02C840DF1BC
:10E940004808194C0023C8F8043004F15009129308
:10E9500040F6330A192740F283362EE0CC530020CC
:10E9600098520020C8530020D48600200C75002047
:10E97000981E0020404B4C0020660020901C002078
:10E98000D866002064500020145700203C66002008
:10E99000DC24002091560020B8680020F8C5002033
:10E9A000EC3B0020B0690020C868002088A500204A
:10E9B000404B002004344C4520D0A278E3789A42A2
:10E9C00017FB0261F6D26278043217FB03633BF94E
:10E9D00012205245A8BF5246B2F5617FB8BF4FF42E
:10E9E00061728A42E6DD9A42E4DC21782329E1D88B
:10E9F00040460434FCF704FB4C45DED1AD4B98E8AF
:10EA000003001E78AC4B83E80300002E00F0538314
:10EA10000121A948FCF704FB002840F00D81059B6B
:10EA20001B68D90500F10381A44C23881EB226F08F
:10EA300001061FFA86F84345A4F8008000F07084B0
:10EA40009F4E02270F204FF0140A4FF0FF09377036
:10EA500086F801A086F802900FF0AEF83946964885
:10EA6000B4F80080FCF7DCFA002840F0DE8728F0DC
:10EA700002039BB2434523800BD0914B1421FF220C
:10EA800002260F201E7059709A700FF095F8B4F896
:10EA900000808C4BDFF848A21978DAF80400029362
:10EAA00018F0030F08BF81F00201C1F34001FBF72A
:10EAB00051F9039B1B6813F00A0F1DD005217E48F6
:10EAC000FCF7AEFA002800F014852688730740F1A1
:10EAD000518779480621FCF7A3FA002800F0F68454
:10EAE000770640F1648707217348FCF799FA0028FC
:10EAF00040F0A781039B1B68980600F1B28126882D
:10EB00006D480C21FCF78CFA002800F0B48046F424
:10EB10008073B342238009D0694B02251421FF2260
:10EB20000F201D7059709A700FF046F8664B1B78D5
:10EB3000082B00F0AC800E2B00F0A980059B1B6811
:10EB40005E0542D5614B1B79002B58D014215A48E1
:10EB5000FCF766FA002856D11EF056F801200EF098
:10EB60004FFF90B3DFF87C8100254FF0CC0902E025
:10EB7000DDB2022D29D809FB05F76B1C58F8076098
:10EB8000002EF5D1C378524A90F9020052F8233092
:10EB9000019603220092012132460DF007FF034641
:10EBA00005EB450000EB0010059353B1314608EB2F
:10EBB0008000CC2230F091FD059B48F807300135EC
:10EBC000EDB22AF03DFC0028D3D1049B1B78DD0771
:10EBD00040F18A803F49404A01230B701370029B29
:10EBE000DAF80000197801F00101FBF7B3F8039B94
:10EBF0001B685A0700F1E88015B0BDE8F08F049B50
:10EC00001B78D807A8D53C2029F052F90028DCD081
:10EC100010F026F93C2029F0EDF80028D5D010F0AE
:10EC20001FF93C2029F0E6F80028F1D1CDE72B4B65
:10EC3000DB78002B3FF4F8AE039B1B689A077FF547
:10EC4000F3AE1E4CB4F8008018F0010F7FF40FAF44
:10EC500048F00103984523803FF409AF184B142175
:10EC6000FF2202260F201E7059709A700EF0A4FF2A
:10EC7000B4F80080FBE626F480739BB2B342238095
:10EC80007FF44AAF104B1B78082B7FF454AF2288D7
:10EC900022F040039BB29A4223803FF44FAF084BCF
:10ECA00002251421FF220F201D7059709A700EF05A
:10ECB00083FF43E7CCC20020D86600201057002015
:10ECC000A43B0020C0C50020C46800205450002090
:10ECD0006809040821660020F4220020404B00202F
:10ECE000C4C5002070A10020814B93F80090B9F1B9
:10ECF000000F5FD1DFF874827E4F18F8030C3E7866
:10ED00004146A8F103052CF0A9FB002800F0288358
:10ED1000002E40F07A8305F1080168792CF09EFB03
:10ED2000002841F052827449A87A2CF097FB002801
:10ED300000F02983022E41F04C827049E87B2CF0D0
:10ED40008DFB002841F031826D49287D2CF086FB37
:10ED5000002800F02983042E41F02B826949687E47
:10ED60002CF07CFB002841F028826749A87F2CF01A
:10ED700075FB002800F02983062E41F022826349AA
:10ED800095F823002CF06AFB002840F06D8760495D
:10ED900095F828002CF062FB002800F02983082E4B
:10EDA00040F078875B4995F82D002CF057FB002840
:10EDB00040F02983584B01221A702CF0D4FD039B9C
:10EDC0001B685A077FF518AF03202CF071FB002851
:10EDD00000F04086238813F008047FF40DAF08206C
:10EDE0000FF02EF84D484E4D4E494F4A4F4BBBF851
:10EDF000066000682E80086014601C6015B0BDE8D5
:10EE0000F08F029A013BD27D3BF91330002A40F08B
:10EE10009E83A3F57A73B3F57A7FA8BF4FF47A7314
:10EE200023EAE37307EE903A9FED417AF8EEE77A32
:10EE300067EE877A3F4AFCEEE77A17EE903A138046
:10EE400083E43D4B3D4AB3F904303D4982FB030264
:10EE5000DB17C3EBA202039B0A801B6898067FF5B1
:10EE60004EAE384B1B78990704D5374F3B78042BAF
:10EE700000F28B86268816F0300F3FF441AE10204A
:10EE80000EF0C6FF20200EF0C3FF304B2688002274
:10EE90001A702F492F48304F304D00220A603049F8
:10EEA0003A6000232A6042608261036083604361AC
:10EEB000C3610B604A608B604B618A61CB611FE666
:10EEC0001D212848FCF7ACF800287FF455AC264AF1
:10EED000029BD2881B8BBBF90660991A8E4240F3C5
:10EEE0003F8613449E42B4BF002601264CE400BF77
:10EEF00021660020280000207F3B0020843B00206A
:10EF0000893B00208E3B0020933B0020983B002053
:10EF10009D3B0020A23B0020F4220020B856002098
:10EF2000D4220020E0220020D8220020D02200207D
:10EF3000AAF1823F3A4B0020C05600206766666601
:10EF4000C82200209156002094560020BE4B00207D
:10EF5000B44C0020644C0020B0240020502300203A
:10EF60008C4C0020D866002094640020753B002063
:10EF70009A4D9B4B2E7802939A4F002E00F0F08210
:10EF8000B6B1DFF8A092DFF8A0B2DFF85882CA4627
:10EF90000024072C4046E1B27B6841F35082984739
:10EFA00000B20134A6422BF8020F0AF1040AF0D194
:10EFB0008D4B05931A4609998C4B12680392A3FB5B
:10EFC000013E42F2010313404FEA9E1E079300F0F8
:10EFD000C3828748874A884B007888490690127810
:10EFE0001A70069B08702BB1834B93F800B08BF01E
:10EFF00001030693824A0299127838781090B1F88A
:10F000002680088D91F822C00B92098B0B9A1191E2
:10F0100095F829107B4B0E9008461146A3FB01136F
:10F020005B0803EB4303D31ADBB20D93039B2C78ED
:10F03000754EDFF8F8B1DFF8F891CDF810800F22A7
:10F040000CF1040C03F4805385F828200A955FFA2C
:10F050008CFC109D0F92A2460893002180461097C9
:10F060002CB9AC4599BFE2466446AA462C46A1425B
:10F0700080F22583069B002B00F0D682634B049818
:10F0800033F9112097B287424FEA410303D30E9818
:10F09000874240F20F8359F82120964580F0CE82B6
:10F0A0003BF90320079F002F40F0E2822BF803205A
:10F0B00001310636D4E7DFF87C91554F09F15A0447
:10F0C0004FF00108494619F8010C2CF0C7F9F8B1C6
:10F0D00099F8040099F8023099F803E000EB400138
:10F0E00005EB8101013BD1F8B42003EB43033B4422
:10F0F00093420DD095F8E02081F8B0E008FA00F0D6
:10F1000022EA0000C1F8B430C1F8B86085F8E00028
:10F1100009F106094C45D5D13E493F4A374B0968AC
:10F12000D2F8009093F800A03C4C0691002663684A
:10F130005BB31F784FB3A268A9EB0202002A0ADB77
:10F1400095F8E0200121B14022EA010209F5FA71A7
:10F1500085F8E020A160BAF1000F16D02278597826
:10F160000432D2B2002940F0318202993BF91220D8
:10F17000098B01F1C800824240F3C68495F8E02073
:10F180009B783241D20740F146850136042E04F1C6
:10F190000C04CCD13CE495F8AB3053B1049B1B7804
:10F1A000D90706D5029BBBF906205B8B9A4200F378
:10F1B000248511211A48FBF733FF002800F0E8816D
:10F1C00095F8AE302BB995F8A93013B93223A5F8CC
:10F1D000AC30012385F8AE30FFF7B1BB981E00209C
:10F1E0000C7500203CC30020D4860020D34D621053
:10F1F000745200200C0900200D090020314B002022
:10F20000CD530020ABAAAAAAC41E00209C1E002039
:10F2100034F9030818570020F8C50020481F0020C3
:10F22000D8660020345400209A1E002088A50020B3
:10F23000D05300208D3A002095F8A790B9F1F90F2E
:10F2400000F2B88109F101095FFA89F985F8A79000
:10F2500085F8A610BCF1000F00F06181B9F1140F20
:10F260007FF464AB5F2940F06D81049E337813F026
:10F27000010300F0558714F019F9337803F0010306
:10F28000002B7FF453AB95F8A620572A00F0B886E0
:10F29000059B1B6813F0040302D05A2A00F0FE8479
:10F2A0005D2A00F01E875B2A00F036875E2A00F098
:10F2B000B884562A00F0B78723782BB16F2A00F064
:10F2C000A287CB4B00211960972A00F0A087A72ABC
:10F2D00000F086840021BB2A129101F06180B72AD8
:10F2E00001F03E80BE2A01F05E80BD2A01F06480FC
:10F2F000792A01F09D807A2A01F093809E2A01F0FC
:10F3000089809D2A01F07E80AE2A01F06780AD2AB7
:10F310007FF40CABFF21002022F004FCFFF706BBBA
:10F320000221B448FBF77CFE00283FF4A0AB268006
:10F3300018F0020F7FF4ADAB48F002034345238081
:10F340003FF4A7ABAC4B022214211A700F20FF220E
:10F3500059709A700EF030FCB4F80080FFF799BB3A
:10F3600008F1050168792CF079F800283FF4DBAC4E
:10F37000012E40F02A8705F10D01A87A2CF06EF8D5
:10F38000002840F026879D49E87B2CF067F800288C
:10F390003FF4DAAC032E40F008879949287D2CF021
:10F3A0005DF8002840F005879649687E2CF056F8F5
:10F3B00000283FF4DAAC052E40F0FF869249A87F82
:10F3C0002CF04CF8002840F0FC86904995F823007A
:10F3D0002CF044F800283FF4DAAC072E40F04484C7
:10F3E0008B4995F828002CF039F8002840F0528419
:10F3F000884995F82D002CF031F800283FF4DAAC5C
:10F40000092E3FF4D7AC4FF009094B4600F02FBC52
:10F41000D5F88C30099AD31A002BFFF696A97E4AAC
:10F4200095F89030517C7D4A029C32F811200C985E
:10F43000A17DC5F88C00013303F00F0385F89030EF
:10F440002B4492B292FBF1F283F8942095F8940049
:10F4500095F8951095F8962095F8973001440A4450
:10F4600095F8980095F899101344184495F89A2047
:10F4700095F89B3001440A4495F89C0095F89D103E
:10F480001344184495F89E2095F89F3001440A448F
:10F4900095F8A00095F8A1101344184495F8A230EF
:10F4A00095F8A32001440B441A4442F30B12642A3A
:10F4B000E17DA8BF642213B209B1C2F1640307EE73
:10F4C000903A9FED577AF8EEE77AB1E426F04003E0
:10F4D0009BB2B34223803FF406AB474B0226142174
:10F4E000FF220F201E7059709A700EF065FBFFF717
:10F4F000FABA238823F00406B6B2B34226803FF45A
:10F50000E8AA3D4B02261421FF220F201E705970DD
:10F510009A700EF051FB2688FFF7DBBAE146002116
:10F520003448FBF77DFD30B3002385F8A83013F095
:10F53000B7FB95F8A730142B7FF4F8A92378002B9C
:10F5400040F0DF87049B1B7803F0010398E6C3F5C6
:10F550003B6308331BB25CE4324B1B78069342E5F5
:10F5600093F822303E780433DBB2B3428EBF2E7064
:10F570002B701E4604E5049B1D4A1B781060DB07B8
:10F5800000F12185B9F1140F3FF47DAEFFF7CEB93C
:10F5900095F8A930002B3FF4D2A9049B1B7813F0F7
:10F5A00001037FF4CCA9012285F8A93085F8AA20AF
:10F5B000FFF7C5B985F8A630BCF1000FAFD0FFF753
:10F5C000B5B9012185F8A410FFF763B9012900F04E
:10F5D000368595F8E0200123B34001361343042E0D
:10F5E00085F8E03004F10C047FF4A1ADFFF710BA08
:10F5F000F03B0020D8660020A43B0020843B002084
:10F60000893B00208E3B0020933B0020983B00204C
:10F610009D3B0020A23B002024A7002040A7002003
:10F6200014AE2341314B0020049B002B40D059F8ED
:10F63000212096454FEA4103FFF432ADB84AB8485D
:10F64000D25CC718002A00F0BA81022A40F0658116
:10F650007A7802EB820202EB820202F2EE2292B28E
:10F66000032940F39280079F12B2002F3FF41EAD92
:10F670000D985F1807440A9800EB4707BA85B8F160
:10F68000000F03D10B9802287FF610ADB6F8028068
:10F690003288B78842441744A24A3FB282FB07022D
:10F6A000A148A2EBE772C75212B24FF00108FDE485
:10F6B0001A464B000EF5967749F82170F2E40F993F
:10F6C0000A9D9A4B109F85F800A00F2942460CBF57
:10F6D0000122002285F8298085F828101A7006D1A9
:10F6E0001B219348FBF79CFC002800F0E58491481F
:10F6F000914B82681968914BC1608A1A0121197077
:10F7000043688F4E9A42029A317088BF002392F864
:10F71000226088BF80F82130089B3878B2F826C074
:10F72000B2F818E00436F6B2002B00F0558186429C
:10F730007B4A40F2C781834E174600210CB98246AE
:10F740000446A14218DA12F8113083B1022B0CD111
:10F750007B7803EB830303EB830303F2EE239BB27B
:10F7600026F8023B01310237E8E73388F8E7CBB2ED
:10F77000032BFAD87346F3E785F800A00B9B724A77
:10F7800001331370089BFEF7D4BF012000FA01F784
:10F790000F9820EA070012B20F9083E412B90122F9
:10F7A0008AF80220694B04931C789AF8218004F0AF
:10F7B00001031B2003932BF07BFEB8F1010F079090
:10F7C00000F0D18104F0020306939AF82020604CE7
:10F7D000DFF884915F4E584F052A00F29580DFE8EC
:10F7E00002F08579032F3E51B8F1010F04BF0523C4
:10F7F0008AF82030039B002B00F0BA80029B386807
:10F80000B3F91810B9F80230002261F30F0263F364
:10F810001F42002361F30F0361F31F43DAF8141052
:10F82000CBF804208142CBF8003080F01E81032306
:10F83000069347F230520323CAF81C208AF820307E
:10F84000338843F00203338013F030FE3A68DAF86D
:10F850001C3013440422CAF818308AF82020B8F16A
:10F86000010F40F037843B68DAF818209A424BD2F7
:10F87000207818B92BF01CFE002845D1338823F0DE
:10F88000020333803A68B9F80630642101FB032390
:10F890004FF4806000228AF820208AF80320CAF8FA
:10F8A00010300EF0B5FA9AF8202095E72BF02CFED8
:10F8B000012800F07084079B002B40F05781B8F1BD
:10F8C000010F21D03B68DAF810209A4246D3012379
:10F8D0008AF82030B8F1010FD4D099F80830012B04
:10F8E0003CD020F0BDFF9AF8202075E7039B002B49
:10F8F000DCD1079B4FF48060002B00F0A8800EF055
:10F900009FFA0022CAF81020069B002B40F0A98025
:10F91000059B1B680393FEF72BBF3BF803209FE674
:10F9200068540020565555550C1F002052C3002026
:10F93000D8660020404B0020F8C500200C090020AC
:10F940000D09002088A50020CD530020206600204E
:10F95000901C00200E570020AC64002020F080FF97
:10F96000032240F6B8338AF82020CAF81C3067E733
:10F970003B685EE746F004039E4223800AD0AE4B0C
:10F9800002261421FF220F201E7059709A700EF06B
:10F9900013F92688A94BAA4AB3F90430A94982FB76
:10F9A0000302DB17C3EBA2030B80FFF792B846F00C
:10F9B0004003B34223807FF490ADFFF794B8CAB2FE
:10F9C000022A40F2FD82032AA7D1119A0898049FC7
:10F9D000002808BF3A4643E6864219469A4A4CD860
:10F9E0009A4817460CB9B24634468C427FF7C4AEEB
:10F9F00012F8113083B1022B0CD17B7803EB830317
:10FA000003EB830303F2EE239BB220F8023B0131A8
:10FA10000237E7E70388F8E7CBB2022B03D9032BC1
:10FA2000F8D16346F1E77346EFE728F001039BB294
:10FA3000434523803FF47CAC0F20377086F801A04B
:10FA400086F802900EF0B8F8B4F8008070E40EF07A
:10FA5000DFF956E708200EF0DBF9FFF7CDB80323F6
:10FA6000069306980EF0A8F852E7B8F1010FF6D108
:10FA700003239AF820200693AEE6744E17460CB97D
:10FA800082460446A142BFF677AE12F8113083B128
:10FA9000022B0CD17B7803EB830303EB830303F28C
:10FAA000EE239BB226F8023B01310237E7E73388A9
:10FAB000F8E7CBB2022B03D9032BF8D16346F1E769
:10FAC0007346EFE76148174600210CB9B246344649
:10FAD0008C427FF751AE12F8113083B1022B0CD15A
:10FAE0007B7803EB830303EB830303F2EE239BB2E8
:10FAF00020F8023B01310237E7E70388F8E7CBB291
:10FB0000032BFAD87346F3E7C8398A425BDA95F8D3
:10FB1000E0209B783241D0073FF537ABC3F10008B6
:10FB200001200EF05DF97A1E162A00F25F81DFE8EF
:10FB300012F0F1010502DA013F0123023402B201A1
:10FB40009F018A01750160015D013F014F0134028F
:10FB5000B2019F012B0117010301C501ED00D9007E
:10FB60000126FEF711BE002306932EE699F8043015
:10FB7000002B3FF4A4AE20F073FE03224FF47A73FF
:10FB80008AF82020CAF81C305AE60A202BF090FC94
:10FB900026888046002800F0A882F20640F1CF8334
:10FBA00095F8F080B8F1000F7EF4AAAF0E200EF0A9
:10FBB00003F8012385F8F0302688B8F1000F7FF4B0
:10FBC00068A9FEF79DBF95F8E0300122B24023EA14
:10FBD000020309F5FA7285F8E030A260FFF7D5BAA2
:10FBE0001B49059B0A781B6842F004020A7003F067
:10FBF0000403184A0392FEF79FBE00211648FBF744
:10FC00000FFA00287FF4D5AA322385F8AB00A5F8B7
:10FC1000AC30FFF7CEBA9846002B0CBF0120022073
:10FC20007FE70E4B022203200D4C0E4922700B6021
:10FC30000EF0D6F8FEF77ABEA43B0020C056002096
:10FC400067666666D44C00206854002088A50020B2
:10FC500091560020B0690020D86600209C3C00200E
:10FC6000E8C20020145700204FF007094B4603EB71
:10FC700083031D4487F80090A978687814F0A8FDE4
:10FC8000049BB84A1B7801211170D9077FF595A80C
:10FC9000FEF7A5BF4FF008094B46E8E795F8A92005
:10FCA000002A40F0918395F8AB2082F0010285F89C
:10FCB000AB20002A40F08383AB49096811F400317E
:10FCC00004D0AA490979002940F047840A46A84887
:10FCD000845C0D2C02F10C0200F0D5830131152952
:10FCE000F6D186E7D5F8E400A24B90F83A109A785E
:10FCF00041446429A8BF642121EAE17180F83A10E7
:10FD0000002A40F019841FF01FFC62E4D5F8E400DB
:10FD1000984B90F83B109A784144FE29A8BFFE21E9
:10FD200021EAE17180F83B10002AECD016202BF07C
:10FD30001DFCD5F8E400E6E7D5F8E40081788D4BAA
:10FD40004144C829A8BFC82121EAE17181709B788C
:10FD5000002BD8D014202BF009FCD5F8E400D2E712
:10FD6000D5F8E4004178834B4144C829A8BFC82195
:10FD700021EAE17141709B78002BC4D013202BF055
:10FD8000F5FBD5F8E400BEE7D5F8E4000178794B3F
:10FD90004144C829A8BFC82121EAE17101709B78BC
:10FDA000002BB0D012202BF0E1FBD5F8E400AAE73D
:10FDB0000698704B81799A7841446429A8BF6421E0
:10FDC00021EAE1718171002A40F097830D2F0DD057
:10FDD0000698684B41799A7841446429A8BF642108
:10FDE00021EAE1714171002A40F0B083D5F8E400C6
:10FDF00089E7D5F8E4005F4B017A9A784144C82935
:10FE0000A8BFC82121EAE1710172002A3FF47BAF4B
:10FE10000B202BF0ABFBD5F8E40074E7D5F8E40039
:10FE2000544BC1799A784144C829A8BFC82121EA16
:10FE3000E171C171002A3FF466AF0A202BF096FBF6
:10FE4000D5F8E4005FE7D5F8E4004A4B81799A7869
:10FE50004144C829A8BFC82121EAE1718171002A63
:10FE60003FF451AF09202BF081FBD5F8E4004AE7BD
:10FE7000D5F8E4003F4B41799A784144C829A8BF9E
:10FE8000C82121EAE1714171002A40F03083112F2D
:10FE90007FF454AF37E7D5F8E400364B01799A7810
:10FEA0004144C829A8BFC82121EAE1710171002A93
:10FEB00040F04683102F7FF455AF24E7069A2D4B70
:10FEC00051784144B1F5967FA8BF4FF4967121EA6D
:10FED000E17151709B78002B88D015202BF046FBE8
:10FEE000D5F8E4000FE7069A17794744642FA8BFB6
:10FEF000642727EAE77717712BF052FB1D4B9B789D
:10FF0000002B3FF473AF032039462BF02FFBD5F8BD
:10FF1000E400F8E6069A174B11784144FA29A8BF85
:10FF2000FA2121EAE17111709B78002B3FF45EAF5A
:10FF300001202BF01BFBD5F8E400E4E6069A0D4BFC
:10FF4000917841446429A8BF642121EAE17191704C
:10FF50009B78002B3FF44AAF02202BF007FBD5F82B
:10FF6000E400D0E6F42200205C390020AC560020EA
:10FF70008C0204084D7600200698B24BC1799A781D
:10FF8000414481F30801C171002A3FF42FAF0520DD
:10FF90002BF0ECFAD5F8E400B5E6D5F8E400A94B6F
:10FFA000C1789A784144C829A8BFC82121EAE171E3
:10FFB000C170002A40F095820F2F7FF4E7AEA2E6D1
:10FFC000119AFFF74DBBA04B1B78002B3EF4AEAC53
:10FFD0009E4BDB78002B7EF4A9AC95F8A83001335A
:10FFE000DBB2032B85F8A8307EF6A0AC984B5B788B
:10FFF00013B9002E7EF49AAC13F058FAFFF799BAB1
:020000040801F1
:10000000944B95491A684FF47A73B3FBF2F3C3EB40
:10001000431203EB8203059A1268DB001606A1F86F
:10002000A83000F1E3808D4B03931B68580700F163
:10003000D480059B1B6803F00403FEF77DBC3BF9ED
:1000400012209978B2F5617F4FF4966393FBF1F338
:10005000C0F2988040F633019142A8BF11460C2FA0
:10006000A1F5617191FBF3F800F07781182F7FF40F
:10007000B0AA5FFA88F1C8290B46A8BFC823D5F8F3
:10008000E400C27DDFB297423FF4A3AA9B1A6D4AF7
:10009000C77548BF0733DB1092785F1CFFB23AB9CF
:1000A000002F3FF496AA38460DF09AFEFFF791BA5A
:1000B00018202BF05BFAF3E76449694BCA681B68A8
:1000C0008B609B1AC82B7FF659AB012381F8213036
:1000D000FFF754BB3968DAF81C200A44CAF8182024
:1000E00012E4604B002201209EE5F30600F1088136
:1000F0000B202BF0DDF9002840F0CC80B70600F192
:10010000548195F8F030002B3FF450ADB8F1000F5A
:100110007EF4BFAEFEF7F4BC534B0122022083E510
:10012000524A1268970304D5514A1279002A40F0C6
:100130005D81504819461A46465C0B2E01F10C01B0
:1001400007D00132152AF7D1002285F8A720FFF742
:1001500097B8494ED6F800E05100BEF1000F07D025
:100160008F1800EB87079EF801E07F787745EBD288
:100170000A44424F424900EB82020020326038803C
:100180000860E1E70C2F00F0C580182F7FF421AA4A
:1001900000210B4673E73A68B9F80630642101FB89
:1001A0000323CAF81030FFF786BB4FF003094B4614
:1001B0005DE54FF004094B4659E54FF005094B4604
:1001C00055E54FF006094B4651E54FF001094B4606
:1001D0004DE54FF002094B4649E5059B294A1B684E
:1001E0000A21118003F00403FEF7A6BB264B1B78FF
:1001F0009C077FF518AF254B1B78042B7FF613AFB8
:1002000014F076F90FE712F04BFDFEF78FBB059B5C
:100210001F4A1B684FF4C8711180104A039203F003
:100220000403FEF789BB19F0D3FFFAF7F3F819F0CE
:10023000B7FFFDF713F801200DF0D2FD95F8A620C9
:10024000FFF73AB84D760020314B0020404B00209C
:10025000B868002030C200200CBA0020B06900202D
:10026000F8C50020083C0020523C00205C390020EA
:10027000AC5600208C02040888240020222500208F
:100280002425002018C600209156002094560020F6
:100290001AC60020B94ABA4B528993ED007A07EE8C
:1002A000902AF8EEE77AB0EEC77AB4EEE77AF1EE8C
:1002B00010FA7FF523AF93ED017AB0EEC77AF4EE32
:1002C000C77AF1EE10FA7FF719AFB3063FF519AF11
:1002D00020200DF0B5FDAB497A68BB68C5F8E82071
:1002E000081FC5F8EC3014F079F9A74B01221A70F9
:1002F00095F8F030002B00F0F0802688FEF7C9BD9D
:1003000010200DF085FDA04B268883F800804FF06B
:100310000108EDE60027B8469C4B5B78BB423FF4F2
:1003200058A938460EF016FB994B9B7823B15FFA1B
:1003300088F10C202BF01AF90137FFB2B0E610203B
:100340000DF07EFD20200DF063FD9249081F14F092
:1003500045F98D4B02221A70CAE75FFA88F7DBE78E
:100360000B464FF6FE718C4A8C4854890390908955
:10037000234401445381918119F02AFFFAF74AF886
:1003800019F00EFFFCF76AFF01200DF029FD059B17
:100390001B68002203F0040385F8A720FEF7CCBAFF
:1003A0000B460221DFE70223DDE720200DF030FDC0
:1003B000754B00221A709BE74FF6FE73D3E70C20B3
:1003C0000DF0FAFBFEF7B2BA0122002185F8AA204F
:1003D000724A85F8A9100392FEF7AEBA01210020F7
:1003E00021F0A0FB95F8A620FEF791BF6C4A127889
:1003F000002A7FF49EAE0DF0C3FB049B1B7803F034
:100400000103A1E60021FF2021F08CFB95F8A62036
:10041000FEF77ABF012021F085FB95F8A620FEF7B4
:1004200070BF604A137A43F001031372FEF77EBA7D
:100430005C4A137A23F001031372FEF777BA029A2B
:10044000115D9847032C1BDC40F2EE2240F6CA0CEB
:1004500000283EF4A6AD39F824E0BAF802104FF4B3
:100460007A73A0EB0E0003FB00F0A1EB0E0190FBF2
:10047000F1F018449042B8BF10466045A8BF6046EE
:1004800000B2FEF78EBD484E37684A003FB154189F
:1004900000EB84047F786478BC42BFF4AAAB0A44C2
:1004A00000EB8202414F424C326000213B4A3980CE
:1004B00021600392FEF740BA002E3EF4B9A995F8E8
:1004C000A5C0BCF1000F3EF4EBA90DF059FB94F868
:1004D00000C085F8A570FEF7E3B94FF00108FFF7FB
:1004E00065BB0F202BF042F8D5F8E40064E511203D
:1004F0002BF03CF8D5F8E400C9E40D202BF036F8D9
:1005000064E495F8A610FEF7ADBE3BB129492A4A2E
:1005100009684FF47A7000FB0313136095F8A53057
:10052000002B3EF4BDA90DF02BFB002385F8A53070
:1005300094F800C0FEF7B4B917202BF017F855E473
:1005400010202BF013F8D5F8E400B3E40E202BF0C4
:100550000DF8D5F8E400FFF7D6BB1149097849B189
:100560001146FFF7B4BB12F0A1FF002385F8A530B8
:10057000FEF794B90DF004FBFEF7D8B9584C0020F3
:1005800064500020841F0020BE4B0020E8C20020E1
:100590004D760020044C002094680020B0690020B3
:1005A00062500020DC4C00208824002022250020FE
:1005B00024250020F8C50020EC3B0020F8B55D4B59
:1005C0001B78DB072DD55C4B5C4D1C785C4E012CF9
:1005D00049D079D3022C1BD06B7A7BB1EB886BB1FD
:1005E000584B1B7853B10EF0C9F900287CD0AB7A78
:1005F00083422CBF01230023337000E0337852493B
:100600002A7A9C4238BF1C460C70002A53D1F8BD90
:100610004E494F4A098812889142DDD901241C7045
:10062000DAE74A4B4B48454D1988EC78B0F8F23080
:10063000A142A1EB030303F1020223D32B788B42E7
:1006400020D33D4B1C78032C51D03D4E424A1278AA
:10065000022A04D13B4F414A3F78D7809480012C35
:10066000A0F8F210B5D13A4A38491288E87A0988D8
:10067000121A914235DD3A4A12888A42ACD20024DD
:100680001C70A9E7B1EB440FDBDC2B4B1C78032C6F
:10069000DBD0042AD9D82A4EDFF8A8C0DFF8C0E0A2
:1006A0002B4F0022032434701C708CF80020AEF80D
:1006B00000203A80CAE7012C36D0022C10D1072046
:1006C000BDE8F8400DF078BA254A20491288E87A4A
:1006D0000988121A91423FF77FAF01241C707BE713
:1006E000F8BD02241C7077E70223337087E7042AE1
:1006F000ABD82A7891FBF2F20132082ADFF844E005
:100700006C78AE78164FA8BF08228EF8002092B2FF
:1007100016FB02F614FB02F20D4C3E80084E2280BE
:10072000002434701C7091E70820BDE8F8400DF0FB
:1007300043BA00BF20660020082B0020AC560020E2
:100740000E2B0020625000203D4B00205050002016
:100750000C2B0020981E0020294F00202C4F002039
:100760000A2B00202DE9F04FB74B1E788BB0002EDE
:1007700040F08180B54BB64C1D78B64FDFF8FCB227
:1007800005F00105A4F10A0954F80A0CB8B14FF0BC
:10079000CC0808FB0698F8F70DFF80B154F80A0C56
:1007A000F8F700FF14F8023C024683B924283BD036
:1007B00075B354F80A0CF8F7FDFE0028EED10136A7
:1007C000032E04F1CC04DFD10BB0BDE8F08F012B78
:1007D0002ED0022B33D0032B40D0042B00F06681A7
:1007E000052B00F05481062BE3D114F801ECBEF187
:1007F000000F00F0D581BEF1010F00F01A82013622
:100800000023032E04F8023C04F1CC04BCD1DBE746
:10081000232A54F80A0C00F07F818F4B93F8323072
:100820009342B8D1FAF750FD012304F8023CC0E727
:100830004D2800F06481002304F8023CB9E700234E
:100840003C2804F8023C00F054813E28B1D101223A
:10085000032304F8012C04F8023CAAE7C028EAD8D4
:100860000021042304F8050C04F8040C04F8061C09
:1008700004F8023C9DE7794B18680028A4D0F9F7EA
:10088000E1FC774B774D03F51C7A774B1868F8F746
:1008900091FE002898D0744B1868F8F783FE092859
:1008A0001BD03F2819D02B68002B67D1042800F0FB
:1008B000B8810C2800F0E4807F28E6D0A0F1200267
:1008C000D2B25E2AE1D80BB92028DED067495A1C83
:1008D000C8542A602AF0FCFCD7E72C68002C5AD1B7
:1008E0002646DFF87C8100E0984608F11003002ED0
:1008F00008BF46465345F7D3002E6CD03068D8F871
:100900000020075D135D9F42204402EB040140F08C
:100910004581564F04F1FF3EBE4422460BB9FD2AE5
:100920005DD90EF8013F01322A6010F8013F11F83D
:1009300001CF9C45F2D00AB1B04512D04C482AF004
:10094000CFFCB04508D356F8100B2AF0C9FC09209B
:100950002AF0BEFC4645F6D946482AF0C1FC2A6872
:100960000024944291D2444E264416F8010F2AF0F6
:10097000AFFC2B6801349C42F7D386E70C287FD06C
:100980000A2833D00D2831D07F2800F0BC80FF2BFF
:100990003FF67BAF92E7324FDFF8D0B04FF0000860
:1009A00007F51C79464602E010374F450DD2224626
:1009B000396858462EF0DCFE0028F5D1B846002EE6
:1009C000F2D13E4610374F45F1D3002E96D1B8F103
:1009D000000F3FF45AAF26482AF082FCB3E7511CBF
:1009E0002020B85429607B540A46A5E71F4F2AF0FF
:1009F000D9FC384623212EF0A5FE002800F00F81F7
:100A0000C01B286080B1431EF95C202940F00F8193
:100A1000FA1843B112F8011D202903F1FF3050D11B
:100A20000346002BF6D12B604FF4807200210F4853
:100A30002EF053FE044B1B78002B3FF4C5AE0D483F
:100A40002AF04EFC21E700BFCCC200202066002027
:100A50007AA10020981E0020C4B900206839002027
:100A6000340A0408803A00207C39002080390020B4
:100A7000CC270408D42704087F3900207CF9030818
:100A80007A482AF02DFC7A482AF02AFCFDE614F870
:100A9000063C14F8051C994274D814F8043C8342AF
:100AA0007FF4C9AE062304F8023C9EE614F8043C29
:100AB00004F8030C5A40052304F8042C04F8023C03
:100AC00077E62B606B4C6C4E002204F51C79FA54CF
:100AD00002E010344C4551D2216830460FF078FFC7
:100AE0000028F6D04C4549D2E368984700232B6094
:100AF0009AE7032204F8013C04F8022C59E6022389
:100B000004F8023C55E6013B5B4A5C482B6000213F
:100B1000D1542AF0E5FBB8E6594B5A49DB785A4ADA
:100B2000DFF888E11060003318BF01230B70574BCA
:100B3000574ACEF80030574BC7F8F8204FF0400E18
:100B40000121C7F8F400C7F8FC0087F800E152481B
:100B500087F8015119702AF070FC45482AF0C0FB53
:100B60004E4A4F49138891F8321043F080032329ED
:100B700013803FF457AE14F8023C34E649482AF09B
:100B8000AFFBB3E714F8041C08EB0300514001333A
:100B900004F8041C04F8063C82720AE62246CAE6FF
:100BA0009BE80F000DF1280C0DF1080888E80F00F4
:100BB0004CF824ED14F8053C14F803AC0694624696
:100BC00023444FF0010C414606A8ADF822E00793FC
:100BD000ADF820A08DF824C000F082FA40B1029A4E
:100BE000314B03924146A4F10A0002930EF0D4F86F
:100BF000DDF80480002304F8023CB8F1000F3FF454
:100C0000DEAD54F80A0C0BF009FE013654F80A0C5C
:100C1000C047032E04F1CC047FF4B6ADD4E52868B8
:100C2000F0E615480FF0B0FD0BB0BDE8F08F0346BD
:100C300048E714F8053C14F8032C06942344079362
:100C40006E2A4FF0000308930993ADF820207FF43B
:100C5000D6AD631C06A80693F9F7ECFD06A8F9F7D4
:100C6000E9FD06A8F9F7E6FDC9E500BFDC270408A1
:100C7000D4270408340A0408803900200428040812
:100C8000E8C20020802B00207C390020901F00202B
:100C900089810008CCC20020082804080E570020D3
:100CA000C4B90020E827040840C7002068390020A4
:100CB0002DE9F047B74C636820469847002800F0BC
:100CC0009F80B54B1B780122042B84F8402000F054
:100CD0009980B4F91210B4F91420B4F91630616394
:100CE000A263E363AD4B1B88002B69D0AC4DD4ED00
:100CF0000D7AD5ED004A95ED090A95ED015A95ED6D
:100D00000A7AD5ED035A95ED026AF8EEE76AD5ED59
:100D1000047AA4EEA60AA5EE267A67EEC07AA5EEBE
:100D2000C07AE6EE267A85ED097AC5ED0A7A2CF0CE
:100D3000C9FBD4ED0E6AD5ED0B4A95ED140A95ED7D
:100D40000C5A95ED157AD5ED0F7AD5ED0E5A95ED35
:100D50000D6A6063F8EEE66AA4EEA60AA5EE267AAE
:100D600067EEC07AA5EEC07AE6EE267A85ED147AB3
:100D7000C5ED157A2CF0A6FBD4ED0F6AD5ED164A19
:100D800095ED1F0A95ED175A95ED207AD5ED1A7A53
:100D9000D5ED195A95ED186AA063F8EEE66AA6EE4D
:100DA000A40AA6EE857A67EEC07AA0EE657AE6EE32
:100DB000867A85ED1F7AC5ED207A2CF083FBE063FF
:100DC000784EA17E784819F0C1F83288002A61D1A6
:100DD000764DD5F84431764A1268520720D404F192
:100DE000340007C8B3F90050401B6063B3F9020038
:100DF000091AA163B3F90430D21AE263BDE8F0879F
:100E0000BDE8F0876B4BB4F91200B4F91410B4F9D3
:100E10001620188060635980A1639A80E26361E7BD
:100E2000B5F8AC10322900F08980002967D195F817
:100E3000AA20002AD3D0D5F860115F4E5F4886FB08
:100E40000172C917C1EB22111980D5F8641186FB14
:100E50000172C917C1EB22115980D5F86821278A80
:100E600086FB0261D217C2EB2112D21B9A800023AB
:100E7000C0F80A3085F8AA3019F0AAF9F9F7CAFAC9
:100E800019F08EF9FCF7EAF901200CF0A9FFD5F86A
:100E90004431A4E7454D616BD5F84431B2F5C87FC4
:100EA0004FF0000262631A80308814BFD5F8487191
:100EB0000027B0F5C87F18BFD5F84C21A06B394486
:100EC0003788C5F848114FF0000E0244B7F5C87FC7
:100ED000C4F838E0C5F84C21A3F802E052D0D4F8A9
:100EE0003CC0D5F85001C4F83CE06044012FA3F8A1
:100EF00004E0C5F8500165D0013F37806BE7D5F8B5
:100F00006061626B00203244C5F860216063188024
:100F1000D5F86461A26BA0633244C5F8642158809F
:100F2000E26BD5F86861E06332440129C5F86821B5
:100F3000988073D00139A5F8AC1078E71A8820485A
:100F40001E4E676BA5F854210022B3F802E0B3F8F7
:100F500004C0D6F80A60426082606263C5F86071BE
:100F60001A80A06BC5F86401A2635A80E06BC5F8D3
:100F70006801E263A5F856E1A5F858C1C5F85C61BF
:100F80009A80D7E7E26BC5F85021C4F83CE0A3F89B
:100F900004E0B1E7C8560020294F00209C520020F1
:100FA000A05200201AC60020FC560020981E0020E7
:100FB000D48600202C4F00201F85EB519468002020
:100FC000F81F0020DFF81081DFF8FCC0C83188FB73
:100FD00001A9C832C917C1EBE91188FB02A9D217D0
:100FE000C2EBE9125A801980C83088FB0028218A98
:100FF000C217C2EBE812521A9A80CCF80AE019F034
:10100000E7F8F9F707FA19F0CBF8FCF727F93846B3
:101010000CF0E6FE3788D5F844316DE7274A85F8AD
:10102000AE00126885F8A91012F4003203D0244AE9
:101030001279002A35D11046224E375C0C2F00F170
:101040000C0011D00132152AF7D1B5F854011E4A0F
:101050001880B5F85671B5F85861D5F85C015F8015
:101060009E80C2F80A0065E7184FD7F800C050000C
:10107000BCF1000F09D000EB020E06EB8E0E9CF8BF
:1010800001C09EF801E0E645DFD20244DFF84CE003
:101090000F4806EB820600223E60AEF80020026098
:1010A000D3E70C4A12780AB10246C5E70CF068FD96
:1010B000D5F84431B5F8AC10C7E700BF5C39002063
:1010C000AC5600208C02040894680020882400207C
:1010D00024250020625000201F85EB51222500208E
:1010E0002DE9F04FB0F908502DED048B0D81EDB2D4
:1010F000382D87B00C4600F088838046914634D95D
:10110000802D00F0F68079D8522D00F08E8040F2CC
:101110007182542D00F061836E2D40F031818A4B35
:101120000A681B88894DFF2BA8BFFF23511C216033
:101130001370A96881F3100189B22046F9F7CEFB3C
:10114000834B20461988F9F7C9FB296801F30F0181
:1011500089B220460125F9F7C1FB2B462846638159
:1011600007B0BDEC048BBDE8F08F042D00F0418387
:1011700040F20B82202D00F0A08040F24682242D08
:1011800000F0F182282D40F0FB800B68DFF8E4814D
:10119000704E591C022221601A70236806275A1CBF
:1011A00022601F7023680A22591C21601A7023686C
:1011B00001255A1922601D70B8F800102046F9F771
:1011C0008DFBB8F802102046F9F788FB23685A19FE
:1011D00022601F7023685022591921601A702368F9
:1011E0000022591921601A7031882046F9F776FBE0
:1011F00071882046F9F772FB2B46AFE7822D2FD07E
:10120000C0F05A82A02D00F04582FE2D40F0B8803B
:10121000514D05F1080635F8021B2046F9F75EFB33
:10122000AE42F8D101252B4698E70A684B4E531C75
:101230000321236006F10C071170334606200121BB
:101240002268551C256011702268BB4202F1010121
:101250002160107000F0A2829979D8790633EFE707
:101260000B683F4A394D11783E4A581C206019706E
:10127000D1882046F9F732FB334B22681B88FF2BBD
:1012800002F10101A8BFFF2321601370A96881F357
:10129000100189B22046F9F721FB296801F30F01FB
:1012A00089B22046F9F71AFB2F4B22681978531C94
:1012B000012523602B46117050E70B68294D591CFE
:1012C0006A7821601A7023682A78591C21601A7084
:1012D0002368AA78591C21601A70E9882046F9F71A
:1012E000FDFA23682A79591C21601A7022686979ED
:1012F000DDE71E4E1E4FDFF880A0DFF8809006F17C
:101300000D080A2517E0322D00F05781A5F13C00A9
:10131000C0B2132840F2588100232268511C21607A
:1013200015702268B04502F10101216013703FF48D
:1013300079AF16F8015B0A2DE5D1B9F80030FF2B23
:10134000A8BFFF23DBB2E8E750500020F85400208C
:101350003A4B0020902A00202C4F00209CFE0308CE
:1013600062500020AC5600203D4B0020CDF9030810
:101370006766666684680020A82A0020D82A0020B4
:10138000A5F10A03E72B00F2EA80DFE813F01C085E
:10139000E800E800E800E800E800E800E800E8000D
:1013A000E800E800E800E800E800E800E800E800FD
:1013B000E800E800E800E800E800E800E800EB07E3
:1013C000E800E800E800DA07E800E800E8003A038F
:1013D000E800FA02E800E202E800D702E80070083C
:1013E000E8004A08E8007508E800E800E800D002D4
:1013F0004108E8003708E800E8002E08E800E800A7
:10140000E800E800E800C302E800E800E800E800BF
:10141000FA06E800D806E800B1069906E800E800F8
:10142000E800E800E800E800E8006707E8001607C1
:10143000E800AB07E8004F06E8000B06E800E8000C
:10144000E800E800E5051C06DC05770565053F05B5
:10145000290510050205E800C804AB04E800E8000F
:10146000E800E8009F04E800E8007D04E800E800E8
:10147000E8006C04530442040304E800E800E800B8
:10148000CE03BA03AF03E800E800E800E800E80094
:10149000E800E800E800E800E800E800E800E8000C
:1014A000E800E800E800E505E800E800E800E800FA
:1014B000E800E800E800E800E800E800E800E800EC
:1014C000E8007603E800E800E800E800E800E8004B
:1014D000E800E800E800E800E800E800E800E800CC
:1014E000E800E800E800E800E800E800E800E800BC
:1014F000E800E800E800E800E800E800E800E800AC
:10150000E800E800E800E800E800E800E800E8009B
:10151000E800E800E800E800E800E800E800E8008B
:10152000E800E800E800E800E800E800E800E8007B
:10153000E800E800E800E800E800E800E800E8006B
:10154000E800E800E800E800E800E800E800E8005B
:10155000E800E800E800E800E80069033E03742DB5
:1015600000F09E81772D65D1D8F80030D8F804209E
:101570009A421EBF5A1CC8F800201978B64A08BF04
:1015800000212046FAF798FF4CE6022D00F0FE807D
:1015900000F2EB80012D7FF4F3AE0B680022591CA2
:1015A00021601A7023685A1C22601D702268242151
:1015B000531C23602B461170D0E5BAF80030FF2B86
:1015C000A8BFFF23DBB2A8E617F004F800283FF419
:1015D000A3AE03780A2B00F27481B0F9023087FBC6
:1015E0000312DB17C3EBA2039BB2FF2BA8BFFF23A1
:1015F000DBB292E6442D7FF4C3AE002A3FF412AE74
:10160000964B136001252B46A8E5052D7FF4B8AE57
:101610000B2293492046F9F719F9082291492046EF
:10162000F9F714F9012507228F492046F9F70EF939
:101630002B4693E5F52D01F06A80762DD8F8003021
:1016400000F04181292D00F0888740F24787392D2D
:1016500000F06A87532D40F09887591CD8F8042071
:10166000C8F800101978D21A531E0329DBB20DD81E
:101670004A1ED2B27D4D7E4802EB420205EB420289
:101680000170527811B1934201F07C814FF0FF3527
:101690002B4663E5774B08461968F9F707F9764B4F
:1016A00020461968F9F702F9744B1968204601259C
:1016B000F9F7FCF82B4651E5DFF8E091704F09F19E
:1016C0000E064FF00A081DE0B8F1500F32D0B8F105
:1016D000320F31D0A8F13C00C0B213282FD9002519
:1016E000294623685A1C2260204683F80080F9F7B7
:1016F000F5F829462046F9F7F1F8B1453FF492ADE7
:1017000019F8018BB8F10A0FDED15E4B9D6819689C
:1017100005EB85054FF6FF736D009D42A8BF1D4682
:101720009942A8BF194625EAE57521EAE171ADB2F3
:1017300089B2D6E7544BE9E797E82200E8E716F0CC
:1017400049FF0028CBD003780A2BC8D8B0F9043061
:10175000B0F9061003EB830383F3500521EAE1712E
:10176000ADB289B2BDE7494B9FE70B680222591C15
:1017700021601A70236801255A1922601D702268A1
:101780000021531923602B461170E7E404224049DD
:1017900020460125F9F75AF82B46DFE4344B21683F
:1017A0001A78481C20600A70002A3FF43BAD013AC9
:1017B000D2B202EB420206EB42025278002A3FF418
:1017C00031AD0132D5180133226813F8011F501CC6
:1017D0009D4220601170F7D124E50B6800215A1C4E
:1017E0002260197022680125531923602B4611705D
:1017F000B4E4284920462A46F9F728F80021204673
:10180000F9F76CF82268002151E50A68224B01259E
:10181000511C21601570226805215019206011703B
:1018200022680A2150192060117022680021501985
:101830002060117022681978501920601170226898
:1018400059785019206011702268997853192360D3
:101850002B46117082E400BFB9BE00089DC100088C
:10186000502804085C280408682804089CFE030823
:1018700058AE0020107AFF1F147AFF1F187AFF1F3E
:10188000A02A0020542A0020942A0020583D00203D
:101890004028040848280408F73B0020BDF9030845
:1018A000D8F80030D8F804209A421EBF5A1CC8F855
:1018B00000201978A54A08BF00212046FAF7FCFD50
:1018C000B0E4002394E65A1CC8F800201B78002BD3
:1018D00000F08787102B07BF9D4A92E82200002561
:1018E00029462268501C206013702046F8F7DEFF5E
:1018F00029462046F8F7DAFF964B20461968F8F794
:10190000D5FF20460021F8F7E9FF00212046F8F72F
:10191000E5FF77E7236800255A1C22602946204608
:101920001D70F8F7C3FF29462046F8F7BFFF0021D6
:1019300020460125F8F7BAFF2B460FE4864D05F146
:10194000800655F8041F2046F8F7B0FFAE42F8D1E4
:1019500068E4824D05F14006B5F880102046F8F79E
:10196000BDFF236895F88220591C21601A702368F6
:1019700095F883200435591CAE4221601A70EBD1D2
:1019800050E4774D23682A7A591C21601A70A98B7C
:101990002046F8F7A3FF298B2046F8F79FFF698BB5
:1019A0002046F8F79BFF2368EA7C591C21601A70D7
:1019B000E98C2046F8F792FF298D2046F8F78EFF34
:1019C0002368AA7F591C21601A70236895F820208B
:1019D000591C21601A70A98C2046F8F77FFF2368F4
:1019E000EA7A591C21601A70E9682046F8F75EFF10
:1019F00023682A7C591C21601A70226895F82110EE
:101A000055E4584B2268197851E4574B03F170059F
:101A100022681978501C2060117022685978501C77
:101A20002060117022689978501C20601170226823
:101A3000D978501C2060117022681979501C2060E0
:101A4000117022685979501C2060117022689979B0
:101A50000733501C9D4220601170D9D1FFF7E2BBC3
:101A6000424D2046A989F8F739FF698920460125AA
:101A7000F8F734FF2B46FFF771BB2368DFF810C17E
:101A8000591C9CF8002021601A709CF80030002B33
:101A90003FF4C8AB364E374D3748384900232268EB
:101AA00016F8017F02F1010EC4F800E017702268F9
:101AB00015F8017F02F1010EC4F800E017702268EA
:101AC00010F8017F02F1010EC4F800E017702268DF
:101AD00011F8017F02F1010EC4F800E017709CF8C4
:101AE000002001339342DADBFFF79CBB244B2549EE
:101AF000B3F9003081FB0321DB17C3EBA101FFF732
:101B000027BB2268204B501C197820601170226876
:101B10005978501C2060117022689978501C206000
:101B200011702268D978FFF7C2BB184D2046A98AE8
:101B3000F8F7D4FEE98A2046F8F7D0FE298B204634
:101B40000125F8F7CBFE2B46FFF708BB75C100084F
:101B5000801F0020E02200203C5800204058002038
:101B60000C750020C4680020585D00209468002097
:101B7000074D0020174D0020374D0020274D002035
:101B8000AC68002067666666EC4C00203070002070
:101B9000054D0020DFF870E30027FEB271460023F8
:101BA0002268501C206016702268501C2060137040
:101BB000226811F8010F0133551C062B25601070A7
:101BC000EED10137062F0EF1060EE6D1B349002300
:101BD0002268501C206017702268501C206013700F
:101BE000226811F8010F0133551C0B2B2560107072
:101BF000EED12368AA49581C072220601A70236876
:101C00000022581C20601A70226891F8F010FFF72B
:101C10004EBB2368A34AA4491078A44A5D1C2560E2
:101C2000187023689278581C20601A70226889788E
:101C3000FFF73DBB22689E4B9E491878551C2560D6
:101C4000107022685878551C2560107022689B78A7
:101C5000501C20601370C98820460125F8F73EFE0D
:101C60002B46FFF77BBA934D20462988F8F736FEBE
:101C700069882046F8F732FEA98820460125F8F742
:101C80002DFE2B46FFF76ABA8B4D05F16006A98839
:101C90002046F8F723FEE9882046F8F71FFE298939
:101CA0002046F8F71BFE2368AA7A591C21601A7097
:101CB0002368EA7A591C21601A7055F80C1B2046DB
:101CC000F8F7F4FDAE42E2D1FFF7ACBA7B495223FC
:101CD0002268501C2060137011F8013F002BF7D1CF
:101CE000FFF7A0BA764800232268056803EB43019A
:101CF000561C6D5C26601570026825680A446E1CCF
:101D0000527826602A70026825680A440133927866
:101D1000691C0A2B21602A70E6D1FFF783BA694D4E
:101D200023682A68591C127821601A702B6822686F
:101D30009978531C2360002311702A6821681A4483
:101D400001335279481C032B20600A70F5D12368B7
:101D50002A68591C127A21601A7023682A68591C53
:101D6000D27821601A7023682A68591C1279216080
:101D70001A702B6820465989F8F7B0FD23682A6845
:101D8000591C527A21601A702B6822685978FFF723
:101D90008EBA4D4B20461968F8F788FD4B4B20460C
:101DA00019880125F8F79AFD2B46FFF7D7B9484D5A
:101DB00020462988F8F792FD69882046F8F78EFDBD
:101DC000B5F904304349DA1781FB0313C2EBA303CF
:101DD00099B220460125F8F781FD2B46FFF7BEB9E1
:101DE0003D4B20461988F8F779FD3C4B2046198871
:101DF000F8F774FD3A4B21681A7801254B1C02F064
:101E0000010223602B460A70FFF7A8B9354B226800
:101E10001B78354D511C03F00203216013702368B9
:101E20002A78591C21601A7069682046F8F73EFD2F
:101E3000A9682046F8F73AFDA9892046F8F74EFD33
:101E4000698A2046F8F74AFDA98A20460125F8F755
:101E500045FD2B46FFF782B9244E3378002B3FF423
:101E6000E1A9234F002537F8021F2046F8F736FD79
:101E7000337801359D42F6DBFFF7D4B91D4D1E4E78
:101E8000DFF88880DFF88890DFED1C8ADFED1C9A90
:101E90009FED1C9A05F1200745E000BF2359002063
:101EA00040580020F8B90020AC6800209468002059
:101EB0008C680020946400202C6500208CF90308B5
:101EC0001457002018570020B8560020BC56002098
:101ED000C056002067666666084C00200A4C002049
:101EE000BC4B002091560020945600203CC300209B
:101EF00086A50020846600203C6E00200000404241
:101F00000040744400E08244FF58002058700020D4
:101F1000D486002020460435F8F7E0FCBD4206F1E7
:101F200018063FF47FA9717C0029F3D095ED008A53
:101F3000B0EE480A2BF0C6FA98F80030002B40F0BB
:101F4000558481B2E6E71022B14920460125F8F711
:101F50007DFC2B46FFF702B90023DFF8F892DFF88B
:101F6000F8B20393029304930593984601214FF628
:101F7000FF7A07E008F10108B8F10B0F00F02C839D
:101F800019F9011F4E1CF5D04AFA08F3D807F1D50C
:101F9000BBF8003043FA08F3DA07EBD504A8F9F7E9
:101FA0002FF8E7E723689B4A9B49D0789B4A5D1C42
:101FB0002560187023681278581C20601A702268F7
:101FC000C978FFF774B9964E338AB3F5007F06F1EE
:101FD000340594BF01270427403655F8041B91FBB4
:101FE000F7F1204689B2F8F779FCAE42F5D18D4D74
:101FF0008D4F05F10C06B5EC010AD7ED087A80EE9D
:10200000270A2BF05FFA81B22046F8F767FCAE4250
:10201000F1D1864D05F10C0655F8041B204689B216
:10202000F8F75CFCAE42F7D1FFF7FCB80021204680
:10203000F8F754FC00212046F8F750FC0021204618
:10204000F8F74CFC22687A4D0023511C2160137074
:1020500022682968501C91F82F10206011702268A6
:102060002968501C91F83A10206011702268296884
:10207000501C91F83B10206011702268511C2160A7
:1020800013702268511C216013702268511C21605A
:1020900013702B682046D98FF8F720FC2B68204658
:1020A000998FF8F71BFC23682A68591C92F8312095
:1020B00021601A702B68226893F83210FFF7F7B886
:1020C00022685C4B0125511C2160157022689978AB
:1020D0005019206011702268197850192060117011
:1020E00022685978531923602B461170FFF736B8D0
:1020F0002368514D01269A1922601E7019F02EFE98
:10210000002840F0B7834D4B2268511C21601070AD
:10211000226841F2B410511C185C216041F2781120
:10212000107059582046890AF8F7C0FBE96B204621
:1021300049080125F8F7BAFB2B46FFF70FB8404EC8
:102140003378002B3FF46EA83E4F0025B846236835
:1021500017F81520591C21601A7098F8011001EB2E
:10216000810101EB810101F2EE2189B22046F8F7ED
:10217000B5FB337801359D4208F10208E7DBFFF734
:1021800051B82368304D591C2A7821601A70236891
:102190006A78591C21601A7069882046F8F79EFBFE
:1021A00023682A79591C21601A70E9882046F8F7BB
:1021B00095FB2268297AFFF77AB8244EF378002B32
:1021C00000F0038323680822591C21601A702368D9
:1021D0000122991821601A7023681D4D591C2A7913
:1021E00021601A702368AA78591C21601A70298806
:1021F0002046F8F773FB698A2046F8F76FFB2368DF
:10220000F279591C21601A702268E978FFF74FB8FB
:102210007466002094680020AC680020A468002048
:10222000C856002034C200200CBA002024C300206D
:10223000145700204D760020D4A300204C8F00209E
:102240003CC3002068540020AC640020F8B9002092
:1022500030700020DCF903081057002012F0CCFA8F
:10226000FF28064600F00D8306A9002501F8125D3F
:102270000DF105008DF8055012F09EFA06A800F841
:10228000115D12F08DFA06A800F8105D12F07CFACC
:1022900006A820F8085D12F06BFA23685A1C226029
:1022A0001E7023689DF80520591C21601A70236850
:1022B0009DF80620591C21601A7023689DF807209C
:1022C000591C21601A7023689DF80820591C216050
:1022D0001A70BDF8101020460125F8F7FFFA2B46BA
:1022E000FEF73CBFAD4D23686A79AD4E591C2160A5
:1022F0001A7033682046198CF8F7F0FA33682046D4
:10230000598CF8F7EBFA69892046F8F7E7FAA989BA
:102310002046F8F7E3FA33682046998CF8F7DEFA9E
:1023200033682046D98CF8F7D9FAE9892046F8F7BE
:10233000D5FA298A20460125F8F7D0FA2B46FEF770
:102340000DBF984D20462988F8F7C8FAA98820467D
:10235000F8F7C4FA298920460125F8F7BFFA2B4679
:10236000FEF7FCBE904D914F05F1500600212878F4
:102370008F4A0B4607E00133242B02F10C0200F0D8
:102380008D8012F80C1C8842F5D103EB43032268C0
:1023900007EB8303511C93F86430216013702368AA
:1023A0006A78591C21601A702368AA78591C216028
:1023B0001A702368EA780435591CAE4221601A70FD
:1023C000D4D1FEF72FBF7B482AF028F800287EF7EB
:1023D00029AF784B1D18226813F8011B501C9D4231
:1023E00020601170F7D1FEF71DBF08227249204608
:1023F0000125F8F72BFA2B46FEF7B0BE22686F4B8B
:10240000501C99782060117022685978FEF74FBFF0
:1024100022680121531823600D460B461170FEF708
:102420009DBE674B03F15A0522685979501C206004
:10243000117022681978501C206011702268597838
:10244000501C2060117022689978501C2060117017
:102450002268D978501C20601170226819790633DF
:10246000501C9D4220601170DED1FEF7DBBE524B46
:102470002268597DFEF71BBF524D534E05F13007C0
:1024800095F902100023F2568A420AD00C33482BE9
:10249000F9D10835BD42F3D1FEF7C4BE00231B7A43
:1024A000FFDE23685A1C2260197029882046F8F73D
:1024B00015FA2368EA78591C21601A7023682A7972
:1024C000591C21601A702368AA79591C21601A705E
:1024D00023686A79591C21601A70DAE7212D54D1DA
:1024E0001A46591CC8F80010384D12F8021B6970C2
:1024F000C8F800205A782A70DA1CC8F800209B78A7
:10250000AB704046F8F796F9D8F80030E880591CCF
:102510001A46C8F8001012F8021B2971C8F80020EA
:102520005B786B71FFF7B2B85A1CC8F800201A78B4
:102530000A2A7FF4ABA89A1CC8F80020244A5978CC
:102540001170D91CC8F8001099785170191DC8F87D
:102550000010DB789370FFF799B85A1CC8F8002078
:102560001B780A2B00F09581502B7FF48FA84046F2
:10257000F8F760F9174E30804046F8F75BF94FF0F6
:10258000FF3570802B46FEF7E9BD28464146FBF734
:102590000FF8054603B2FEF7E1BD00BFF8B9002011
:1025A00014570020F0380020C86800208CF9030878
:1025B000F4F90308EDC200200C750020B868002073
:1025C0008C3A0020C4B90020C4740020AC5600200E
:1025D000F73B0020902A0020DFF8A4A34FF000086A
:1025E0004FF0080908F10108B8F1240F1BD0C8F119
:1025F000200209FA02F22AFA08F6A8F1200316438B
:1026000029FA03F31E4306F0010200231343E9D025
:102610005FFA88F028F04CFF0028E3D0414604A878
:10262000F8F7EEFCDEE7C34B1B78DB0700F13681E1
:102630000026C14FB04602E00136242E0ED03146AE
:102640003846F8F7EDFC0028F6D0314604A8F8F734
:10265000E7FC002856D108F10108EDE7B74BB84E6A
:10266000B3F850102046F8F739F9B64B19882046D0
:1026700089B2F8F733F9B44B1A68530103F020011B
:10268000C2F340030B43C2F3800143EA4103C2F3A8
:10269000C00143EA8103C2F3401143EAC10102F0E1
:1026A000100211432046F8F719F902A90422204626
:1026B000F8F7CCF823683178A44A581C20601970C8
:1026C00011886429A8BF64212046F8F707F9962DE0
:1026D00000F0E98000212046F8F700F92168B8F100
:1026E000190348BFA8F11203A3F3C4034A1C2260D4
:1026F00020460B701A4603A90125F8F7A7F82B46C8
:10270000FEF72CBD414602A8F8F77AFCA3E7D8F8FB
:102710000030D8F804209A4240F0D780864BFF2240
:102720001A724FF000088A4D0CF0D4F8414630225E
:10273000884885F800802CF0D0FF8DF810809DF837
:1027400010300B2B00F24781834F824E42469DF89A
:10275000103003EB430307EBC3035B7CE3B19DF84D
:10276000103003EB430307EBC3035B69A3B19DF890
:10277000103003EB430307EBC3032021586946F8ED
:102780002200F7F7D7F82B7856F82300F7F7DCFA92
:102790002A780132D2B22A709DF810300133DBB2B0
:1027A0008DF810309DF810300B2BD0D92368591CB0
:1027B00021601A70B9F1000F3EF434AD674BC9F8CF
:1027C000003001252B46FEF7C9BC2368B178644A66
:1027D000581C2060197023681278591C21601A70E7
:1027E000FAE4604A92E82200FFF77BB8D9F800309B
:1027F00013F48053B4EEE88A60D0F1EE10FAC0F220
:10280000E180B4EEC98AF1EE10FA0DD8DFED567A08
:102810009FED567A77EEC87AB4EEC78AF1EE10FAD9
:10282000B0EE678A00F2CE80F7EE007A78EE677A33
:10283000B6EE007AF0EE696AE7EE876A40F2E932B6
:10284000FDEEE67A17EE901AB1F5FA6FA8BF4FF4D5
:10285000FA619142B8BF114689B2002B3FF45AABDE
:10286000B5EE408AF1EE10FA40F2DC5308BF19468B
:10287000FFF750BB95F824203D4B002A50D130463D
:1028800042E422680125531923602B461070FEF79D
:1028900065BC4046F7F7CEFF364E6CE6049B43F02E
:1028A00001030493C4E623680322591C21601A70B3
:1028B00023687278591C21601A700FE7F1EE10FA44
:1028C000B2DA4FF47A71FFF725BB5A1C1946C8F8E3
:1028D0000020194811F8022B0272C8F800105B782A
:1028E0004372042A03D9FF2A7EF48CAF19E72249E8
:1028F0000978994205D8022A7EF484AFFF2B7EF432
:1029000081AF236801255A1922601D70B9F1000FAB
:102910003EF488AC194BC9F800302B46FEF71EBCBC
:102920005978022951D003290CBF04203046FFF703
:10293000EBBB00BF20660020042000206C090020B3
:10294000E8C2002004C40020B06900207A390020C9
:10295000835B0020345B00203C6E0020B1E2020863
:1029600088680020004C002000C0884400C08244D9
:102970004C8F0020846800201A4F0020A9C1000855
:1029800090E33FF4821C00211160516011726BB121
:102990000133D8F800101844531E0131C8F8001054
:1029A00011F8012C03F8012F9842F6D10B4B1B783C
:1029B000002B3EF46BAE4FF0FF3526F01FFD2B468B
:1029C000FEF7CCBB4FF47A714AE7042A34BF0220E9
:1029D0000320FFF799BB4246E8E600BF28390020F4
:1029E0002DE9F04F2DED028B91B005461AF00CF950
:1029F000814B1F7827B111B0BDEC028BBDE8F08F81
:102A00007E4B1A685205F6D57D4A1278002A40F0AE
:102A100098817C4B1B78002B6DD07B4C7B4AD4F883
:102A20001C31EB1A934201F26C8494F82471A7BB19
:102A3000DFF80C82D8F80000F6F7BCFDC0B2012820
:102A40000ED9022841F09686714B1A78002A42F07E
:102A50007580D4F82821AA1AB2F57A6F82F02A81FB
:102A6000D4F82C31002B46D094F82431C3B9694BEB
:102A70001B689B7801211E3B00228B4284F82411A5
:102A800084F8382142F2BF80D8F8000002210430D7
:102A900019F096FF94F8303110E0D4F82C3153B38C
:102AA000D4F8343140F6B732EB1A934223D994F874
:102AB0003031002B01F08085DFF88481013BDBB2EF
:102AC00084F83031002B01F05485D4F82C7194F83F
:102AD000382117F8011B94F83931D8F80000C4F8F0
:102AE0002C710A44013384F8382184F83931F6F71F
:102AF00065FDC4F8345119F05FFB474B1B786BB18F
:102B0000DFF84091D9F8003043B1444B3E4C1B688C
:102B1000D4F83C219A1A632A00F2F681404C2378BB
:102B2000022B01F03685DFF8208198F80030032B66
:102B300001F00B853B4B1B7873B13B4F3B685BB19E
:102B4000314CF6F74DFBD4F84431019044F61F6246
:102B5000C31A934200F2BA82344B1B78002B75D112
:102B6000334B1B7843B1284CD4F8943203F5C3336C
:102B7000A0339D4281F086832E4B1B78002B3FF4BF
:102B80003AAF214E2C4C2D4D06F2B5272068F6F7B2
:102B900011FD00283FF42FAF2068F6F703FD2B78D6
:102BA00080465A1E33B120682A70F6F703FD0028CC
:102BB000F2D120E703223946781E2CF074FD96F8F6
:102BC000B43296F8B52286F8B78283F47F4383F057
:102BD000FF039B1A1FFA88F89BB2B8EB132FD5D1CD
:102BE00096F8B622DBB29A42D0D1781E15F06CFD71
:102BF0002B7818442870C9E7CCC20020D486002066
:102C00007857002082570020102000203F0D03003D
:102C100029000020205700208C570020F8C50020F4
:102C2000F85A002094570020985700202C58002074
:102C30003A5800209E570020A4570020A857002093
:102C40001C57002008550020890E00209D4C22783A
:102C5000002A41F00E839C4CD4F88C3203F5C33328
:102C6000A0339D42FFF47CAF984A94F89032C4F8A8
:102C70008C52D75CFA0701F1E585BB0701F1A0850D
:102C8000780701F12C863A074FD5914BDFF86C821B
:102C9000099310AA1146A3F1210241F8202D00202A
:102CA000A3F124020E4603F8240C02910223112101
:102CB000517093703046D8F80410F7F7D1FD3046C4
:102CC000D8F80810F7F7CCFDB8F81230814903EBBB
:102CD000C3039B00053381FB0321DB17C3EBA10179
:102CE000304689B2F7F7D4FDB8F8143003EB83030C
:102CF000590089B23046F7F7CBFD774B029E1B781F
:102D00009B0743BFB8F80C1001F57A7189B24FF4F4
:102D10007A713046F7F7BCFD089B98F80020591CE3
:102D2000089130461A7019F02DFF6C4A94F89032D1
:102D30001178013393FBF1F201FB123384F89032E6
:102D40000EE7614C664BD4F8102119688A1A7C2A68
:102D50007FF65FAE94F81421DFF8A4919FED618AAD
:102D6000C4F81011013284F81421A9F1340A4FF08B
:102D70002408404619F09CFEBAF81030F9EC016ABC
:102D800007EE103AF8EEE66AB8EEC77A08F10108E5
:102D9000C6EE877A5FFA88F867EE887AFDEEE77A02
:102DA000CDED017ABDF904B05FFA8BF019F056FE53
:102DB000CBF3072019F052FEB8F1270FD9D13020FC
:102DC00019F076FE484ADFF83C91D2F800805FFAAD
:102DD00088F019F043FEC8F3072019F03FFED9F838
:102DE00000005E21F6F7EAFB94F8142193072DD139
:102DF000D4F8101141F28832914201F22C8714204C
:102E000019F056FE394A3349B2F9042081FB0231E8
:102E10004FEAE278C8EBA1080FFA88F85FFA88F069
:102E200019F01CFEC8F3072019F018FE1C2019F039
:102E30003FFE002019F012FE002019F00FFE5E2167
:102E4000D9F80000F6F7BAFB94F8142112F007083D
:102E500001F0A685282A7FF4DCAD214B4FF0000855
:102E600017201F6884F8148119F022FE404619F0DB
:102E7000F5FD1F4B1F4CA3FB07239B0BA4FB031269
:102E80005209C2EB0212A3EB8203D8B219F0E6FD9D
:102E9000182019F00DFE184BA3FB07239B09A4FB78
:102EA00003125209C2EB0212A3EB8203D8B219F04B
:102EB000D5FD404619F0D2FDD9F800005E21F6F7A5
:102EC0007DFBA6E57057002010200020345800201C
:102ED0004C570020676666669156002039580020DE
:102EE000F8C5002000007A44BC560020C0560020DF
:102EF00073B2E74589888888D34D621094560020C4
:102F0000FC56002024570020DFF8B08101934120B7
:102F100019F03CF9644FB8F90220DFF8A4B187FB3F
:102F20000230D217C2EBA00080B219F019F9B8F93B
:102F3000002087FB0230D217C2EBA00080B219F04C
:102F40000FF9B8F9042087FB0230D217C2EBA000BA
:102F500080B219F005F99BF80010D9F80000F6F7D7
:102F60002DFB94F84071019B17F0010801F07D835F
:102F7000DFF844A1DAF80020910640F185804B4A41
:102F8000DFF840811278920741F13A8698F80020E4
:102F9000042A8CBF032702274720029319F0F6F872
:102FA000D8F8040019F0B4F8D8F8080019F0B0F80F
:102FB000B8F812203E49D9F80000A1FB0232C2F352
:102FC000471211460192F6F7F9FA9BF80000DAF879
:102FD0000010019A029B424011F0140F8BF8002060
:102FE00041F0A885B8F80C20642000FB02F00193A2
:102FF00019F08EF898F80020D9F8000047EA820707
:10300000FFB23946F6F7DAFA9BF80020D9F800004B
:10301000574039468BF80070F6F7D0FA94F84071B3
:10302000019B8FBBDFF8A08001934F2019F0AEF811
:10303000D8F8000019F06CF8D8F8040019F068F816
:10304000384619F065F80121D9F80000F6F7B6FA0C
:1030500016499BF800200F78D9F8000007F0010707
:10306000394682F001028BF80020F6F7A7FA9BF8A8
:103070000020D9F80000574039468BF80070F6F769
:103080009DFA94F84071019B0A4AC4F83C317B1CBC
:10309000DBB2A2FB0312D20802EB8202A3EB4203D3
:1030A00084F840313AE500BF6766666691560020B5
:1030B0001F85EB51CDCCCCCCB0690020C056002090
:1030C0000C55002094560020004C002094F84A3102
:1030D000002B41F03383E84B1B6803F00802002A01
:1030E00048F603414AF60B404BF60F4249F60748B3
:1030F00004BF0246884613F0040F4FF0190118BFB1
:1031000090469B0684F84A1103D548F4804848F05D
:103110002008DA4B1A79C8F3090B002A41F0FE8522
:103120005B79002B41F08C87994664204FF0FF3388
:103130004FF0000ACDF82080CDF82480CDF828B0DB
:10314000ADF82E90ADF830308DF83E00ADF82CA0E3
:10315000CDF832A0CDF836A0CDF83AA00DF1200E72
:10316000BEE80F00DFF824C384F805A0ACE80F0028
:103170009EE80F00ACE807002CF8023B61464FF0D8
:1031800001081B0C4FF0FE0E1F20C82201F81E394B
:1031900084F802E0A27184F80780E07094F85A0184
:1031A000207180F0F10383EA0313DAB2130983F08C
:1031B000E70343EA022383EAC2031BB283EA031252
:1031C000D2B2C3F3072383EA121343EA022383EA4A
:1031D000C2031BB283F0C80282EA0212D2B2C3F366
:1031E000072383EA121343EA022383EAC2031BB2D2
:1031F00083EA080E8EEA0E1E5FFA8EFEC3F30722E4
:1032000082EA1E1242EA0E2200EB080382EACE0E88
:103210000CEB080084F85A31A4F800E011F8013BE7
:1032200083EA0E0383EA0313DBB21A0982EA1E2241
:1032300042EA032282EAC3031BB21FFA83FE8142E1
:10324000A4F800E0EAD183F07C0383EA0313DBB245
:103250004FEA131C8CEA1E2C8CEA032C8CEAC30C5C
:103260000FFA8CFC1FFA8CFADFF82492A4F800A065
:103270005FFA8CFC4FEA1A2A84F828A084F827C049
:1032800009F5C17B04F12208D9F80000D9F804102F
:10329000D9F80820D9F80C30DE46AEE80F0009F165
:1032A0001009C145F346EFD1D9F80000CEF800006F
:1032B000DFF8E08199F804308EF8043008F127092E
:1032C00084F8A9C184F8AAA118F8011F3868F6F794
:1032D00075F9C145F8D194F84B21002A41F0788165
:1032E0006749684B08781B680A2184F84B1100284D
:1032F00001F05182DFF8A0C10128BCF80010039151
:1033000041F296860228BCF8029001F04B85BCF889
:1033100004100291032801F0A3860428BCF806B02B
:1033200001F099860528BCF808E001F0908606288F
:10333000BCF80A8001F066860728BCF80C1001D0A2
:10334000BCF80E2094F85A010893064686F0300324
:1033500083EA0313DBB24FEA131C4B4804968CF04C
:103360007A0C4CEA032C008826718CEAC303DFF840
:103370002CC1C0EB00208CFB00AC8444C0171BB2F6
:10338000C0EB6C200646C3F3072C83EA0310039BB3
:103390008DF83560C0B24FF0000A63F30F0A8CEA73
:1033A000101303934FF0000C029B69F31F4A6EF356
:1033B0000F0C4FF000094FF0000E63F30F0961F39B
:1033C0000F0E039BCDF824A068F31F4C62F31F4E31
:1033D0004FF000086BF31F49CDF82890CDF82CC0B2
:1033E000CDF830E08DF8348043EA00230DF1200958
:1033F00083EAC00EB9E80F000FFA8EFE8EF0C80AFD
:103400008AEA0A1ADFF884C084F805805FFA8AFA2B
:10341000CEF3072EACE80F008EEA1A1E4EEA0A23FE
:1034200099E8030083EACA031BB283F0230E4CF829
:10343000040B8EEA0E1E5FFA8EFEC3F3072282EAA9
:103440001E12049B604642EA0E2203F1010882EA42
:10345000CE0E20F814194FF02309FE211622C8239E
:1034600084F85A81A4F800E084F807900CF1020C6B
:10347000A170E27014E000BFB0690020AC560020DB
:103480003CC30020F8C500203A4B00201820002043
:10349000122000209321002088A50020030820800E
:1034A000A37110F8013B83EA0E0383EA0313DBB236
:1034B0001A0982EA1E2242EA032282EAC3031BB2ED
:1034C0001FFA83FE6045A4F800E0EAD183F0F4031C
:1034D00083EA0313DBB21A0982EA1E2282EA03227C
:1034E00082EAC3031BB21FFA83FEDFF80C84A4F840
:1034F00000E05FFA83FC4FEA1E2A84F81EC084F8BD
:103500001FA0D8F80410D8F80820D8F80000D8F880
:103510000C3008F5C17EAEE80F00D8F81000D8F8DE
:103520001410D8F8182004F2A119AEE8070004F22C
:10353000831884F8A1A184F8A0C118F8011F386885
:10354000F6F73CF8C145F8D194F84E31002B41F024
:10355000FA80DFF8B0A3DAF800301922980684F870
:103560004E2140F12083E34BDFF89C831B789907C1
:1035700041F1D08398F80030042B8CBF4FF0030941
:103580004FF00209F5F72CFEB8F81430B8F80C200B
:10359000089003EB83035B00ADF83A304FF47A7088
:1035A000D8F804300A93B8F8121098F800E0D8F868
:1035B00008308DF83C9000FB02F24FF0000C4FF009
:1035C000FF3008AE8DF83DE0CDF824C00C920B938F
:1035D000ADF838100D90B146B9E80F00DFF82CE3D4
:1035E0000296AEE80F0099E80F00AEE807007246B9
:1035F000182122F81C39E17194F85A1184F805C099
:1036000081F0780383EA0313D8B2030983F0F60349
:1036100043EA002383EAC0031BB283EA0310C0B26B
:10362000C3F3072383EA101343EA002383EAC003AA
:103630001BB283F0C80080EA001C5FFA8CFCC3F365
:10364000072080EA1C1040EA0C2080EACC0000B27F
:1036500080F0180383EA0313DBB2C0F3072080EA8B
:10366000131040EA032080EAC30301F101091E2080
:103670004FF0FE0C4FF0C80BE0700EF1020E2171FE
:1036800084F85A91238084F802C084F806B0184662
:1036900012F8011B414081EA0111C9B20B0983EA0A
:1036A000102343EA012383EAC10109B288B27245BB
:1036B0002080EDD181F0180181EA0111C9B20A0917
:1036C00082EA102383EA012383EAC1031BB29AB280
:1036D00089492280DBB2120A039104921E4684F8C3
:1036E000272084F826308E4601F5C17B04F122099B
:1036F000DEF80000DEF80410DEF80820DEF80C30FA
:10370000DC46ACE80F000EF1100ECE45E346EFD1DB
:10371000DEF80000CCF80000DFF8F4919DF81030DE
:1037200084F8A86184F8A931CB461BF8011F3868DA
:10373000F5F744FF714B5B45F7D1F5F751FDDAF82A
:103740000030B8F80C20D8F804A0D8F808804FF45E
:103750007A7113F0140F01FB02F141F05D828E4685
:1037600094F85AB108908BF06A00654BDFF8A4C159
:10377000B3F90420CDF824A080EA0010C0B20309F8
:1037800083F0D50343EA002383EAC0031BB283EA34
:103790000310C0B2C3F3072383EA101343EA0023E4
:1037A00083EAC0031BB28CFB020CD2174FF0000A55
:1037B000CDF82880C2EBAC02DDF80880CDF830E00F
:1037C00083F0C80C0B91ADF83A20ADF834A0ADF8F9
:1037D00036A0ADF838A08CEA0C1C5FFA8CFCC3F361
:1037E000072EB8E80F008EEA1C1E4EEA0C2E8EEA59
:1037F000CC0CDFF818E184F804B00FFA8CFCAEE8CA
:103800000F008CF0210398E8070083EA0313DBB272
:10381000CCF3072C8CEA131C4CEA03280BF1010CA7
:103820008EE8070088EAC30384F85AC14FF0210BE1
:103830004FF0FE084FF01C0CC8220EF10C0E84F85D
:1038400005A084F807B084F8028084F803C0AEF1C4
:103850001C01A2711846238011F8012B424082EA14
:103860000212D2B2130983EA102343EA022383EA45
:10387000C20212B290B271452080EDD182F068028E
:1038800082EA0212D2B24FEA121B8BEA102B8BEAA9
:10389000022B8BEAC20B0FFA8BFB1FFA8BF3DFF8BC
:1038A00058E023805FFA8BFB1B0A1E4684F8253004
:1038B00084F824B00EF5C17A04F12208DEF8000085
:1038C000DEF80410DEF80820DEF80C30D446ACE850
:1038D0000F000EF1100EC645E246EFD1BEF80030E3
:1038E000DFF83480ACF80030CA4684F8A6B184F81A
:1038F000A76113E09156002012200020B92100207A
:10390000C0560020B06900209456002018200020E6
:103910009321002067666666B72100201AF8011F10
:103920003868F5F74BFED045F8D194F85AA1E14A32
:10393000E14E84F804A08AF0EB0383EA0313D9B2C2
:103940000B0983F0C50343EA012383EAC1031BB2D9
:1039500083EA0310C0B2C3F3072181EA101141EAE0
:10396000002181EAC0010CCA09B281F0C80E8EEABA
:103970000E1E5FFA8EFE4FF0000C0892C1F3072175
:10398000029A0993CDF828C081EA1E1343EA0E2358
:1039900007CA83EACE031BB283F0310E86E8070024
:1039A0008EEA0E1E5FFA8EFEC3F3072383EA1E1310
:1039B00043EA0E2383EACE0394F808E0607AA27A01
:1039C000E17A84F805C01BB28EEA030E8EEA0E1E61
:1039D0005FFA8EFEC3F3072383EA1E1343EA0E2326
:1039E00083EACE031BB2584080EA0010C0B2C3F392
:1039F000072383EA101343EA002383EAC0031BB2C0
:103A00005A4082EA0210C0B2C3F3072282EA1012BF
:103A100042EA002282EAC00212B2514081EA011158
:103A2000C9B2C2F3072383EA111343EA012383EAED
:103A3000C10394F80CC094F80DE0A07BE17B227CDC
:103A400094F811801BB28CEA030C8CEA0C1C5FFA10
:103A50008CFCC3F3072383EA1C1343EA0C2383EA99
:103A6000CC031BB28EEA030E8EEA0E1E5FFA8EFEA8
:103A7000C3F3072383EA1E1343EA0E2383EACE032C
:103A80001BB2584080EA0010C0B2C3F3072383EA98
:103A9000101343EA002383EAC0031BB2594081EAB2
:103AA0000111C9B2C3F3072383EA111343EA0123C7
:103AB00083EAC1031BB25A4082EA0212D2B2C3F3B4
:103AC000072383EA121343EA022383EAC2031BB2E9
:103AD00088EA030888EA08185FFA88F8C3F307231E
:103AE00083EA181343EA082383EAC803A17CE27C33
:103AF0001BB2594081EA0111C9B2C3F3072383EA1B
:103B0000111343EA012383EAC1031BB25A4082EA3C
:103B10000212D2B2C3F3072383EA121343EA022349
:103B200083EAC2031BB283F0270E8EEA0E12D2B2D2
:103B3000C3F3072E8EEA121E4EEA022E8EEAC20E42
:103B40000AF101030FFA8EFE1FFA8EF24FF0310ACE
:103B5000FE200C2184F85A31C8234FEA122C06F5B6
:103B6000BE785FFA8EFE228084F807A0A070E17014
:103B7000A371039E84F814E084F815C07168B268DC
:103B8000F3683068B6F810A0A8E80F0028F803AB77
:103B900084F897C184F896E119F8011F3868F5F7A1
:103BA0000DFDC845F8D194F852C1BCF1000F40F0AA
:103BB0005685424B94F85A91B3F90010B3F902209C
:103BC000B3F904309FED3E6A84F805C007EE103A61
:103BD0003C4B1B68089389F06A0383EA031306EEE3
:103BE000901AD9B20B0983F0D50343EA012383EA83
:103BF000C1031BB283EA03115242C9B207EE902AF5
:103C0000C3F3072383EA111343EA0123F8EEE77AAB
:103C1000F8EEE66AB8EEC77A83EAC1031BB267EE34
:103C2000867A66EE866A27EE067A002083F0C80858
:103C3000CDED0A7ACDED096A8DED0B7A0C900D90E1
:103C40000E9088EA081E0DF1200A5FFA8EFEC3F37B
:103C50000728BAE80F0088EA1E1848EA0E2888EA02
:103C6000CE08DFF854E00FFA88F8AEE80F0088F0CD
:103C70001E0C9AE807008CEA0C1C5FFA8CFCC8F357
:103C8000072383EA1C1343EA0C238EE8070083EA28
:103C9000CC0CC8214FF0050A4FF01E08FE231C2053
:103CA00009F10102A17184F852A184F80780A37080
:103CB000E07009E0004C002018200020C0560020D1
:103CC00088C3E43AF8C50020AEF1100184F80490EE
:103CD0000EF10C0EA4F800C084F85A2111F8013B33
:103CE00083EA0C0383EA0313DBB21A0982EA1C227B
:103CF00042EA032282EAC3031BB21FFA83FC714526
:103D0000A4F800C0EAD183F0270383EA0313DBB2EF
:103D10001A0982EA1C2C8CEA032C8CEAC30C0FFAD9
:103D20008CFC1FFA8CFADFF81094A4F800A05FFA5C
:103D30008CFC4FEA1A2A84F825A084F824C009F5DF
:103D4000C17B04F12208D9F80000D9F80410D9F891
:103D50000820D9F80C30DE46AEE80F0009F1100952
:103D6000C145F346EFD1DFF8E483B9F80030AEF88F
:103D7000003008F1240984F8A6C184F8A7A118F836
:103D8000011F3868F5F71AFCC145F8D194F853A122
:103D9000BAF1000F40F05E84E04B1B68052284F806
:103DA00053219A0640F10185DD4ADFEDDE7A518A22
:103DB00007EE101AB8EEC77A13F0140F27EE277A21
:103DC00001F0E380D84BDFEDD76AD3ED007AF8EE4F
:103DD000E77A67EEA67A94F85A91D44BD44AB3F9AD
:103DE0000410B2F90620DFF868E3D2488DED097AB5
:103DF00089F0220383EA03135FFA83FC4FEA1C1362
:103E000083F0590343EA0C2383EACC03B2F5FA6F3B
:103E10001BB2A8BF4FF4FA6283EA031C5FFA8CFC62
:103E2000B2F57A7FC3F3072383EA1C13B8BF4FF4BC
:103E30007A724FF0640843EA0C23A2F57A7208FB09
:103E400002F283EACC0C8EFB026E80FB01600FFA5B
:103E50008CFCC917D217C2EBAE12C1EBA0034FF016
:103E6000000B08A98CF0C80ECDED0A7AADF832200F
:103E7000ADF83030CDF820B0CDF82CB088468EEAC1
:103E80000E1E5FFA8EFE0291CCF3072CB8E80F00ED
:103E90008CEA1E1C4CEA0E2C8CEACE0EDFF8B4C263
:103EA000D8F8008084F80490ACE80F000FFA8EFE7A
:103EB0008EF04A0383EA0313DBB2CEF3072181EAD3
:103EC0001311624641EA032109F1010981EAC303A2
:103ED000142042F810894FF0FE0E4FF04A080021DE
:103EE00084F85A914FF0C809E07023800CF1040C5B
:103EF00084F8078084F802E0617184F8069018461F
:103F000012F8011B414081EA0111C9B20B0983EA91
:103F1000102343EA012383EAC10109B288B2624552
:103F20002080EDD181F0140181EA0111C9B24FEA7C
:103F3000111E8EEA102E8EEA012E8EEAC10E7E4BE5
:103F40000FFA8EFE1FFA8EFC1E464FEA1C2B5FFAFC
:103F50008EFE84F81DB084F81CE059689A683068B9
:103F6000DB68A4F800C006F5C17CACE80F0030693E
:103F70007169B6F818900396ACE8030004F2831850
:103F8000ACF8009084F89FB1C14684F89EE104F239
:103F90009F1B19F8011F3868F5F710FBCB45F8D1C6
:103FA000664B674A1B781278013B12F00100DBB2C6
:103FB00014BFC0214021172B03D8624A134493F841
:103FC00008A0614B1A8896071ABF002341F0100120
:103FD000012312F4027F18BF022312F0100F18BF42
:103FE000062312F0200F18BF1023002840F0298666
:103FF0004FF0030994F85AE108938EF0460383EAE0
:104000000313DAB2130983F0920343EA022383EA2B
:10401000C2031BB283EA0310C0B2C3F3072282EAD1
:10402000101242EA002282EAC00212B282F0C80CE8
:104030008CEA0C1C5FFA8CFCC2F3072282EA1C1289
:1040400000238DF82790032042EA0C29029A8DF86C
:1040500024A08DF825308DF826108DF8280007CA89
:1040600089EACC0C0FFA8CFCDFF8E890E3718CEA5B
:104070000C1AA9E803005FFA8AFACCF3072C8CEA41
:104080001A1C4CEA0A2181EACA0A94F808C089F885
:1040900000200FFA8AFA8CEA0A0C8CEA0C1C5FFAF0
:1040A0008CFCCAF3072282EA1C1242EA0C22607AD4
:1040B000A17A94F80BA0637182EACC0212B250404C
:1040C00080EA001C5FFA8CFCC2F3072080EA1C1017
:1040D00040EA0C2080EACC0000B2414081EA0111A4
:1040E000C9B2C0F3072282EA111242EA012282EA2F
:1040F000C10212B28AEA020A8AEA0A1A5FFA8AFA44
:10410000C2F3072282EA1A1242EA0A2294F80CC089
:10411000607BA17B84F804E01EE000BFB069002052
:10412000945600200AD7233CB8560020C0560020E1
:1041300088A500206766666612200020C4680020FB
:104140002066002098FB03081057002093210020D0
:10415000D34D62101820002082EACA0212B28CEA03
:10416000020C8CEA0C1C5FFA8CFCC2F3072282EA78
:104170001C1242EA0C2282EACC0212B2504080EABF
:104180000010C0B2C2F3072282EA101242EA0022F3
:1041900082EAC00212B2514081EA0111C9B2C2F3EF
:1041A000072282EA111242EA012282EAC102E17B7D
:1041B00094F810A013B281EA030282EA0212D2B28A
:1041C000C3F3072383EA121343EA022383EAC203F9
:1041D0001BB28AEA030282EA0212D2B2C3F30723B5
:1041E00083EA121343EA022383EAC2031BB283F079
:1041F000320282EA0212D2B2C3F3072383EA121315
:1042000043EA022383EAC2031BB29AB24FF0FE0CC8
:104210000920C8210EF1010EDBB284F802C04FEA7A
:10422000122CE070A17184F85AE1228084F812C047
:104230006374039E30687168B268B6F80CB009F513
:10424000BA7EAEE8070009F5C2798EF802A0AEF892
:1042500000B084F894C184F8933118F8011F3868CD
:10426000F5F7ACF9C145F8D1019BC4F84431FEF72C
:1042700073BCDA4BDA491868F5F768F90023237044
:10428000FEF7E9BC94F89832D64AC4F8945202EB8F
:104290008302126A42B310AD04F29F23D24E45F856
:1042A000203D002104F2B1233180099380211523A0
:1042B000A52784F89E32284684F89D1284F89C72C3
:1042C000904728463188F6F709FB089DC74804F552
:1042D00027716D1A152DA8BF15252A4628F07EFFD7
:1042E000C34A94F898321570C24A013382FB031214
:1042F000A2EBE37202EB42029B1A84F89832FEF7BB
:104300003BBCDFF828E3BC4ABC4BD4F82011DEF8F4
:1043100000001B8892F80BC0B94A401A4FF47A711A
:10432000DFB201FB0CF11B0A9777177588424FF03B
:104330000007D37753759770177180F00C82B14BDB
:10434000B14E1B68B149DFF8E89208688968DFF868
:10435000E4E2DFF8E482DEF800E086FB036CDB17C2
:10436000C3EB6C1303F5FA739BB293761B0AD376F7
:1043700089FB003AC01789FB0139CB17C0EBAA01B2
:1043800011770912DFF8B4C251779F499CF800C039
:10439000C3EBA9030EF5EA4081FB0E1982F8203029
:1043A0004FEAEE711B12C1EB6911303082F82130F7
:1043B000974B98F8009083F81A90001278310EF11C
:1043C000300E1CF0020F82F8230082F8241082F8CD
:1043D00022E000F0BD81D8F804C08E49D8F808A0CA
:1043E000DFF85CB28C4A81FB0C604FEAEC7E81FB0B
:1043F0000A61CEEBA05E4FEAEA70C0EBA1510BFB65
:104400000EC00BFB01AB0BEB4B0B4FEA4B0600EB6B
:1044100040000196400082FB007B01EB810182FBA2
:104420000672019E92140EEB8E0E01EB81014FEA93
:10443000AB4B04920EEB8E07B8F8122005914FEAB1
:10444000E67EC117B8F80C80744E03974FEADC7C07
:1044500083F809C0ABEB010C06FB1C0108F5FA78E8
:10446000049E03981FFA88F70297A6EB0E086B4F7D
:10447000019EDFF8D0E1B9F1050F4FFA8CF909EB95
:104480008009404607FB1868059EDFF8BCC140B2B2
:1044900000EB860002EBC2025B4E4FEA82024FEA5B
:1044A000DA7A8CFB02BC83F80EA086FB017A86FBCD
:1044B00008B74FEAE27B9DF808205A75CBEBAC12A7
:1044C0000192029ABEF80060DFF880E14FEAE878D6
:1044D0004FEAE1711FFA89F980B2C8EB6717C1EBA7
:1044E0006A114FEA1228019A83F80A904FEA102BBA
:1044F0004FEA192C4FEA212A4FEA272983F810B0F6
:10450000BEF800E083F80BC0D873C2F3072C4FEA63
:10451000162034BF4FF0320B4FF0330B197383F872
:104520000DA05F7483F8129083F816809DF8042024
:10453000DA7183F808C0DE74187583F81BB083F84D
:104540001CE0C4F81C51FEF770BA354F3868036898
:104550005B69984700283EF4EDAA3868036801219A
:104560009B6998470222002388F800202370FEF7F9
:10457000E1BA94F8381194F83931D8F800004A1C9F
:10458000013384F8382184F83931F5F717F8FEF74C
:10459000B0BAF4F725FE234B1A6840F6B833801AF8
:1045A000984200F2EE80204F3B793A2B00F0CB820C
:1045B00000232370FEF7BEBAC4F82C3184F82431EE
:1045C000DFF88C8018F030FA94F83031FEF776BAC4
:1045D000013A84F84B21FEF7B7BF00BF30580020E6
:1045E0004C57002098FB0308F45400205851002039
:1045F0006D51002056555555545000205050002004
:10460000AC570020B85600201F85EB51F85400200D
:10461000D85700206BCA5F6B83DE1B4340420F00FC
:104620001C540020005B0020E85A0020F8C5002040
:1046300067666666BC56002094560020915600209E
:10464000806967FF084C0020D34D62100A4C00209F
:104650001C5700200AF1FF3A84F853A104E60CF13C
:10466000FF3C84F852C1FFF791BBB94A1288D705C5
:1046700015D4D00600F1D882910600F19A8357062E
:1046800000F18A84100700F18B84D10700F1AE8419
:1046900012F0020F0CBF4FF004084FF00C08AD49A8
:1046A000AD4A0F78D27807F001070AB147F0020748
:1046B0005320019317F06AFDA84A128802EB820288
:1046C00002EB8202900080B217F04AFD002017F042
:1046D00047FDA34AA3491288D9F80000C2EBC212D1
:1046E000520081FB02311144D217C2EB61225FFA02
:1046F00082FA5146F4F762FF9BF80020D9F80000D7
:104700008AEA020248EA070700218BF80020F4F742
:1047100055FF3946D9F80000F4F750FF9BF8002008
:10472000D9F800007A40D2B211468BF80020F4F795
:1047300045FF94F84071019BFEF773BC013B84F880
:104740004A31FEF7C8BD013B84F84E31FFF72BBA62
:104750002D22DA76F5E6844BDEF800101B78C4F8DB
:104760002011013B012B3FF6EAAD1021022391708D
:104770001371E4E518F048F97C4B01221A70FEF73A
:104780006FB97B4AB2F8423100210133A2F84231BD
:104790002170FEF7CFB901468046864683460290D7
:1047A000814603900246FEF7CDBD9FED727A13F06D
:1047B000140F08BFF0EE477A7FF404ABFFF70BBB92
:1047C0006D4B664909930DF14008A3F1210048F8AB
:1047D000200D4FF0080E4FF000090A2003F822ECDC
:1047E00003F8230C03F8249C40460988F6F750F898
:1047F000624B63491B6881FB0321DB17C3EBA101FB
:10480000404689B2F6F744F85E4BB3F806A00AF0CA
:10481000B5F8089B5A1C089283F80090089B4FEA51
:104820001A22591C08911A70089B5A1C089283F886
:1048300000A0089B5A1C08921870404618F0A2F974
:10484000FEF71EBADFF850919FED4F8AB9F902309A
:10485000494A099207EE903AF8EEE77A0DF14008DE
:1048600067EE887AA2F12403FDEEE77AA2F1210136
:10487000002048F8201D02F8240C0822CDED017A12
:104880005A701E229A70BDF804104046F6F700F8E0
:10489000B9F9003007EE903AF8EEE77A404667EE55
:1048A000887AFDEEE77ACDED017ABDF80410F5F7D0
:1048B000EFFFB9F9043007EE903AF8EEE77A404698
:1048C00067EE887AFDEEE77ACDED017ABDF8041047
:1048D000F5F7DEFF404618F055F9FEF7CEB92B4A42
:1048E000254B12680993A3F12408002103F8241C26
:1048F0002123D10088F8023040F1008224490326A8
:10490000134B1B885A0500F1F681D80700F1F58298
:1049100003F002031F4A002B1CBF03261146DFF8D9
:104920007C903246484628F059FC06EB090310A853
:104930000133A9F1020140F8203D00225B1A06F87C
:10494000092088F8013018F01DF9FEF79CB900BF66
:104950001057002020660020404B002050500020BF
:104960003A4B0020030820803D4B00202900002006
:1049700010200020000000004C570020F8540020B8
:1049800067666666AC56002058A08B41D86600204A
:10499000142A0408242A0408C05600202B5700209B
:1049A000022018F085F8FF2013F014FE0278FF2A89
:1049B00000F0E98290F901004FEAE0785FFA88F8A8
:1049C000C0B218F04BF8404618F048F8032018F031
:1049D0006FF8FF2013F0FEFD0278FF2A00F0CF826F
:1049E000B0F908805FFA88F0C8F30728DFF898A3C9
:1049F00018F034F8404618F031F89AF80420002AEC
:104A000040F0E781D14A1268900640F11081DFF84A
:104A10007CA3DFF87C839AF80020910700F1708274
:104A20004FF0000B012018F043F8384618F016F844
:104A3000584618F013F8092018F03AF8002018F03A
:104A40000DF8002018F00AF8B8F8161098F80030A1
:104A5000B1F5967F0AD994F8142102F00F02072AC3
:104A600004D842F20F738B4228BF0B46DFF824B301
:104A70000193052018F01CF89BF80820019B002AE0
:104A800000F0A482203B07EE903A9FEDB17AF8EE59
:104A9000E77AF6EE006A67EE877ABEEE007AF5EE08
:104AA000C07AF1EE10FA58BFB0EE667A77EE877AE8
:104AB000FDEEE77ACDED017ABDF904300193D8B26D
:104AC00017F0CCFF019BC3F3072017F0C7FF9AF83C
:104AD0000020002306930793930700F16D8194F85B
:104AE0001831012B00F06881BBF90030DFED996AC5
:104AF00007EE103ABBF9023007EE903AB8EEC77AEB
:104B0000F8EEE77A27EE267A67EEA67ABDEEC77A48
:104B1000FDEEE77A08A88DED087ACDED097A17F059
:104B2000D9FF5E21D9F80000F4F748FD94F814216C
:104B3000FEF790B9884A1068FEF759BAC4F82851B0
:104B40001F70FDF78DBFBB78DBB103F1FF3C5FFA4F
:104B50008CFC0CF1010CBC44BE4600221EF8013B4B
:104B6000534083EA0313DBB2120AD90042EA03225C
:104B7000F44581EA131382EA0302EFD1002A7FF49D
:104B800017AD764BDFF810E21968734BD1F830C0DF
:104B90001B68734ADFF8EC81CEF83830714BB8F8F7
:104BA0000080CEF86800B3F8423110689268CEF801
:104BB0001880CEF82800CEF84820CEF85830BCF146
:104BC000000F00F01782DCF80430886C83423BBF92
:104BD000CA681B1A1B1A9B18002B7DF4A4AF0B6824
:104BE000DFF8B8819B690846022198470423F878CA
:104BF00088F8003028F06CF903232370FDF795BF87
:104C00000127FEF7C9B90221D8F80000F4F7BEFC6D
:104C100094F83031FDF752BF4F4B1B6803EB830311
:104C20004FEA430EFEF79CBD4FF0340837E54E4B7C
:104C300093E8030008AB83E80300184617F04AFF27
:104C40006FE74A4AD278002A0CBF4FF004094FF0B0
:104C50000509FFF7CFB9DFF800B1DFF844A1102054
:104C600017F026FFDBF800208AFB0238D217C2EBD0
:104C700068185FFA88F017F0F1FEC8F3072017F004
:104C8000EDFE212017F014FFDBF800108AFB013A3B
:104C9000CA17C2EB6A12642000FB1212002AD8BFA6
:104CA000524212B2D0B217F0D9FE002017F0D6FE51
:104CB000FEF7A5B80122D8F800001A70F4F772FCCC
:104CC0000746D8F80000F4F76DFC7F067DF4C8AE07
:104CD0008A2800F069818E287DF4C2AE94F82431D0
:104CE000002B7DF4DAAE224BC4F82C312D2384F84E
:104CF0003031FDF7BCBE03261E4910E61E4B1F4A8D
:104D00001B681F4903F48003002B16BF11460426BD
:104D10000326F5E54FF00109FEF734BC19495A792D
:104D20000B8803EB830303EB83034FEA83091FFA2A
:104D300089F9002A00F09A81094B1B681BB2029383
:104D400009F01CFE029B40B2FEF7F2B9B0690020E8
:104D5000E4380E3F0050C347B85600201C540020D2
:104D6000F85400201020002098FB0308404B00203E
:104D7000AC570020182A0408D4860020142A0408FE
:104D80000C2A040850500020AC56002091560020F8
:104D90009456002054500020180E0020890E002048
:104DA0001F85EB5111469046964693460292FEF7B8
:104DB000C9BA4FF0240872E40121D8F80420D8F8C9
:104DC000083084F8181106A80692079317F082FE9F
:104DD000A7E6DFF8C0B29BF80020002A3FF412AE2D
:104DE000A449B4F81681088802914FEA08184FF0D8
:104DF000640E1FFA88F80EFB00204FEA420EB0FB4B
:104E0000FEF048EA00281FFA88F8C0F3032048EAB9
:104E100000080620019217F04BFE5FFA88F017F0A9
:104E20001DFE4FEA182017F019FEB4F81601019A7A
:104E3000914B0299013080B290FBF2FC02FB1C0204
:104E4000587AB1F80080A4F81621012800F0E48017
:104E50005A7B6E2303FB08F8152198FBF1F8002A12
:104E600040F0D3803A2017F023FE1FFA88F84FF065
:104E7000640BB8FBFBF291B2C8B20292019117F039
:104E8000EDFD0199080A17F0E9FD3B2017F010FE2F
:104E9000029A0BFB128080B20A22053090FBF2F0DE
:104EA000C0B217F0DBFD002017F0D8FDDFF8E0B14D
:104EB000282017F0FDFD4FF00A08DBF8002092FBD8
:104EC000F8F85FFA88F017F0C9FDC8F3072017F06B
:104ED000C5FD042017F0ECFDBAF80620002A7DD1AC
:104EE000DBF8082082F310085FFA88F017F0B6FDAF
:104EF000C8F3072017F0B2FD84E5604904260EE5EB
:104F0000112017F0D5FDB8F812205D494FF4F36B6E
:104F10000BFB02F281FB0231D217C2EB6132D0B23D
:104F2000019217F09BFD019AC2F3072017F096FD3E
:104F3000192017F0BDFDB8F8122052490BFB02F200
:104F400081FB0230D217C2EB601281FB0230D11715
:104F5000C1EB6011642000FB1120C0B217F07EFD90
:104F6000002017F07BFD9AF80020B8F80CB09207EB
:104F70007FF556AD5FFA8BF74FEA1B2B52E54FF0EA
:104F80000008404632E540461BE5938907EE903A1B
:104F9000F8EE677AFEF71FBF4FF01008FFF77FBBF0
:104FA0004FF02008FFF77BBB374B1B6898067DF559
:104FB00057AD94F82431002B7DF46FAD334BC4F81A
:104FC0002C312D2384F83031FDF751BDD8B217F0C4
:104FD00045FD019B180A17F041FD78E509F0CEFC6C
:104FE00017F03CFD002017F039FD0BE54FF00808E5
:104FF000FFF755BBCA690B6A9A423CBFC8681218D2
:10500000D31AE9E51146FEF79DB91FFA88F89BF817
:10501000002098FBF2F825E7392017F049FD5FFAE8
:1050200088F017F01BFD4FEA182017F017FD3DE739
:10503000114690469646934602929146FEF782B9F3
:10504000134B9146B3F900306420FEF771B8114656
:105050009046FEF777B9114690469646FEF772B92C
:105060001146904696469346FEF76CB94FF0FF33D3
:1050700064E600BF50500020545000201C2A040851
:1050800089B5F8141F85EB51B0690020D85700206E
:10509000F8540020625000202DE9F04F2DED028BD6
:1050A000C74B1B7891B0072B069001F011830023AA
:1050B0000893C44B1B6805935D0500F1E286C24B63
:1050C000D3F8008018F0080F40F07986BF4BC04D30
:1050D000B3F800B0DFF81CA30793BE4BBE491E68AF
:1050E000B1F906907289914580F2A784BB4B4FF0CD
:1050F0007E521A60BA4F9AF90420B1F900C03C8B75
:105100009AF800009AF801E0002AACEB040314BFFF
:1051100001224FF0FF32002B40F3F184B3F5FA7F08
:10512000C0F2F3844FF4FA731B1A07EE903AF8EECC
:10513000E77AA445C5ED007A03DAF1EE677AC5EDAA
:10514000007AB1F902C0ACEB0403002B40F3E48415
:10515000B3F5FA7FC0F2E6844FF4FA731B1A07EE38
:10516000903AF8EEE77AA445C5ED017A03DAF1EE5C
:10517000677AC5ED017AB1F90430191B0029D8BF4F
:10518000E11AB1F5FA7F80F252847145D8BF4FF031
:10519000000E00F34E8402FB0EF207EE902AF8EEAA
:1051A000E77AA342059BC5ED027ABCBFF1EE677AB0
:1051B000C5ED027A13F48053049300F0ED80B9F545
:1051C000FA6F4A46A8BF4FF4FA62B2F57A7FB8BFC9
:1051D0004FF47A72A2F57A728249DFF81CE281FB01
:1051E0000230D317C3EB6013581C6FF0630C3EF909
:1051F00010003EF913E00CFB0323A0EB0E0003FBB1
:1052000000F381FB0321DB17C3EB61139E440FFA0C
:105210008EFE07EE90EA049BB8EEE78A85ED038ADE
:10522000002B40F075861BF0400F40F038856E4C27
:1052300018F0140F03D01BF4027F40F0F1866B4B83
:105240001B781BB17B8B4B4580F20B8594F8263085
:105250001BB11BF0030F41F00D8094F82C20FB7F55
:10526000002A40F08286B97F002900F0C980022917
:1052700000F0D287032940F0B78797F82010C1EBE0
:10528000411001EB8001C90089B20233DBB2002A70
:1052900000F0B187002900F0AE8755480068B1FBE7
:1052A000F0F10FFA81F9A4F85C90ABB307EE909A95
:1052B000F8EEE77AF7EE006A86EEA77A012BD5EDD5
:1052C000007AD4ED1C6A77EEE67A67EE877AC4ED51
:1052D000187A21D0D5ED017AD4ED1D6A77EEE67A01
:1052E000022B67EE877AC4ED197A15D0D5ED027AD4
:1052F000D4ED1E6A77EEE67A032B67EE877AC4ED6B
:105300001A7A09D0D5ED037AD4ED1F6A77EEE67AE2
:1053100067EE877AC4ED1B7A29490978092901F0DB
:105320006585B9F1000F71DD93B394ED1C7AD4ED6E
:10533000187A77EE877A012BC4ED1C7AC5ED007AD6
:1053400021D094ED1D7AD4ED197A77EE877A022B6D
:10535000C4ED1D7AC5ED017A15D094ED1E7AD4ED19
:105360001A7A77EE877A032BC4ED1E7AC5ED027A9E
:1053700009D0D4ED1F7A94ED1B7A77EE877AC4EDCD
:105380001F7AC5ED037A013B022BB8BF0223DBB2C3
:10539000002A18BF02233AE0798B8945C0F2708455
:1053A000B9F5FA6FD4BFC1EB0903C1F5FA634FF445
:1053B0007A7202FB03F2C1F5FA61B2FBF1F20BE77C
:1053C000294F0020D4860020B0690020105700200B
:1053D000645000201857002088A500209024002049
:1053E0000C7500201F85EB51C8220020901C002066
:1053F000C06800208C68002000C600200AD7233C2B
:10540000A4F85C108946002A00F0728102233278E9
:105410005FED066AB17807EE902AF8EEE77AB0EE13
:10542000007A67EEA67ADB4AF4EEC77AF1EE10FA5C
:10543000107840F3C084DFEDD86A37EEC77AB0EE5B
:10544000676AA7EE266AF0EE466A95ED007A9FED50
:10545000D36ADFF870E3DFF870C327EE066AF0EE78
:10546000C65ACEED005A8CED006A99B107EE101ABB
:10547000B8EEC75A9FEDCA7A66EE064A25EE075A7D
:10548000B7EE007A37EE457A64EEA54AA5EE247AA7
:1054900026EE076A9FEDC37A727926EE877A27EEA9
:1054A000067AAAB1DFEDBE6A9FEDBF6A65EEA65A25
:1054B00006EE902AF8EEE66A66EEA56AF4EEC66A93
:1054C000F1EE10FA40F363869FEDB86A27EE067A94
:1054D0000C289FEDB78ADFEDB76ADFF8F08200F0A5
:1054E0003186B4EEC87AF1EE10FA98BFB0EE478A72
:1054F000B4EEE68AF1EE10FAB8BFB0EE668A88ED37
:10550000008A002B00F0E680B0EE007AF4EEC77A55
:10551000F1EE10FA05DD37EEC77ADFED9F6AE7EEB0
:10552000267A95ED017ADFED9D6A27EE267AF0EE78
:10553000C75A8CED017ACEED015A99B106EE901A58
:105540009FED976AF8EEE66A27EE075A66EE866ADE
:10555000B7EE006A36EE666A25EE255AA6EE856A33
:1055600027EE067ADFED8F6AB27967EEA67A67EEEC
:10557000877AFAB107EE102AB8EEC77A9FED886AEB
:10558000DFED896A27EE257A27EE067AB4EEE67A11
:10559000F1EE10FA00F3F785B5EEC07AF1EE10FAED
:1055A00001F10281B7EE006A36EE477AC6EE076A6D
:1055B00067EEA67A0C2800F0A685DFED7D6A9FEDE8
:1055C0007D7AF4EEE67AF1EE10FA88BFF0EE667AB4
:1055D000F4EEC77AF1EE10FAB8BFF0EE477A012B7D
:1055E000C8ED017A76DD7378DFED6D6A07EE903AEB
:1055F000F8EEE77AB0EE007A67EEA67A737AF4EE08
:10560000C77AF1EE10FA05DD37EEC77ADFED626A90
:10561000E7EE267A95ED027ADFED606A27EE267ACC
:10562000F0EEC75A8CED027ACEED025A9BB106EE2F
:10563000903A9FED5B6AF8EEE66A27EE075A66EE4F
:10564000866AB7EE006A36EE666A25EE255AA6EE41
:10565000856A27EE067ADFED536AF37967EEA67A5C
:1056600067EE877AFBB107EE103AB8EEC77A9FED86
:105670004C6ADFED4D6A27EE257A27EE067AB4EE06
:10568000E67AF1EE10FA00F37A85B5EEC07AF1EE23
:1056900010FA01F18580B7EE006A36EE477AC6EE61
:1056A000076A67EEA67A0C2800F02585DFED406AD0
:1056B0009FED407AF4EEE67AF1EE10FA88BFF0EE54
:1056C000667AF4EEC77AF1EE10FAB8BFF0EE477AD8
:1056D000C8ED027A092800F0048597F82150002DC2
:1056E00040F0B984344BD3F80080002384F82C3088
:1056F00018F0200F06D0079B1B8803F03003002B07
:1057000040F040822D4D2E4F95F82420DFF8C080C8
:10571000DFF8C0A0531E082B00F20781DFE813F06A
:105720002301A101A90005015C000900A3010501F5
:10573000B60198F80030002B40F031852B68297AAB
:105740004FF4807203EB0121002025F06FF92B7AD2
:105750000133DBB2022B2B7240F05881002025F080
:10576000A5F9002025F0A2F9FF2025F09FF900F00F
:105770001F00052801F01B8415F030FDEE68002E97
:1057800000F04A8400222B6969680120B04795F82F
:105790002420BFE7294F0020D7A368416F12033BA5
:1057A0000AD7233C00004843A4707D3F0000C84254
:1057B00000C0F94400C0F9C4B0690020D4A300209F
:1057C000F8C50020C0240020B42400209824002024
:1057D000E8540020886002404FF40071286815F0FA
:1057E000AFFC012800F01E85C0F03286022840F090
:1057F0000D8115F01BFD15F0F1FCEE68002E00F098
:105800000B84002210462B696968B04795F8242064
:1058100080E71021CF4815F093FC8346002840F024
:10582000F38001217F2022F09BFC0128814640F07B
:10583000EB805846022122F093FC002801F05B82A5
:10584000012840F0E18016213A2022F089FC431C17
:105850009B02EB6315F0EAFC3068F4F76FFA002165
:105860000A2015F08BFC002840F06487032385F89C
:10587000243010210CA815F063FC002840F0C680ED
:105880009DF83A209DF839009DF83C109DF83D3078
:105890009DF83B60120442EA00620A431B019DF836
:1058A0003E109DF83100DBB243EA111342EA0622B2
:1058B00003F5FA636A632B879DF832209DF8383030
:1058C00042EA002201F00F01180903F00F0385F8E6
:1058D0003A106A859DF830109DF8332085F83230F3
:1058E0009DF8343085F8281085F82C209DF8351067
:1058F0009DF8362085F82D309DF8373085F830300A
:1059000085F8310085F82E1085F82F2015F08EFCD3
:10591000AB7E002B00F00D818F4825F037F9002376
:1059200004222B6285F824200323DBB2022B73D9D7
:10593000042A00F0BE80082A00F0BB80874B1B7849
:1059400023B9874EB278002A40F09685069806F073
:105950005DFD844B1B78072B00F0158511B0BDEC65
:10596000028BBDE8F08F804E3068F4F7E7F9002134
:10597000084615F003FC814615F058FCB9F1010FFB
:1059800044D130684FF0000B85F819B0F4F7D6F920
:1059900040F2AB11082015F0F1FB052800F0A684B9
:1059A000012800F0AA8615F041FC6B7E002B01F067
:1059B000FA82022385F824303068F4F7BFF96B7E51
:1059C000022B14BF4FF000094FF08049002137200F
:1059D00015F0D4FB4946292015F0D0FB814615F07F
:1059E00025FCB9F1000F11D16B7E022B00F09286DD
:1059F00085F81A903068F4F7A1F90021092015F014
:105A0000BDFB00283FF405AF15F010FC95F82420ED
:105A1000531EDBB2022B8BD8544B69691B685B1A8F
:105A2000C82B88D915F0DAFB95F8242080E74FF4CD
:105A3000FA71A1EB0E0EFFF7AEBBB9F5FA6FC0F22B
:105A40002281337AC3F1640307EE903A9FED487ADE
:105A5000484BF8EEE77A67EE877AC3ED007AFFF7F6
:105A600049BB414EA8E70826FF2025F01FF8FF2874
:105A700000F09484013EF7D16B693A68FA3393429F
:105A8000C4D215F0ABFB95F8242043E6FF2025F0A7
:105A90000DF8FF284FF0080606D0013EECD0FF209D
:105AA00025F004F8FF28F8D115F0C0FB042385F891
:105AB0002430314D16F00EF86B78022B00F00D8675
:105AC000032B7FF43BAF41F2B813EB5C002B41F0AA
:105AD000338141F2A403EB5C002B41F0288141F2B9
:105AE000E803EB5C002B41F02C8141F22C13EB5CC2
:105AF000002B3FF423AF21481DF032F91EE7A4EB41
:105B00000C03B3F5FA7FBFF60DAB9842FFF60CAB72
:105B1000DFED1B7AFFF70DBBA4EB0C03B3F5FA7FA7
:105B2000BFF61AAB9842FFF619ABDFED157AFFF717
:105B30001ABB0D4E3068F4F701F94FF400711020D4
:105B400015F01CFB064615F071FB002E3FF4E4AE89
:105B500097E700BF14A40020003C0040CCC2002006
:105B60004D760020294F0020EC540020F8C500207D
:105B70000AD7233C902400204C8F002078A00020DE
:105B800000000000C54B1B78D8077FF5BBADC44BA8
:105B9000C44AB3F90430DFEDC47A82FB0312DB1789
:105BA000C3EBA2031BB208EE103AB8EEC88A28EE87
:105BB000278AB0EE480AF5F75BF9F0EE408AB0EEBE
:105BC000480AF5F7DBF8B94BD878002800F03286A0
:105BD000B749B4F98A20B1F9023044F250659B1AF2
:105BE000AB4241F3CD80A3F50C43A03B45429D421F
:105BF00001F3C3808342A8BF0346B1F90010B4F992
:105C0000886013448A1B44F250611BB28A42A4F894
:105C10008A3041F3BD80A2F50C42A03A954203DCE4
:105C20009042A8BF10460546721912B207EE902A9C
:105C300007EE103AF8EEE77AF8EEC76A27EEE87A50
:105C400060EE277AA0EE267A9A49A4F88820E8EE3A
:105C5000A67ADFED996A27EE267A67EEA67A00F03B
:105C600005BE964B1B78012B00F08283192B00F0A8
:105C70007F830E2B3FF4EAAA082B3FF4E7AA7CE3CC
:105C80001A46FFF798BB307AA9EB020303FB00F337
:105C9000C2F5FA6293FBF2F3C3F16403D4E6804BDE
:105CA0008049B3F90430864CDFED7F6A22889FED8E
:105CB000857A81FB0301DB17C3EBA1039B1A1BB29F
:105CC00007EE903AF8EEE77A67EEA67A77EE876A03
:105CD000BDEEE66A16EE103A2033402B40F2718397
:105CE000DFED796ABDEEE77A17EE103A2033402BEC
:105CF00000F264839FED757AF4EEC77AF1EE10FA44
:105D000041F33780DFED725A9FED726A01E0F0EEE9
:105D1000477AF4EEC67AF1EE10FA37EEE57AF6DC61
:105D2000DFED6D7AB4EEE77AF1EE10FA41F11D8005
:105D3000DFED675A9FED696A01E0B0EE677AB4EE75
:105D4000C67AF1EE10FA77EE257AF6D49FED5D7AF9
:105D5000F4EEC77AF1EE10FA00F3C3829FED607A99
:105D6000F4EEC77AF1EE10FA44BF9FED5B7A77EE5E
:105D7000677A67EEA75A9FED5B5A9FED5B6A9FEDCE
:105D80005B7AA5EE856A27EEA55AA5EE867AE5EE42
:105D9000077A95ED016AD5ED005A27EEC67A65EED1
:105DA000A77AA5EEA67AE6EE267A85ED007AC5ED0D
:105DB000017AFFF73DBAF0EE676AFFF746BB4C4D3C
:105DC0004C4BD5ED027A0793B2EE0E7AF0EEE76A0D
:105DD000F4EEC76AF1EE10FAB3F800B0304B42D5DA
:105DE0001BF0040F3FD0B3F904302E4A4249DFF8CC
:105DF0001CA1098882FB0302DB17C3EBA2035B1A19
:105E00009BB21AB212F1B30FBCBF03F5B4731AB24E
:105E1000B32AC8BFA2F5B4732049C8BF1AB29AF812
:105E200004300978002B4FF6FF7318BF01230C07CD
:105E30007FF553A93149096812FB03F3097E304A03
:105E40009BB211FB03F382FB03121A44DB17C3EB73
:105E5000221307EE103AB8EEC77A77EEC77AC5ED8F
:105E6000027AFFF73AB9B3F904300E49224ADFF853
:105E70009CA081FB0301DB17C3EBA1031380FFF799
:105E80002CB920488368002B3FF419A900F1440184
:105E900098471D4B1B680593FFF711B991560020D9
:105EA000C05600206766666635FA8E3C584C002066
:105EB000B44C0020B0240020CDCCCC3DC4680020E0
:105EC000C8220020DB0FC93F00000000DB0F494063
:105ED000DB0FC940E4CB1641DB0F49C0E4CB16C150
:105EE000DB0FC9BF92E741B99730083C15A82ABE1D
:105EF0006450002010570020D44C0020145700207C
:105F0000898888880CBA0020D48600208C680020FC
:105F10001D21C848F5F784F800283FF484A9C64B32
:105F2000DB78002B7FF47FA9DFEDC47AC44938EE1B
:105F3000678AC4F5FA62FDEEC87A12B2CDED097A2D
:105F4000BDF924301B0381FB0301DB17C3EBA11355
:105F500002FB03F343F30F33234407EE903AB8EE0A
:105F6000E78A85ED038AFFF75EB9B649B148D1F8F3
:105F7000EC10006844F6206E7145A8BF7146B1F57B
:105F80007A7FB8BF4FF47A7189B2C006E18540F1DB
:105F9000B1810498002840F00B84AB48D0F800A0F1
:105FA000BAF936B0DFF898E2206BD5ED037AAEFB94
:105FB00001E14FEA911E642191FBFEF11429BDEE2F
:105FC000E77A04EB400CA8BF14210130884220631B
:105FD00017EE109AA4BF0020206304EB4000ACF839
:105FE0003490B0F9341007EE101AB8EEC77A77EE95
:105FF000C77AFDEEE77ACDED047ABDF9100080EAAC
:10600000E071A1EBE071594500F3A0868F494FF094
:106010007E500860FFF727B995F82420FFF77ABB78
:106020008B4B1B7813F0100300F074812279A36866
:1060300095ED017A002A0CBF01224FF0FF3203FBDD
:1060400002F307EE903AF8EEE77A77EE877AC5ED3D
:10605000017AFFF7F4B81E217648F4F7E1FF002833
:106060003FF440AB079B1B885E063FF53BAB94F8C3
:106070008030AB4240F00687764BD4ED217AD3EDE9
:10608000006A98ED025ADFED745A9FED746A27EEAC
:10609000C57A68EE277AA8EE267AE5EE267AB4EE7F
:1060A000E57AF1EE10FA88BFB0EE657AB4EEC67A02
:1060B000F1EE10FAF4EEE57AB8BFB0EE467AF1EE02
:1060C00010FA88BFF0EE657AF4EEC67AF1EE10FAB7
:1060D000B8BFF0EE467A88ED007AC8ED027AFFF795
:1060E00001BBFDEEC87A5E4A17EE903AA2F8049022
:1060F000D380FFF7F2BABDEEE77A594B17EE102ABC
:106100009A80FFF7D3BA9FED547ADFED546A544971
:10611000F4EEC77AF1EE10FA98BFB0EE677AFDEEB2
:10612000E77AB4EEE67AF1EE10FA17EE902AB8BFED
:10613000B0EE667A012B88ED017A4A803FF753AAC8
:10614000FFF7CBBAB4EEC87AF1EE10FA98BFB0EE12
:10615000478ABDEEC77AB4EEE68ADFF804A1F1EE15
:1061600010FA17EE102AB8BFB0EE668A88ED008AE2
:10617000AAF80020002B7FF4C7A9FFF7AEBADFED25
:10618000396AFFF78EBADFED376AFFF711BAF7EE1B
:10619000005A75EEE66A85EEA66AFFF797B9324BAC
:1061A000596809057FF5C7AB4FF40062DA60DAF889
:1061B00000202E4B22F00102CAF800201A89D207D3
:1061C00000F19E8023F00EF90028FBD1274A938826
:1061D00023F002031B041B0C938098F80030002B63
:1061E0007FF4BCAAFFF7AABA214902334988DBB27F
:1061F000002A7FF44FA8B4F85C9009F1FF390FFA38
:1062000089F9B9F1000FA4F85C903FF78DA8002A36
:106210007FF4FCA8FFF76CBAE18D01F57A7189B2C1
:10622000FFF733B86B693A6864339342FFF4E1AA2D
:10623000FFF7ECBBD8660020404B002000007A44FA
:10624000D34D62106C09002014570020300000204C
:10625000915600202C00002000C0F94400C0F9C471
:106260002C4F00200000C84200600240003C00406B
:106270003CC30020894ADFED8A7A92ED080A09932F
:10628000B4EEE70AF1EE10FA40F2808227F0B0F99E
:10629000D4ED0A7A20EE270A27F014F9B0F5617FD1
:1062A000099B00F38E8207EE900AF8EEE76ADFEDB5
:1062B0007D7A66EEA76A07EE903AB8EEE77AFDEED1
:1062C000E67A17EE903A2033402B40F2CC869FEDD1
:1062D000760A27F0F7F800B207EE900AB8EEE77AF0
:1062E00056E29FED727A77EE677A42E585F819906B
:1062F000FFF759BB0598C0003FF54BAEFEF7B3BFA3
:106300009A891A89D207FBD423F06CF800287FF40D
:1063100059AF5BE79AF80320002A40F0B382B4F942
:106320000CE09AF80210A9EB0E0383EAE370A0EBED
:10633000E370884240F3348503EBD37301225B1092
:10634000E36184F820202275A3689E44BEF5FA6FAD
:10635000A8BF4FF4FA6EBEF57A7FB8BF4FF47A7ECD
:1063600007EE90EAF8EEE77AC5ED037AFEF767BF2D
:106370004F4B9B7B002B7EF469AF4E4A0023AB60F2
:106380009360FEF763BFF2F72BFF089A4A4B801A1F
:10639000988011B0BDEC028BBDE8F08F2B6A002213
:1063A000012B2A7641F28980EA69013B01322B6296
:1063B0000823EA6185F82430FFF77BBBDFED3A7AEA
:1063C000E7E4F4EEC77AF1EE10FA40F3E485DFED8E
:1063D0003B5A9FED3B6A01E0F0EE476AF4EEC66A75
:1063E000F1EE10FA36EEE57AF6DCDFED366AB4EE61
:1063F000E67AF1EE10FA40F1D285DFED305A9FEDEA
:10640000326A01E0B0EE667AB4EEC67AF1EE10FAC6
:1064100077EE256AF6D49FED2D7AF4EEC76AF1EE99
:1064200010FA40F398819FED217A77EE666A66EE66
:10643000A65A9FED275A9FED276A9FED277AA5EE72
:10644000856A26EEA55AA5EE867AE5EE076A49E446
:1064500014F0ECFEEE680423002085F82430287642
:10646000002E3FF426AB2B692A686968B04795F87F
:106470002420531EFFF7CDBA184F3B78013B0A2B5F
:106480007BD8DFE813F08D027F02480233021C0242
:10649000E802D202BF029C0203032D00945B00209D
:1064A0008FC2753CD06D393A00000000DB0F4940C7
:1064B0005C6F0020982400202C4F0020DB0FC94087
:1064C000E4CB1641DB0F49C0E4CB16C1DB0FC93F5B
:1064D00092E741B99730083C15A82ABE4C760020B7
:1064E000022A38D1C34BDFF848831B78002B41F0D8
:1064F0007E80D8F8005045B32B7833B395F8282028
:10650000002A40F034812B7EAA6385F83C200422C7
:1065100085F8282013F008036A6AEA622A6303D028
:10652000B54A41F29413D3586B634FF00009C5F894
:106530002490C5F80890C5F80C90284621F0C2FDBB
:106540000523C5F8409085F8283000220423C8F8B8
:10655000002088F81430A94BA94A5B681268C83338
:10656000934204D320F07CFE002800F0D281B27860
:10657000032A01F06F8001233B70022A00F0F780AC
:10658000F378002B3FF4E2A99E4B1B68D90440F13D
:10659000B0859D4B9B8807EE903AF8EEE77A9B49D1
:1065A00091ED012AD1ED022A91ED033AD1ED043AA1
:1065B00091ED054AD1ED064A91ED075AD1ED085A01
:1065C00091ED096AD1ED0A6A91ED0B7AB4EE672A72
:1065D000F1EE10FAF4EE672A14BF01230023F1EE66
:1065E00010FAB4EE673A18BF43F00103F1EE10FA67
:1065F000F4EE673A18BF43F00103F1EE10FAB4EE7F
:10660000674A18BF43F00103F1EE10FAF4EE674A4F
:1066100018BF43F00103F1EE10FAB4EE675A18BF49
:1066200043F00103F1EE10FAF4EE675A18BF43F09D
:106630000103F1EE10FAB4EE676A18BF43F00103EC
:10664000F1EE10FAF4EE676A18BF43F00103F1EEC1
:1066500010FAB4EE677A18BF43F00103F1EE10FAB6
:1066600018BF43F00103002B40F07B8491ED007ACA
:10667000B4EE677AF1EE10FA40F07384604DD4F80E
:1066800090102B68994200F273843B78012B3FF401
:106690005DA994F88C20002A3FF458A90B2B0DD843
:1066A00001229A4040F6030112EA01060BD112F4CE
:1066B000C06F03D0093B012B40F2E9874F4B2A689A
:1066C0005A600B233B70002384F88C30FFF73EB9EF
:1066D000F2F786FD0890FEF7ECBCAB784FF0010BAB
:1066E000072B3FF62BA9DFE813F0E401E202920248
:1066F00087022102CC02D602FD01594604220CA8D1
:1067000024F094F99DF83330AB2B04BF02236B7651
:10671000FFF749B93068F3F711FB49463A2014F006
:106720002DFD4946834604220CA824F07FF9BBF1D5
:10673000000F07D014F07AFD14F050FD95F82420D6
:10674000FEF7E8BF14F072FD0C9B1BBAC3F3807315
:10675000AB76FFF74FB99FED2E7AF4EEC76AF1EEF4
:1067600010FA44BF9FED2B7A77EE666A5FE6224A05
:1067700041F2B513D35C002B00F09B8794F88C306A
:1067800001223A70002B3FF4E1A89CE79FED227AAA
:10679000D5ED037A77EE877AC5ED037AFEF75DBD16
:1067A000F7EE006AFEF77DBFF7EE006AFEF700BF66
:1067B0001A48D0F800A0BAF836B04FEA5B0BFFF7E2
:1067C000F1BB07EE903ADFED166AB8EEE77A66EEB7
:1067D000A65A9FED145A9FED146ADFED147AA5EEC8
:1067E000856A26EEA55AE5EE867AE5EE276A26EE5C
:1067F000870A6EE5646800204C8F00207C680020CA
:10680000F8C50020D4860020946400209C630020FA
:10681000DB0FC9BFDB0F49C0000000001457002088
:1068200084F9223F92E741B99730083C15A82ABE67
:1068300034760020AD4B9FEDAE6AB3F90020B3F97A
:106840000230AC4907EE902A06EE903AF8EEE77A6D
:10685000F8EEE66A27EEE87A60EE277AA0EE267A6E
:10686000E8EEA67A27EE067A67EE867ABDEEC77A5C
:10687000FDEEE77A17EE102A17EE903A0A804B8069
:10688000FEF740BFB4F90C209AF80210A9EB020EF3
:106890008EEAEE70A0EBEE70884240F38D82914557
:1068A000C8BF494207EE901AF8EEE77A012037EEAA
:1068B000888A2361207585ED038AFEF7C0BC20F02D
:1068C00095FC8D4B002102208DE80300A3F1080206
:1068D000029148201DF04CFDD8B9884BB278186061
:1068E0004FF0FF31596006233B7046E620F07EFCF6
:1068F000834A0292A2F10C03292101930091A2F193
:106900000A035021163A49201DF032FD002800F0FC
:10691000B985B27831E6DFF8E48120F067FC794A86
:10692000D8F80430126864339342F2D2402020F049
:1069300041FC0028EDD1D8F80030734DDFF8CCA130
:106940004FF040090FE020F0C7FCDAF80020D8F83B
:106950000030013A0133B9F10109CAF80020C8F842
:10696000003000F07186EB5C1846002BEBD1002361
:106970004FF0FF32C8F800300423C8F804203B7001
:10698000B278FAE5022A00F017845E4B5B491B6877
:106990004B605E4800230B60032103603970ECE517
:1069A0005B4B1B78DB077FF5E8AD802021F080FA98
:1069B00008B108F055FA1DF0C5FDB278DDE51A20E2
:1069C00024F076FDD0B1534B1B88BBB9524B452008
:1069D0001D6820F081FC0E2020F07EFC28461CF073
:1069E000F9FB069D28461CF0F5FB4C4A4FF48051FC
:1069F0000A23284611803B701CF09CFC1CF0E2FF2F
:106A0000B278BAE520F0F2FB1CF0FCFF002880D041
:106A100020F026FC00283FF47CAF404BB2784FF4C6
:106A2000805119800A233B70A7E520F0DFFB3C4B27
:106A3000002105208DE80300A3F1080202915320F4
:106A40001DF096FC00287FF464AF2C4BB2781860E0
:106A500008233B7091E520F0C9FB324A0292A2F173
:106A60000C03072501930095A2F108030021143AB5
:106A700047201DF07DFC00287FF44BAF1F4B3D707D
:106A80004FF0FF3283E80500B27876E5264B1B789D
:106A9000002B00F0A0821A2024F00AFD002840F00C
:106AA0009A8294F88C30002B40F0958209233B7039
:106AB000A4E700230DF1300949461846092214F0D5
:106AC000C3FB01287EF43AAF0C9B93F8FE21552AB4
:106AD00000F0878241F2B41202210123A9546B70A5
:106AE000FEF72CBF03236B70FEF728BFB44C0020C9
:106AF000CDCCCC3DB024002018FE03087C680020DB
:106B00003AFC0308F8C50020C4FB03089C7600206B
:106B100020660020E0660020E4660020CC660020AD
:106B20007CFE030834FE0308186900202A782B7DB8
:106B3000BF4EDFF818A3032A14BF4FF480778027D5
:106B4000002B45D0012BFBD1BA4B326819686B681A
:106B50004FEA412E4FF000094FF0FF31B1FBFEFE2E
:106B60001EEB030049F100014FF00009494502F115
:106B7000020208BF904238BF03EB0E02AE4902206A
:106B800014F07EFE032800F22A8201A353F820F0BD
:106B90003D590108A16B01083D590108A16B01088D
:106BA0006968D5F808E02B69AEEB01029A4284BF10
:106BB000E9602A61032836D00EF10103B3FBF7F236
:106BC00007FB12320AB13B449B1A00226B602A7504
:106BD000326851460232002014F052FE032800F2BF
:106BE000FE8101A353F820F03D590108EB6C010828
:106BF0003D590108276C010841F27013EB5C002B32
:106C00003EF49CAE8D481CF0ABF8FEF797BE8C4B63
:106C100000930320A870302305228A4987481CF07E
:106C200021F9FEF78BBE2B690622652BAA7032D99B
:106C30002A78032A14BF6FF0FF026FF07F02A3F1DE
:106C4000650303EA020303F1010314BF4FF48072EA
:106C500080229A422B611ED23268EE6802329F195E
:106C6000974280F0CE84784A6E60D16FAF6049025F
:106C700003FB01F30521166042F81C3C42F8183C66
:106C8000A970AA687149012014F0C2FC012840F0E3
:106C900025840623AB700021684814F081FC01288C
:106CA00040F01C84AB780133DBB2AB7018E50DF11A
:106CB000300941F2FC164946A8590023092214F074
:106CC000C3FA01287EF43AAE00230C9A2B70B2F876
:106CD0000B30B3F5007F00F0298441F2B412032198
:106CE0000123A9546B70FEF729BE6B6885F814B0B8
:106CF0000133AB6028E704212C2021F031FA032175
:106D000083464E2021F02CFA0C210490362021F0ED
:106D100027FA049B421C02339A4009FA0BF9A2FBA2
:106D20000901420A42EAC152EA63FEF793BD4848AC
:106D30001CF016F8FEF7D3BE46481CF011F8FEF71B
:106D4000C8BE45481CF00CF8FEF7CFBEBAF83810A4
:106D50009FED427A07EE901AF8EEE77A404967EE27
:106D6000877AC1ED007AFEF77EBAF0EE477AFEF739
:106D7000EDBFB0EE677AFEF7D3BF2B46FEF73DBFFF
:106D8000384DAB42BCBF03F50C43A033FEF72EBF1A
:106D900034498A42BCBF02F50C42A032FEF73EBF26
:106DA000237D002B3FF4D0AA2F4B84F820201B68B2
:106DB0002275A361FFF7C8BA217D19B12A4923754D
:106DC0000B68A361A3681344B3F5FA6FA8BF4FF42F
:106DD000FA63B3F57A7FB8BF4FF47A7307EE903A4F
:106DE000F8EEE77AC5ED037AFEF729BA95ED000AC9
:106DF0000493059226F066FB1C49DFF874E0D1F895
:106E0000EC10DFF870C0059AACF800008EFB013E74
:106E1000C917C1EBAE1107EE901AF8EEE77A049BA2
:106E2000FDEEE77A17EE901AACF80210FEF779BA89
:106E300054A100205CA10020548F0020BCA00020A1
:106E4000E11B0308282A0408E0A00020508F00203E
:106E5000F09F002004A1002034A000206F12833A8C
:106E600030000020B0B9FFFFB85600206C090020A8
:106E7000D34D62102C4F002035FA8E3CDB0FC93FFA
:106E80000000000007EE905A5FED056A1FED057ADD
:106E900084F88050F8EEE77A67EEA67A77EE876A94
:106EA000BDEEE66A16EE103A2033402B40F23181F7
:106EB0005FED0D6ACB4BBDEEE77AC3ED006A17EECE
:106EC000103A2033402B00F221819FEDC77AF4EE77
:106ED000C77AF1EE10FA40F3CD83DFEDC45A9FED8F
:106EE000C46A01E0F0EE477AF4EEC67AF1EE10FAE9
:106EF00037EEE57AF6DCDFEDBF7AB4EEE77AF1EE55
:106F000010FA40F1B483DFEDB95A9FEDBB6A01E09E
:106F1000B0EE677AB4EEC67AF1EE10FA77EE257A23
:106F2000F6D49FEDB67AF4EEC77AF1EE10FA40F39C
:106F300037819FEDAD7A77EE677A67EEA75A9FEDBE
:106F4000B05A9FEDB06A9FEDB07AA5EE856A27EE44
:106F5000A55AA5EE867AE5EE077AC4ED217AFFF709
:106F600090B8AA4B1B6803F59C530833C4F89030C3
:106F70003B78012B7EF4EAAC94F88C30002B7EF445
:106F8000E5AC032A00F07C831DF0DCFA012384F8D1
:106F90008C30FEF7DBBCB0EE667AFFF726BAF0EE77
:106FA000476AFFF738BA85F82430FEF7C7BC974B1D
:106FB000EE681B686B61072385F82430002E3EF4D1
:106FC000BDAC2B692A6869680120B04795F8242078
:106FD000531EFEF7AABC06981CF0ACF90EE52B7DFB
:106FE000AEE593F8FF21AA2A7FF474ADD3F8C61159
:106FF00049B193F8C221A2F10B0001282DD902F06A
:10700000F702062A29D0D3F8D61149B193F8D22134
:10701000A2F10B00012820D902F0F702062A1CD0A9
:10702000D3F8E61149B193F8E221A2F10B0001284F
:1070300013D902F0F702062A0FD0D3F8F61100296F
:107040003FF448AD93F8F231A3F10B02012A04D9C1
:1070500003F0F703062B7FF43DAD41F2FC12012350
:10706000A950AB7025E6DFED607AF4EEE76AF1EE49
:1070700010FA40F32483DFED5D5A9FED5D6A01E075
:10708000F0EE676AF4EEC66AF1EE10FA76EEE57A93
:10709000F6DCDFED586AF4EEE67AF1EE10FA40F134
:1070A0000B83DFED525A9FED546A01E0F0EE667AF1
:1070B000F4EEC67AF1EE10FA77EEA56AF6D4DFEDBB
:1070C0004F7AF4EEE76AF1EE10FA05DDDFED467A6D
:1070D00077EEE66AFFF77BBBDFED4D7AF4EEE76A09
:1070E000F1EE10FA44BFDFED437A77EEE66AFFF780
:1070F0006EBB484B1B78002B40F0C081464B1B8B6E
:1071000007EE903AF8EEE77AFFF749BADFED437AF7
:1071100023E7F4EEC77AF1EE10FA40F38B82DFED4D
:10712000335A9FED336A01E0F0EE476AF4EEC66A27
:10713000F1EE10FA36EEE57AF6DCDFED2E6AB4EE0B
:10714000E67AF1EE10FA40F17282DFED285A9FEDF7
:107150002A6A01E0B0EE667AB4EEC67AF1EE10FA71
:1071600077EE256AF6D49FED257AF4EEC76AF1EE44
:1071700010FA40F396819FED1C7A77EE666A66EE10
:10718000A65A9FED1F5A9FED1F6A9FED1F7AA5EE2D
:10719000856A26EEA55AA5EE867AE5EE076A89E6A7
:1071A0009FED1B7AF4EEC77AF1EE10FA44BF9FED23
:1071B000117A77EE677AC0E6DFF8648098F81430C9
:1071C000052B3FF6A6AB01A252F823F03974010853
:1071D00013690108BD73010883720108B9720108BF
:1071E000777401082C000020DB0F4940DB0FC940F9
:1071F000E4CB1641DB0F49C0E4CB16C1DB0FC93F1E
:1072000092E741B99730083C15A82ABEF8C500207E
:10721000DB0FC9BF58700020307000200000000054
:1072200034760020D8F8042092F91A104D1C5C46E0
:107230000AD0AF4B01F5817103EB0113FF20D9791F
:107240006FF30001D971907692F91B10481C15D08C
:10725000A74D01F5817105EB011305EB0115DB79F4
:10726000E979C3F34503012BC6BF03F1FF33DBB25A
:107270000023FF2063F34601E971D076032388F8E9
:1072800014309C48D8F804100378002B7FF441ABED
:10729000002900F0208291F82830002B7FF439ABD0
:1072A0002838442225F09AFF0021D8F804001BF06A
:1072B0003DFD0023C8F80430D8F81050DFF858A27C
:1072C000DFF858E2DFF858C28B4B05F1010BAAFB3F
:1072D0000B59ACFB0B5CAEFB0BE50595874DA5FB95
:1072E0000BE50795059D0FCBAD090995079D4FEA65
:1072F000D90E4FEA5C1C6D0B0DF13009CDF810C0B2
:107300000595AAFB0EC5CC46ACE80700049A8CF89C
:107310000030AAFB02020998D20801460792ED0844
:10732000AAFB0112059905EB8505AEEB4505AAFB05
:10733000011AD108079A079501EB8101049DA0EB82
:1073400041014FEADA0A059802EB8202A5EB4202FC
:107350000AEB8A0A664D41F2A4030EEB8E0EA0EBF7
:107360004A0A0798EB5CABEB4E0B303001F1300E64
:107370000BF1300B30320AF1300A01218DF8360062
:107380008DF837B08DF835208DF834E08DF833A0C6
:1073900088F81410002B00F03A8141F2E803EB5C0E
:1073A000002B00F0338141F22C13EB5C002B00F03A
:1073B0009081042388F81430FFF7ABBA504DDFF802
:1073C0006491DFF864A1A3460BAA2946D8F804000B
:1073D00014F07AF8012849464FF0030240F0768114
:1073E0000B9C2046002C3FF41DAF2378002B3FF46C
:1073F00019AF28F0E4F9032251460028E4D104F142
:10740000080028F0DCF903460028DDD154F8030F0A
:107410000C9022798DF834200CA88DF8353025F0A9
:10742000B5FED8F81030984203D90CA825F0AEFE6E
:107430000346C8F81030C7E72D4D6B78032B7FF457
:1074400068AA41F2A4020123AA5C88F81430002A39
:1074500000F0588141F2E802AA5C002A00F0438162
:1074600041F22C13EB5C002B00F03C81002388F8E8
:107470001430FFF74EBAB278FFF787BADFED217A02
:10748000FFF78DB8204B1B6813F080031CD01F4BF7
:10749000B27818604FF0FF31596005233B70FFF759
:1074A0006CB89FED1B7AF4EEC76AF1EE10FA44BF98
:1074B0009FED187A77EE666A61E600F0BE800423DD
:1074C00085F82430FEF7A0BA1049B2780B604FF06F
:1074D000FF334B6007233B70FFF74FB802287EF461
:1074E0002DAA41F2B4120123AB546B70FEF726BAF9
:1074F0004C8F00202CA10020502A04085917B7D126
:107500003C76002000000000D48600207C6800202B
:10751000DB0FC9BFDB0F49C0CDCCCCCCD34D621043
:107520001F85EB513C2A0408402A0408137C022BD7
:107530007FF4D3AB92F8FE31552B7FF4CEAB92F8AB
:10754000FF31AA2B7FF4C9ABB2F80EE0AF596E4BF6
:1075500077441F60567B41F21021731E7F2B6E50C3
:107560003FF6BBAB734236EA03037FF4B6AB73025C
:1075700041F21821013B6B50D08A00B9506A63492F
:1075800041F20423E850B2F811305B0103F2FF131B
:107590005B120B60B2F8131001B9116A0EEB030C09
:1075A00040008444A1EB0C0141F2082E40F6F47C2B
:1075B000B1FBF6F1614545F80E1076D94FF6F47639
:1075C000B1427FD903212970D26A51493B44184402
:1075D00041F20C2641F21C230978A851EA5009B95E
:1075E0001AF01CFFAB780133AB70FEF7A7B900218E
:1075F000D8F800001BF09AFB00287EF4A6AFFFF736
:1076000088B91AF039FF2B69FFF72DBB0B4603EB46
:10761000031305EB830000F585503E4B009349466C
:107620003C23202204301BF01DFCFFF772B9F0EE62
:10763000476A98E5B0EE667A7FE513F011FD0228FF
:107640007EF4E4A9FEF7E0B9EB5C002B7FF461A9BE
:10765000FFF78DB9304D286805F07EF92F4B1B7868
:107660000022022B2A6008D0B278FEF784BFF0EE29
:10767000477A56E4B0EE677A3DE407F009FCF3E799
:10768000802020F015FC00287EF460A97CE44520D1
:107690001FF022FEFF201FF01FFE21481FF0F2FD09
:1076A00030461FF019FEFFF709B801232B70FFF7D2
:1076B00014BB0222FEF764BFF0EE676AFFE4F0EE4F
:1076C000667AE6E402222A7000227EE75C46FFF733
:1076D00020B902239BE71AF0A1FE00287FF4E4AD55
:1076E000FFF717B90223442202FB035303F5855029
